; -----------------------------------------------------------------------------
; Z80 Second Processor OS v1.20 (c) Acorn
; reverse engineered by Eelco Huininga using phpDisassembler v1.08 (using 6502 architecture)
; DOS Filename   : H:\Backup\Acorn\projects\disassembler\OSMv200.rom
; Acorn filename : $.OSMV200
; Load address   : Unknown
; Exec address   : Unknown
; Length         : 00002000
; -----------------------------------------------------------------------------

copro_register1                         = $00
copro_register2                         = $01

.
0000  00                 .       NOP
0001  00                 .       NOP
0002  00                 .       NOP
0003  AF                 .       XOR    A
0004  D3 00              ..      OUT    ($00), A
0006  21 24 00           !$.     LD     HL, $0024
0009  11 00 DA           ...     LD     DE, $DA00
000C  01 61 1D           .a.     LD     BC, $1D61
000F  ED B0              ..      LDIR
.
0011  31 FF FE           1..     LD     SP, $FEFF
0014  DB 00              ..      IN     A, ($00)
0016  B7                 .       OR     A
0017  C2 11 00           ...     JP     NZ $0011
001A  DB 01              ..      IN     A, ($01)
001C  FE AA              ..      CP     $AA
001E  C2 11 00           ...     JP     NZ $0011
0021  C3 00 F0           ...     JP     $F000
0024  C3 55 DC           .U.     JP     $DC55
0027  C3 4D DC           .M.     JP     $DC4D
002A  7F                        LD     A, A
002B  00                 .       NOP
002C  20 20                      JR     NZ $004E
002E  20 20                      JR     NZ $0050
0030  20 43               C      JR     NZ $0075
0032  6F                 o       LD     L, A
0033  70                 p       LD     (HL), B
0034  79                 y       LD     A, C
0035  72                 r       LD     (HL), D
0036  69                 i       LD     L, C
0037  68                 h       LD     L, B
0038  74                 t       LD     (HL), H
0039  20 28               (      JR     NZ $0063
003B  43                 C       LD     B, E
003C  29                 )       ADD    HL, HL
003D  20 31               1      JR     NZ $0070
003F  39                 9       ADD    HL, SP
0040  38 32              82      JR     C, $0074
0042  20 53               S      JR     NZ $0097
0044  63                 c       LD     H, E
0045  69                 i       LD     L, C
0046  66                 f       LD     H, (HL)
0047  61                 a       LD     H, C
0048  78                 x       LD     A, B
0049  20 4D               M      JR     NZ $0098
004B  69                 i       LD     L, C
004C  63                 c       LD     H, E
004D  72                 r       LD     (HL), D
.
004E  6F                 o       LD     L, A
004F  73                 s       LD     (HL), E
.
0050  6F                 o       LD     L, A
0051  66                 f       LD     H, (HL)
0052  74                 t       LD     (HL), H
0053  77                 w       LD     (HL), A
0054  61                 a       LD     H, C
0055  72                 r       LD     (HL), D
0056  65                 e       LD     H, L
0057  20 20                      JR     NZ $0079
0059  20 20                      JR     NZ $007B
005B  00                 .       NOP
005C  00                 .       NOP
005D  00                 .       NOP
005E  00                 .       NOP
005F  00                 .       NOP
0060  00                 .       NOP
0061  00                 .       NOP
0062  00                 .       NOP
.
0063  00                 .       NOP
0064  00                 .       NOP
0065  00                 .       NOP
0066  00                 .       NOP
0067  00                 .       NOP
0068  00                 .       NOP
0069  00                 .       NOP
006A  00                 .       NOP
006B  00                 .       NOP
006C  00                 .       NOP
006D  00                 .       NOP
006E  00                 .       NOP
006F  00                 .       NOP
.
0070  00                 .       NOP
0071  00                 .       NOP
0072  00                 .       NOP
0073  00                 .       NOP
.
0074  00                 .       NOP
.
0075  00                 .       NOP
0076  00                 .       NOP
0077  00                 .       NOP
0078  00                 .       NOP
.
0079  00                 .       NOP
007A  00                 .       NOP
.
007B  00                 .       NOP
007C  00                 .       NOP
007D  00                 .       NOP
007E  00                 .       NOP
007F  00                 .       NOP
0080  00                 .       NOP
0081  00                 .       NOP
0082  00                 .       NOP
0083  00                 .       NOP
0084  00                 .       NOP
0085  00                 .       NOP
0086  00                 .       NOP
0087  00                 .       NOP
0088  00                 .       NOP
0089  00                 .       NOP
008A  00                 .       NOP
008B  00                 .       NOP
008C  00                 .       NOP
008D  00                 .       NOP
008E  00                 .       NOP
008F  00                 .       NOP
0090  00                 .       NOP
0091  00                 .       NOP
0092  00                 .       NOP
0093  00                 .       NOP
0094  00                 .       NOP
0095  00                 .       NOP
0096  00                 .       NOP
.
0097  00                 .       NOP
.
0098  00                 .       NOP
0099  00                 .       NOP
009A  00                 .       NOP
009B  00                 .       NOP
009C  00                 .       NOP
009D  00                 .       NOP
009E  00                 .       NOP
009F  00                 .       NOP
00A0  00                 .       NOP
00A1  00                 .       NOP
00A2  00                 .       NOP
00A3  00                 .       NOP
00A4  00                 .       NOP
00A5  00                 .       NOP
00A6  00                 .       NOP
00A7  00                 .       NOP
00A8  00                 .       NOP
00A9  00                 .       NOP
00AA  00                 .       NOP
00AB  00                 .       NOP
00AC  30 31              01      JR     NC $00DF
00AE  2E 30              .0      LD     L, $30
00B0  36 34              64      LD     (HL), $34
00B2  00                 .       NOP
00B3  24                 $       INC    H
00B4  24                 $       INC    H
00B5  24                 $       INC    H
00B6  20 20                      JR     NZ $00D8
00B8  20 20                      JR     NZ $00DA
00BA  20 53               S      JR     NZ $010F
00BC  55                 U       LD     D, L
00BD  42                 B       LD     B, D
00BE  00                 .       NOP
00BF  00                 .       NOP
00C0  00                 .       NOP
00C1  00                 .       NOP
00C2  00                 .       NOP
00C3  00                 .       NOP
00C4  00                 .       NOP
00C5  00                 .       NOP
00C6  00                 .       NOP
00C7  00                 .       NOP
00C8  00                 .       NOP
00C9  00                 .       NOP
00CA  00                 .       NOP
00CB  00                 .       NOP
00CC  00                 .       NOP
00CD  00                 .       NOP
00CE  00                 .       NOP
00CF  00                 .       NOP
00D0  00                 .       NOP
00D1  00                 .       NOP
00D2  0D                 .       DEC    C
00D3  0A                 .       LD     A, (BC)
00D4  0D                 .       DEC    C
00D5  0A                 .       LD     A, (BC)
00D6  00                 .       NOP
00D7  3E 00              >.      LD     A, $00
00D9  00                 .       NOP
.
00DA  00                 .       NOP
00DB  00                 .       NOP
00DC  00                 .       NOP
00DD  00                 .       NOP
00DE  00                 .       NOP
.
00DF  00                 .       NOP
00E0  00                 .       NOP
00E1  00                 .       NOP
00E2  43                 C       LD     B, E
00E3  4F                 O       LD     C, A
00E4  4D                 M       LD     C, L
00E5  00                 .       NOP
00E6  00                 .       NOP
00E7  00                 .       NOP
00E8  00                 .       NOP
00E9  00                 .       NOP
00EA  00                 .       NOP
00EB  00                 .       NOP
00EC  00                 .       NOP
00ED  00                 .       NOP
00EE  00                 .       NOP
00EF  00                 .       NOP
00F0  00                 .       NOP
00F1  00                 .       NOP
00F2  00                 .       NOP
00F3  00                 .       NOP
00F4  00                 .       NOP
00F5  00                 .       NOP
00F6  00                 .       NOP
00F7  00                 .       NOP
.
00F8  00                 .       NOP
00F9  00                 .       NOP
00FA  00                 .       NOP
00FB  00                 .       NOP
00FC  00                 .       NOP
00FD  00                 .       NOP
00FE  00                 .       NOP
00FF  00                 .       NOP
.
0100  00                 .       NOP
0101  00                 .       NOP
0102  00                 .       NOP
0103  00                 .       NOP
0104  00                 .       NOP
0105  00                 .       NOP
0106  00                 .       NOP
0107  00                 .       NOP
0108  00                 .       NOP
0109  00                 .       NOP
010A  00                 .       NOP
010B  20 00               .      JR     NZ $010D
.
010D  00                 .       NOP
010E  00                 .       NOP
.
010F  00                 .       NOP
0110  00                 .       NOP
0111  00                 .       NOP
0112  00                 .       NOP
0113  00                 .       NOP
0114  00                 .       NOP
0115  00                 .       NOP
0116  00                 .       NOP
0117  00                 .       NOP
0118  20 00               .      JR     NZ $011A
.
011A  20 20                      JR     NZ $013C
011C  00                 .       NOP
011D  00                 .       NOP
011E  00                 .       NOP
011F  00                 .       NOP
0120  3F                 ?       CCF
0121  44                 D       LD     B, H
0122  2F                 /       CPL
0123  55                 U       LD     D, L
0124  53                 S       LD     D, E
0125  2D                 -       DEC    L
0126  46                 F       LD     B, (HL)
0127  2D                 -       DEC    L
0128  42                 B       LD     B, D
0129  61                 a       LD     H, C
012A  64                 d       LD     H, H
012B  20 63               c      JR     NZ $0190
012D  6F                 o       LD     L, A
012E  6D                 m       LD     L, L
012F  6D                 m       LD     L, L
0130  61                 a       LD     H, C
0131  6E                 n       LD     L, (HL)
0132  64                 d       LD     H, H
0133  2E 00              ..      LD     L, $00
0135  3F                 ?       CCF
0136  44                 D       LD     B, H
0137  49                 I       LD     C, C
0138  52                 R       LD     D, D
0139  2D                 -       DEC    L
013A  49                 I       LD     C, C
013B  2D                 -       DEC    L
.
013C  4E                 N       LD     C, (HL)
013D  6F                 o       LD     L, A
013E  20 66               f      JR     NZ $01A6
0140  69                 i       LD     L, C
0141  6C                 l       LD     L, H
0142  65                 e       LD     H, L
0143  73                 s       LD     (HL), E
0144  20 66               f      JR     NZ $01AC
0146  6F                 o       LD     L, A
0147  75                 u       LD     (HL), L
0148  6E                 n       LD     L, (HL)
0149  64                 d       LD     H, H
014A  2E 00              ..      LD     L, $00
014C  3F                 ?       CCF
014D  45                 E       LD     B, L
014E  72                 r       LD     (HL), D
014F  61                 a       LD     H, C
0150  73                 s       LD     (HL), E
0151  65                 e       LD     H, L
0152  2D                 -       DEC    L
0153  46                 F       LD     B, (HL)
0154  2D                 -       DEC    L
0155  00                 .       NOP
0156  3F                 ?       CCF
0157  52                 R       LD     D, D
0158  65                 e       LD     H, L
0159  6E                 n       LD     L, (HL)
015A  61                 a       LD     H, C
015B  6D                 m       LD     L, L
015C  65                 e       LD     H, L
015D  2D                 -       DEC    L
015E  46                 F       LD     B, (HL)
015F  2D                 -       DEC    L
0160  00                 .       NOP
0161  3F                 ?       CCF
0162  53                 S       LD     D, E
0163  61                 a       LD     H, C
0164  76                 v       HALT
0165  65                 e       LD     H, L
0166  2D                 -       DEC    L
0167  46                 F       LD     B, (HL)
0168  2D                 -       DEC    L
0169  00                 .       NOP
016A  3F                 ?       CCF
016B  54                 T       LD     D, H
016C  79                 y       LD     A, C
016D  70                 p       LD     (HL), B
016E  65                 e       LD     H, L
016F  2D                 -       DEC    L
0170  46                 F       LD     B, (HL)
0171  2D                 -       DEC    L
0172  00                 .       NOP
0173  3F                 ?       CCF
0174  55                 U       LD     D, L
0175  73                 s       LD     (HL), E
0176  65                 e       LD     H, L
0177  72                 r       LD     (HL), D
0178  2D                 -       DEC    L
0179  46                 F       LD     B, (HL)
017A  2D                 -       DEC    L
017B  00                 .       NOP
017C  4D                 M       LD     C, L
017D  69                 i       LD     L, C
017E  73                 s       LD     (HL), E
017F  73                 s       LD     (HL), E
0180  69                 i       LD     L, C
0181  6E                 n       LD     L, (HL)
0182  67                 g       LD     H, A
0183  20 6F               o      JR     NZ $01F4
0185  70                 p       LD     (HL), B
0186  65                 e       LD     H, L
0187  72                 r       LD     (HL), D
0188  61                 a       LD     H, C
0189  6E                 n       LD     L, (HL)
018A  64                 d       LD     H, H
018B  28 73              (s      JR     Z, $0200
018D  29                 )       ADD    HL, HL
018E  2E 00              ..      LD     L, $00
.
0190  46                 F       LD     B, (HL)
0191  69                 i       LD     L, C
0192  6C                 l       LD     L, H
0193  65                 e       LD     H, L
0194  20 6E               n      JR     NZ $0204
0196  6F                 o       LD     L, A
0197  74                 t       LD     (HL), H
0198  20 66               f      JR     NZ $0200
019A  6F                 o       LD     L, A
019B  75                 u       LD     (HL), L
019C  6E                 n       LD     L, (HL)
019D  64                 d       LD     H, H
019E  2E 00              ..      LD     L, $00
01A0  46                 F       LD     B, (HL)
01A1  69                 i       LD     L, C
01A2  6C                 l       LD     L, H
01A3  65                 e       LD     H, L
01A4  6E                 n       LD     L, (HL)
01A5  61                 a       LD     H, C
.
01A6  6D                 m       LD     L, L
01A7  65                 e       LD     H, L
01A8  28 73              (s      JR     Z, $021D
01AA  29                 )       ADD    HL, HL
01AB  20 6D               m      JR     NZ $021A
01AD  69                 i       LD     L, C
01AE  73                 s       LD     (HL), E
01AF  73                 s       LD     (HL), E
01B0  69                 i       LD     L, C
01B1  6E                 n       LD     L, (HL)
01B2  67                 g       LD     H, A
01B3  2E 00              ..      LD     L, $00
01B5  57                 W       LD     D, A
01B6  69                 i       LD     L, C
01B7  6C                 l       LD     L, H
01B8  64                 d       LD     H, H
01B9  63                 c       LD     H, E
01BA  61                 a       LD     H, C
01BB  72                 r       LD     (HL), D
01BC  64                 d       LD     H, H
01BD  73                 s       LD     (HL), E
01BE  20 6E               n      JR     NZ $022E
01C0  6F                 o       LD     L, A
01C1  74                 t       LD     (HL), H
01C2  20 70               p      JR     NZ $0234
01C4  65                 e       LD     H, L
01C5  72                 r       LD     (HL), D
01C6  6D                 m       LD     L, L
01C7  69                 i       LD     L, C
01C8  74                 t       LD     (HL), H
01C9  74                 t       LD     (HL), H
01CA  65                 e       LD     H, L
01CB  64                 d       LD     H, H
01CC  2E 00              ..      LD     L, $00
01CE  42                 B       LD     B, D
01CF  61                 a       LD     H, C
01D0  64                 d       LD     H, H
01D1  20 70               p      JR     NZ $0243
01D3  61                 a       LD     H, C
01D4  67                 g       LD     H, A
01D5  65                 e       LD     H, L
01D6  20 6E               n      JR     NZ $0246
01D8  75                 u       LD     (HL), L
01D9  6D                 m       LD     L, L
01DA  62                 b       LD     H, D
01DB  65                 e       LD     H, L
01DC  72                 r       LD     (HL), D
01DD  2E 00              ..      LD     L, $00
01DF  44                 D       LD     B, H
01E0  69                 i       LD     L, C
01E1  72                 r       LD     (HL), D
01E2  65                 e       LD     H, L
01E3  63                 c       LD     H, E
01E4  74                 t       LD     (HL), H
01E5  6F                 o       LD     L, A
01E6  72                 r       LD     (HL), D
01E7  79                 y       LD     A, C
01E8  20 66               f      JR     NZ $0250
01EA  75                 u       LD     (HL), L
01EB  6C                 l       LD     L, H
01EC  6C                 l       LD     L, H
01ED  2E 00              ..      LD     L, $00
01EF  44                 D       LD     B, H
01F0  69                 i       LD     L, C
01F1  73                 s       LD     (HL), E
01F2  6B                 k       LD     L, E
01F3  20 66               f      JR     NZ $025B
01F5  75                 u       LD     (HL), L
01F6  6C                 l       LD     L, H
01F7  6C                 l       LD     L, H
01F8  2E 00              ..      LD     L, $00
01FA  42                 B       LD     B, D
01FB  61                 a       LD     H, C
01FC  64                 d       LD     H, H
01FD  20 63               c      JR     NZ $0262
01FF  6C                 l       LD     L, H
.
0200  6F                 o       LD     L, A
0201  73                 s       LD     (HL), E
0202  65                 e       LD     H, L
0203  2E 00              ..      LD     L, $00
0205  42                 B       LD     B, D
0206  61                 a       LD     H, C
0207  64                 d       LD     H, H
0208  20 75               u      JR     NZ $027F
.
020A  73                 s       LD     (HL), E
020B  65                 e       LD     H, L
020C  72                 r       LD     (HL), D
020D  20 6E               n      JR     NZ $027D
020F  75                 u       LD     (HL), L
0210  6D                 m       LD     L, L
0211  62                 b       LD     H, D
0212  65                 e       LD     H, L
0213  72                 r       LD     (HL), D
0214  2E 00              ..      LD     L, $00
0216  46                 F       LD     B, (HL)
0217  69                 i       LD     L, C
0218  6C                 l       LD     L, H
0219  65                 e       LD     H, L
.
021A  20 61               a      JR     NZ $027D
021C  6C                 l       LD     L, H
.
021D  72                 r       LD     (HL), D
021E  65                 e       LD     H, L
021F  61                 a       LD     H, C
0220  64                 d       LD     H, H
0221  79                 y       LD     A, C
0222  20 65               e      JR     NZ $0289
0224  78                 x       LD     A, B
0225  69                 i       LD     L, C
0226  73                 s       LD     (HL), E
0227  74                 t       LD     (HL), H
0228  73                 s       LD     (HL), E
0229  2E 00              ..      LD     L, $00
022B  0D                 .       DEC    C
022C  0A                 .       LD     A, (BC)
022D  45                 E       LD     B, L
.
022E  72                 r       LD     (HL), D
022F  61                 a       LD     H, C
0230  73                 s       LD     (HL), E
0231  65                 e       LD     H, L
0232  2D                 -       DEC    L
0233  51                 Q       LD     D, C
.
0234  2D                 -       DEC    L
0235  41                 A       LD     B, C
0236  72                 r       LD     (HL), D
0237  65                 e       LD     H, L
0238  20 79               y      JR     NZ $02B3
023A  6F                 o       LD     L, A
023B  75                 u       LD     (HL), L
023C  20 73               s      JR     NZ $02B1
023E  75                 u       LD     (HL), L
023F  72                 r       LD     (HL), D
0240  65                 e       LD     H, L
0241  3F                 ?       CCF
0242  00                 .       NOP
.
0243  0D                 .       DEC    C
0244  0A                 .       LD     A, (BC)
0245  00                 .       NOP
.
0246  44                 D       LD     B, H
0247  49                 I       LD     C, C
0248  52                 R       LD     D, D
0249  20 20                      JR     NZ $026B
024B  5B                 [       LD     E, E
024C  DF                 .       RST    18H
024D  54                 T       LD     D, H
024E  59                 Y       LD     E, C
024F  50                 P       LD     D, B
.
0250  45                 E       LD     B, L
0251  20 50               P      JR     NZ $02A3
0253  E1                 .       POP    HL
0254  45                 E       LD     B, L
0255  52                 R       LD     D, D
0256  41                 A       LD     B, C
0257  20 20                      JR     NZ $0279
0259  06 E0              ..      LD     B, $E0
.
025B  52                 R       LD     D, D
025C  45                 E       LD     B, L
025D  4E                 N       LD     C, (HL)
025E  20 20                      JR     NZ $0280
0260  51                 Q       LD     D, C
0261  E0                 .       RET    PO
.
0262  53                 S       LD     D, E
0263  41                 A       LD     B, C
0264  56                 V       LD     D, (HL)
0265  45                 E       LD     B, L
0266  20 A2               .      JR     NZ $020A
0268  E0                 .       RET    PO
0269  55                 U       LD     D, L
026A  53                 S       LD     D, E
.
026B  45                 E       LD     B, L
026C  52                 R       LD     D, D
026D  20 AE               .      JR     NZ $021D
026F  E1                 .       POP    HL
0270  FF                 .       RST    38H
0271  AF                 .       XOR    A
0272  32 07 DA           2..     LD     ($DA07), A
0275  3A 04 00           :..     LD     A, ($0004)
0278  4F                 O       LD     C, A
.
0279  31 AE DA           1..     LD     SP, $DAAE
027C  21 4D DC           !M.     LD     HL, $DC4D
.
027F  E5                 .       PUSH   HL
.
0280  C5                 .       PUSH   BC
0281  1E 00              ..      LD     E, $00
0283  0E 0E              ..      LD     C, $0E
0285  CD 05 00           ...     CALL   $0005
0288  C1                 .       POP    BC
.
0289  C5                 .       PUSH   BC
028A  79                 y       LD     A, C
028B  E6 0F              ..      AND    $0F
028D  5F                 _       LD     E, A
028E  0E 0E              ..      LD     C, $0E
0290  CD 05 00           ...     CALL   $0005
0293  C1                 .       POP    BC
0294  CB 39              .9      SRL    C
0296  CB 39              .9      SRL    C
0298  CB 39              .9      SRL    C
029A  CB 39              .9      SRL    C
029C  59                 Y       LD     E, C
029D  0E 20              .       LD     C, $20
029F  CD 05 00           ...     CALL   $0005
02A2  21 07 DA           !..     LD     HL, $DA07
02A5  7E                 ~       LD     A, (HL)
02A6  B7                 .       OR     A
02A7  C2 2D DD           .-.     JP     NZ $DD2D
02AA  21 8E DA           !..     LD     HL, $DA8E
02AD  11 5C 00           .\.     LD     DE, $005C
02B0  01 10 00           ...     LD     BC, $0010
.
02B3  ED B0              ..      LDIR
02B5  11 5C 00           .\.     LD     DE, $005C
02B8  0E 0F              ..      LD     C, $0F
02BA  CD 05 00           ...     CALL   $0005
02BD  B7                 .       OR     A
02BE  FA 0E DD           ...     JP     M $DD0E
02C1  DD 21 5C 00        .!\.    LD     IX, $005C
02C5  DD 7E 0F           .~.     LD     A, (IX+$0F)
02C8  B7                 .       OR     A
02C9  C2 B3 DC           ...     JP     NZ $DCB3
.
02CC  11 5C 00           .\.     LD     DE, $005C
02CF  0E 13              ..      LD     C, $13
02D1  CD 05 00           ...     CALL   $0005
02D4  C3 0E DD           ...     JP     $DD0E
02D7  F5                 .       PUSH   AF
02D8  0E 0B              ..      LD     C, $0B
02DA  CD 05 00           ...     CALL   $0005
02DD  B7                 .       OR     A
02DE  28 0C              (.      JR     Z, $02EC
02E0  0E 01              ..      LD     C, $01
02E2  CD 05 00           ...     CALL   $0005
02E5  FE 7F              .      CP     $7F
02E7  20 03               .      JR     NZ $02EC
02E9  F1                 .       POP    AF
02EA  18 E0              ..      JR     $02CC
.
02EC  F1                 .       POP    AF
02ED  3D                 =       DEC    A
02EE  DD 77 20           .w      LD     (IX+$20), A
02F1  11 07 DA           ...     LD     DE, $DA07
02F4  0E 1A              ..      LD     C, $1A
02F6  CD 05 00           ...     CALL   $0005
02F9  11 5C 00           .\.     LD     DE, $005C
02FC  0E 14              ..      LD     C, $14
02FE  CD 05 00           ...     CALL   $0005
0301  DD 21 5C 00        .!\.    LD     IX, $005C
0305  DD 35 0F           .5.     DEC    (IX+$0F)
0308  DD CB              ..      ****BUG****			DD CB 05 FE   SET 7,(IX+05)
030A  0E BE              ..      LD     C, $BE
030C  11 5C 00           .\.     LD     DE, $005C
030F  0E 10              ..      LD     C, $10
0311  CD 05 00           ...     CALL   $0005
0314  11 1F DC           ...     LD     DE, $DC1F
0317  CD 4C DF           .L.     CALL   $DF4C
031A  11 08 DA           ...     LD     DE, $DA08
031D  CD 4C DF           .L.     CALL   $DF4C
0320  1E 0D              ..      LD     E, $0D
0322  0E 02              ..      LD     C, $02
0324  CD 05 00           ...     CALL   $0005
0327  3A 08 DA           :..     LD     A, ($DA08)
032A  FE 21              .!      CP     $21
032C  CA 4D DC           .M.     JP     Z $DC4D
032F  C3 7E DC           .~.     JP     $DC7E
.
0332  3A 04 00           :..     LD     A, ($0004)
0335  E6 0F              ..      AND    $0F
0337  C6 41              .A      ADD    A, $41
0339  32 B2 DA           2..     LD     ($DAB2), A
033C  11 B0 DA           ...     LD     DE, $DAB0
033F  CD 4C DF           .L.     CALL   $DF4C
0342  11 06 DA           ...     LD     DE, $DA06
0345  0E 0A              ..      LD     C, $0A
0347  CD 05 00           ...     CALL   $0005
034A  21 07 DA           !..     LD     HL, $DA07
034D  7E                 ~       LD     A, (HL)
034E  B7                 .       OR     A
034F  28 E1              (.      JR     Z, $0332
0351  23                 #       INC    HL
0352  E5                 .       PUSH   HL
0353  4F                 O       LD     C, A
0354  AF                 .       XOR    A
0355  47                 G       LD     B, A
0356  09                 .       ADD    HL, BC
0357  77                 w       LD     (HL), A
0358  21 5C 00           !\.     LD     HL, $005C
035B  77                 w       LD     (HL), A
035C  23                 #       INC    HL
035D  11 5E 00           .^.     LD     DE, $005E
0360  36 20              6       LD     (HL), $20
0362  0E 0B              ..      LD     C, $0B
0364  ED B0              ..      LDIR
0366  77                 w       LD     (HL), A
0367  0E 03              ..      LD     C, $03
0369  ED B0              ..      LDIR
036B  21 5C 00           !\.     LD     HL, $005C
036E  0E 10              ..      LD     C, $10
0370  ED B0              ..      LDIR
0372  EB                 .       EX     DE, HL
0373  06 04              ..      LD     B, $04
.
0375  36 00              6.      LD     (HL), $00
0377  23                 #       INC    HL
0378  10 FB              ..      DJNZ   $0375
037A  E1                 .       POP    HL
037B  CD 9C DD           ...     CALL   $DD9C
037E  DA 4D DC           .M.     JP     C $DC4D
0381  CD CB DD           ...     CALL   $DDCB
0384  E5                 .       PUSH   HL
0385  E5                 .       PUSH   HL
0386  21 D7 DA           !..     LD     HL, $DAD7
0389  3E 20              >       LD     A, $20
038B  BE                 .       CP     (HL)
038C  CA 58 DE           .X.     JP     Z $DE58
038F  2B                 +       DEC    HL
0390  11 B5 DA           ...     LD     DE, $DAB5
0393  01 09 00           ...     LD     BC, $0009
0396  ED B0              ..      LDIR
0398  E1                 .       POP    HL
0399  CD 35 DE           .5.     CALL   $DE35
039C  DA 71 DE           .q.     JP     C $DE71
039F  E5                 .       PUSH   HL
03A0  21 D6 DA           !..     LD     HL, $DAD6
03A3  11 5C 00           .\.     LD     DE, $005C
03A6  01 0C 00           ...     LD     BC, $000C
03A9  ED B0              ..      LDIR
03AB  E1                 .       POP    HL
03AC  CD 35 DE           .5.     CALL   $DE35
03AF  DA 71 DE           .q.     JP     C $DE71
03B2  21 D6 DA           !..     LD     HL, $DAD6
03B5  11 6C 00           .l.     LD     DE, $006C
03B8  01 0C 00           ...     LD     BC, $000C
03BB  ED B0              ..      LDIR
03BD  C3 71 DE           .q.     JP     $DE71
03C0  AF                 .       XOR    A
03C1  32 D6 DA           2..     LD     ($DAD6), A
03C4  CD 46 DE           .F.     CALL   $DE46
03C7  D8                 .       RET    C
03C8  FE 20              .       CP     $20
03CA  CA A0 DD           ...     JP     Z $DDA0
03CD  47                 G       LD     B, A
03CE  7E                 ~       LD     A, (HL)
03CF  FE 3A              .:      CP     $3A
03D1  C2 C2 DD           ...     JP     NZ $DDC2
03D4  78                 x       LD     A, B
03D5  D6 40              .@      SUB    $40
03D7  FE 01              ..      CP     $01
03D9  38 0E              8.      JR     C, $03E9
03DB  FE 11              ..      CP     $11
03DD  30 0A              0.      JR     NC $03E9
03DF  32 D6 DA           2..     LD     ($DAD6), A
03E2  23                 #       INC    HL
03E3  C3 C3 DD           ...     JP     $DDC3
03E6  2B                 +       DEC    HL
03E7  AF                 .       XOR    A
03E8  C9                 .       RET
.
03E9  CD 06 DF           ...     CALL   $DF06
03EC  C3 4D DC           .M.     JP     $DC4D
03EF  11 D7 DA           ...     LD     DE, $DAD7
03F2  06 0B              ..      LD     B, $0B
03F4  3E 20              >       LD     A, $20
.
03F6  12                 .       LD     (DE), A
03F7  13                 .       INC    DE
03F8  10 FC              ..      DJNZ   $03F6
03FA  11 D7 DA           ...     LD     DE, $DAD7
03FD  06 08              ..      LD     B, $08
.
03FF  CD 46 DE           .F.     CALL   $DE46
0402  DA 04 DE           ...     JP     C $DE04
0405  FE 20              .       CP     $20
0407  CA 04 DE           ...     JP     Z $DE04
040A  FE 2E              ..      CP     $2E
040C  CA 04 DE           ...     JP     Z $DE04
040F  FE 2A              .*      CP     $2A
0411  CA 07 DE           ...     JP     Z $DE07
0414  12                 .       LD     (DE), A
0415  13                 .       INC    DE
0416  10 E7              ..      DJNZ   $03FF
0418  CD 46 DE           .F.     CALL   $DE46
041B  DA 04 DE           ...     JP     C $DE04
041E  FE 20              .       CP     $20
0420  CA 04 DE           ...     JP     Z $DE04
0423  FE 2E              ..      CP     $2E
0425  C2 F4 DD           ...     JP     NZ $DDF4
0428  2B                 +       DEC    HL
0429  AF                 .       XOR    A
042A  C9                 .       RET
042B  3E 3F              >?      LD     A, $3F
.
042D  12                 .       LD     (DE), A
042E  13                 .       INC    DE
042F  10 FC              ..      DJNZ   $042D
0431  C9                 .       RET
0432  06 03              ..      LD     B, $03
0434  11 DF DA           ...     LD     DE, $DADF
.
0437  CD 46 DE           .F.     CALL   $DE46
043A  DA 32 DE           .2.     JP     C $DE32
043D  FE 20              .       CP     $20
043F  CA 32 DE           .2.     JP     Z $DE32
0442  FE 2A              .*      CP     $2A
0444  CA 07 DE           ...     JP     Z $DE07
0447  12                 .       LD     (DE), A
0448  13                 .       INC    DE
0449  10 EC              ..      DJNZ   $0437
044B  CD 46 DE           .F.     CALL   $DE46
044E  DA 32 DE           .2.     JP     C $DE32
0451  FE 20              .       CP     $20
0453  CA 27 DE           .'.     JP     Z $DE27
0456  2B                 +       DEC    HL
0457  AF                 .       XOR    A
0458  C9                 .       RET
0459  CD 9C DD           ...     CALL   $DD9C
045C  D8                 .       RET    C
045D  CD CB DD           ...     CALL   $DDCB
0460  D8                 .       RET    C
0461  3E 2E              >.      LD     A, $2E
0463  BE                 .       CP     (HL)
0464  C0                 .       RET    NZ
0465  23                 #       INC    HL
0466  CD 0E DE           ...     CALL   $DE0E
0469  C9                 .       RET
046A  7E                 ~       LD     A, (HL)
046B  23                 #       INC    HL
046C  FE 60              .`      CP     $60
046E  DA 54 DE           .T.     JP     C $DE54
0471  FE 7B              .{      CP     $7B
0473  D2 54 DE           .T.     JP     NC $DE54
0476  CB AF              ..      RES    5, A
0478  B7                 .       OR     A
0479  C0                 .       RET    NZ
047A  3F                 ?       CCF
047B  C9                 .       RET
047C  E1                 .       POP    HL
047D  E1                 .       POP    HL
047E  3A D6 DA           :..     LD     A, ($DAD6)
0481  3D                 =       DEC    A
0482  FA 06 DF           ...     JP     M $DF06
0485  5F                 _       LD     E, A
0486  3A 04 00           :..     LD     A, ($0004)
0489  E6 F0              ..      AND    $F0
048B  B3                 .       OR     E
048C  32 04 00           2..     LD     ($0004), A
048F  0E 0E              ..      LD     C, $0E
0491  CD 05 00           ...     CALL   $0005
0494  C9                 .       RET
0495  E1                 .       POP    HL
0496  11 81 00           ...     LD     DE, $0081
0499  01 00 00           ...     LD     BC, $0000
049C  7E                 ~       LD     A, (HL)
049D  ED A0              ..      LDI
049F  B7                 .       OR     A
04A0  C2 78 DE           .x.     JP     NZ $DE78
04A3  79                 y       LD     A, C
04A4  2F                 /       CPL
04A5  32 80 00           2..     LD     ($0080), A
04A8  21 B6 DA           !..     LD     HL, $DAB6
04AB  06 08              ..      LD     B, $08
04AD  3E 3F              >?      LD     A, $3F
.
04AF  BE                 .       CP     (HL)
04B0  CA 06 DF           ...     JP     Z $DF06
04B3  23                 #       INC    HL
04B4  10 F9              ..      DJNZ   $04AF
04B6  21 22 DC           !".     LD     HL, $DC22
04B9  11 B6 DA           ...     LD     DE, $DAB6
04BC  01 05 00           ...     LD     BC, $0005
04BF  1A                 .       LD     A, (DE)
04C0  13                 .       INC    DE
04C1  ED A1              ..      CPI
04C3  C2 B9 DE           ...     JP     NZ $DEB9
04C6  EA 9B DE           ...     JP     PE $DE9B
04C9  7E                 ~       LD     A, (HL)
04CA  23                 #       INC    HL
04CB  66                 f       LD     H, (HL)
04CC  6F                 o       LD     L, A
04CD  E5                 .       PUSH   HL
04CE  11 80 00           ...     LD     DE, $0080
04D1  0E 1A              ..      LD     C, $1A
04D3  CD 05 00           ...     CALL   $0005
04D6  11 1F DC           ...     LD     DE, $DC1F
04D9  CD 4C DF           .L.     CALL   $DF4C
04DC  C9                 .       RET
04DD  09                 .       ADD    HL, BC
04DE  23                 #       INC    HL
04DF  23                 #       INC    HL
04E0  7E                 ~       LD     A, (HL)
04E1  B7                 .       OR     A
04E2  F2 95 DE           ...     JP     P $DE95
04E5  AF                 .       XOR    A
04E6  32 D5 DA           2..     LD     ($DAD5), A
04E9  11 B5 DA           ...     LD     DE, $DAB5
04EC  0E 0F              ..      LD     C, $0F
04EE  CD 05 00           ...     CALL   $0005
04F1  B7                 .       OR     A
04F2  FA 06 DF           ...     JP     M $DF06
04F5  11 00 01           ...     LD     DE, $0100
04F8  ED 53 E2 DA        .S..    LD     ($DAE2), DE
04FC  0E 1A              ..      LD     C, $1A
04FE  CD 05 00           ...     CALL   $0005
0501  11 B5 DA           ...     LD     DE, $DAB5
0504  0E 14              ..      LD     C, $14
0506  CD 05 00           ...     CALL   $0005
0509  B7                 .       OR     A
050A  C2 F5 DE           ...     JP     NZ $DEF5
050D  ED 5B E2 DA        .[..    LD     DE, ($DAE2)
0511  21 80 00           !..     LD     HL, $0080
0514  19                 .       ADD    HL, DE
0515  EB                 .       EX     DE, HL
0516  C3 D4 DE           ...     JP     $DED4
0519  11 80 00           ...     LD     DE, $0080
051C  0E 1A              ..      LD     C, $1A
051E  CD 05 00           ...     CALL   $0005
0521  11 1F DC           ...     LD     DE, $DC1F
0524  CD 4C DF           .L.     CALL   $DF4C
0527  C3 00 01           ...     JP     $0100
052A  11 21 DC           .!.     LD     DE, $DC21
052D  21 FC DA           !..     LD     HL, $DAFC
0530  E5                 .       PUSH   HL
0531  D5                 .       PUSH   DE
0532  11 1F DC           ...     LD     DE, $DC1F
0535  CD 4C DF           .L.     CALL   $DF4C
0538  D1                 .       POP    DE
0539  CD 4C DF           .L.     CALL   $DF4C
053C  D1                 .       POP    DE
053D  CD 4C DF           .L.     CALL   $DF4C
0540  C9                 .       RET
0541  21 5D 00           !].     LD     HL, $005D
0544  AF                 .       XOR    A
.
0545  32 E6 DA           2..     LD     ($DAE6), A
0548  7E                 ~       LD     A, (HL)
0549  FE 20              .       CP     $20
054B  CA 48 DF           .H.     JP     Z $DF48
054E  23                 #       INC    HL
054F  FE 30              .0      CP     $30
0551  D8                 .       RET    C
0552  FE 3A              .:      CP     $3A
0554  3F                 ?       CCF
0555  D8                 .       RET    C
0556  D6 30              .0      SUB    $30
0558  5F                 _       LD     E, A
0559  3A E6 DA           :..     LD     A, ($DAE6)
055C  CB 27              .'      SLA    A
055E  D8                 .       RET    C
055F  4F                 O       LD     C, A
0560  CB 27              .'      SLA    A
0562  D8                 .       RET    C
0563  CB 27              .'      SLA    A
0565  D8                 .       RET    C
0566  81                 .       ADD    A, C
0567  D8                 .       RET    C
0568  83                 .       ADD    A, E
0569  D8                 .       RET    C
056A  18 D9              ..      JR     $0545
056C  3A E6 DA           :..     LD     A, ($DAE6)
056F  C9                 .       RET
0570  1A                 .       LD     A, (DE)
0571  B7                 .       OR     A
0572  C8                 .       RET    Z
0573  D5                 .       PUSH   DE
0574  5F                 _       LD     E, A
0575  0E 02              ..      LD     C, $02
0577  CD 05 00           ...     CALL   $0005
057A  D1                 .       POP    DE
057B  13                 .       INC    DE
057C  C3 4C DF           .L.     JP     $DF4C
057F  21 5D 00           !].     LD     HL, $005D
0582  7E                 ~       LD     A, (HL)
0583  FE 20              .       CP     $20
0585  20 07               .      JR     NZ $058E
0587  06 0B              ..      LD     B, $0B
.
0589  36 3F              6?      LD     (HL), $3F
058B  23                 #       INC    HL
058C  10 FB              ..      DJNZ   $0589
.
058E  DD 21 5C 00        .!\.    LD     IX, $005C
0592  DD 36 0C 00        .6..    
0596  DD 36 0D 00        .6..    
059A  DD 36 0E 00        .6..    
059E  11 5C 00           .\.     LD     DE, $005C
.
05A1  0E 11              ..      LD     C, $11
05A3  CD 05 00           ...     CALL   $0005
.
05A6  B7                 .       OR     A
05A7  FA FD DF           ...     JP     M $DFFD
05AA  32 F9 DA           2..     LD     ($DAF9), A
05AD  06 04              ..      LD     B, $04
05AF  C5                 .       PUSH   BC
05B0  3A F9 DA           :..     LD     A, ($DAF9)
05B3  4F                 O       LD     C, A
05B4  06 05              ..      LD     B, $05
.
05B6  CB 21              .!      SLA    C
05B8  10 FC              ..      DJNZ   $05B6
05BA  21 80 00           !..     LD     HL, $0080
05BD  09                 .       ADD    HL, BC
05BE  E5                 .       PUSH   HL
05BF  DD E1              ..      POP    IX
05C1  DD CB              ..      ****BUG****			DD CB 05 FE   SET 7,(IX+05)
05C3  0A                 .       LD     A, (BC)
05C4  7E                 ~       LD     A, (HL)
05C5  C2 EF DF           ...     JP     NZ $DFEF
05C8  23                 #       INC    HL
05C9  11 E8 DA           ...     LD     DE, $DAE8
05CC  06 0C              ..      LD     B, $0C
05CE  3E 20              >       LD     A, $20
.
05D0  12                 .       LD     (DE), A
05D1  13                 .       INC    DE
05D2  10 FC              ..      DJNZ   $05D0
05D4  11 E8 DA           ...     LD     DE, $DAE8
05D7  01 08 00           ...     LD     BC, $0008
05DA  CB BE              ..      RES    7, (HL)
05DC  7E                 ~       LD     A, (HL)
05DD  FE 20              .       CP     $20
05DF  28 05              (.      JR     Z, $05E6
05E1  ED A0              ..      LDI
05E3  EA B6 DF           ...     JP     PE $DFB6
.
05E6  3E 2E              >.      LD     A, $2E
05E8  12                 .       LD     (DE), A
05E9  13                 .       INC    DE
05EA  41                 A       LD     B, C
05EB  04                 .       INC    B
05EC  18 01              ..      JR     $05EF
.
05EE  23                 #       INC    HL
.
05EF  10 FD              ..      DJNZ   $05EE
05F1  01 03 00           ...     LD     BC, $0003
05F4  CB BE              ..      RES    7, (HL)
05F6  ED A0              ..      LDI
05F8  EA D0 DF           ...     JP     PE $DFD0
05FB  11 E7 DA           ...     LD     DE, $DAE7
05FE  CD 4C DF           .L.     CALL   $DF4C
0601  C1                 .       POP    BC
0602  10 08              ..      DJNZ   $060C
0604  11 1F DC           ...     LD     DE, $DC1F
0607  06 04              ..      LD     B, $04
0609  C3 EB DF           ...     JP     $DFEB
.
060C  11 F6 DA           ...     LD     DE, $DAF6
060F  C5                 .       PUSH   BC
0610  CD 4C DF           .L.     CALL   $DF4C
0613  0E 12              ..      LD     C, $12
0615  CD 05 00           ...     CALL   $0005
0618  C1                 .       POP    BC
0619  B7                 .       OR     A
061A  F8                 .       RET    M
061B  32 F9 DA           2..     LD     ($DAF9), A
061E  C3 8B DF           ...     JP     $DF8B
0621  11 11 DB           ...     LD     DE, $DB11
0624  21 21 DC           !!.     LD     HL, $DC21
0627  C3 0C DF           ...     JP     $DF0C
062A  3A 5D 00           :].     LD     A, ($005D)
062D  FE 20              .       CP     $20
062F  CA 46 E0           .F.     JP     Z $E046
0632  11 5C 00           .\.     LD     DE, $005C
0635  0E 11              ..      LD     C, $11
0637  CD 05 00           ...     CALL   $0005
063A  B7                 .       OR     A
063B  FA 41 E0           .A.     JP     M $E041
063E  11 07 DC           ...     LD     DE, $DC07
0641  CD 4C DF           .L.     CALL   $DF4C
0644  3E 01              >.      LD     A, $01
0646  32 80 00           2..     LD     ($0080), A
0649  11 80 00           ...     LD     DE, $0080
064C  0E 0A              ..      LD     C, $0A
064E  CD 05 00           ...     CALL   $0005
0651  3A 82 00           :..     LD     A, ($0082)
0654  FE 59              .Y      CP     $59
0656  CA 38 E0           .8.     JP     Z $E038
0659  FE 79              .y      CP     $79
065B  C0                 .       RET    NZ
065C  11 5C 00           .\.     LD     DE, $005C
065F  0E 13              ..      LD     C, $13
0661  CD 05 00           ...     CALL   $0005
0664  C9                 .       RET
0665  21 6C DB           !l.     LD     HL, $DB6C
0668  18 05              ..      JR     $066F
066A  21 7C DB           !|.     LD     HL, $DB7C
066D  18 00              ..      JR     $066F
.
066F  11 28 DB           .(.     LD     DE, $DB28
0672  C3 0C DF           ...     JP     $DF0C
0675  21 5C 00           !\.     LD     HL, $005C
0678  3E 3F              >?      LD     A, $3F
067A  06 20              .       LD     B, $20
.
067C  BE                 .       CP     (HL)
067D  28 2F              (/      JR     Z, $06AE
067F  23                 #       INC    HL
0680  10 FA              ..      DJNZ   $067C
0682  3A 5D 00           :].     LD     A, ($005D)
0685  FE 20              .       CP     $20
0687  28 2A              (*      JR     Z, $06B3
0689  3A 6D 00           :m.     LD     A, ($006D)
068C  FE 20              .       CP     $20
068E  28 23              (#      JR     Z, $06B3
0690  21 5C 00           !\.     LD     HL, $005C
0693  7E                 ~       LD     A, (HL)
0694  11 6C 00           .l.     LD     DE, $006C
0697  12                 .       LD     (DE), A
0698  0E 11              ..      LD     C, $11
069A  CD 05 00           ...     CALL   $0005
069D  B7                 .       OR     A
069E  F2 99 E0           ...     JP     P $E099
06A1  11 5C 00           .\.     LD     DE, $005C
06A4  0E 17              ..      LD     C, $17
06A6  CD 05 00           ...     CALL   $0005
06A9  B7                 .       OR     A
06AA  FA 94 E0           ...     JP     M $E094
06AD  C9                 .       RET
.
06AE  21 91 DB           !..     LD     HL, $DB91
06B1  18 0D              ..      JR     $06C0
.
06B3  21 7C DB           !|.     LD     HL, $DB7C
06B6  18 08              ..      JR     $06C0
06B8  21 6C DB           !l.     LD     HL, $DB6C
06BB  18 03              ..      JR     $06C0
06BD  21 F2 DB           !..     LD     HL, $DBF2
.
06C0  11 32 DB           .2.     LD     DE, $DB32
06C3  C3 0C DF           ...     JP     $DF0C
06C6  3A 5D 00           :].     LD     A, ($005D)
06C9  FE 20              .       CP     $20
06CB  CA 2E E1           ...     JP     Z $E12E
06CE  3A 6D 00           :m.     LD     A, ($006D)
06D1  FE 20              .       CP     $20
06D3  CA 2E E1           ...     JP     Z $E12E
06D6  21 5D 00           !].     LD     HL, $005D
06D9  CD 1D DF           ...     CALL   $DF1D
06DC  38 79              8y      JR     C, $0757
06DE  4F                 O       LD     C, A
06DF  06 00              ..      LD     B, $00
06E1  CB 21              .!      SLA    C
06E3  CB 10              ..      RL     B
06E5  ED 43 FA DA        .C..    LD     ($DAFA), BC
06E9  21 6C 00           !l.     LD     HL, $006C
06EC  11 5C 00           .\.     LD     DE, $005C
06EF  01 10 00           ...     LD     BC, $0010
06F2  ED B0              ..      LDIR
06F4  21 5D 00           !].     LD     HL, $005D
06F7  3E 3F              >?      LD     A, $3F
06F9  06 0B              ..      LD     B, $0B
.
06FB  BE                 .       CP     (HL)
06FC  CA 38 E1           .8.     JP     Z $E138
06FF  23                 #       INC    HL
0700  10 F9              ..      DJNZ   $06FB
0702  11 5C 00           .\.     LD     DE, $005C
0705  0E 13              ..      LD     C, $13
0707  CD 05 00           ...     CALL   $0005
070A  11 5C 00           .\.     LD     DE, $005C
070D  0E 16              ..      LD     C, $16
070F  CD 05 00           ...     CALL   $0005
0712  B7                 .       OR     A
0713  FA 3D E1           .=.     JP     M $E13D
0716  11 00 01           ...     LD     DE, $0100
.
0719  ED 4B FA DA        .K..    LD     BC, ($DAFA)
071D  78                 x       LD     A, B
071E  B1                 .       OR     C
071F  28 24              ($      JR     Z, $0745
0721  0B                 .       DEC    BC
0722  ED 43 FA DA        .C..    LD     ($DAFA), BC
0726  ED 53 E2 DA        .S..    LD     ($DAE2), DE
072A  0E 1A              ..      LD     C, $1A
072C  CD 05 00           ...     CALL   $0005
072F  11 5C 00           .\.     LD     DE, $005C
0732  0E 15              ..      LD     C, $15
0734  CD 05 00           ...     CALL   $0005
0737  B7                 .       OR     A
0738  20 2C               ,      JR     NZ $0766
073A  ED 5B E2 DA        .[..    LD     DE, ($DAE2)
073E  21 80 00           !..     LD     HL, $0080
0741  19                 .       ADD    HL, DE
0742  EB                 .       EX     DE, HL
0743  18 D4              ..      JR     $0719
.
0745  11 5C 00           .\.     LD     DE, $005C
0748  0E 10              ..      LD     C, $10
074A  CD 05 00           ...     CALL   $0005
074D  B7                 .       OR     A
074E  FA 47 E1           .G.     JP     M $E147
0751  C9                 .       RET
0752  21 58 DB           !X.     LD     HL, $DB58
0755  18 17              ..      JR     $076E
.
0757  21 AA DB           !..     LD     HL, $DBAA
075A  18 12              ..      JR     $076E
075C  21 91 DB           !..     LD     HL, $DB91
075F  18 0D              ..      JR     $076E
0761  21 BB DB           !..     LD     HL, $DBBB
0764  18 08              ..      JR     $076E
.
0766  21 CB DB           !..     LD     HL, $DBCB
0769  18 03              ..      JR     $076E
076B  21 D6 DB           !..     LD     HL, $DBD6
.
076E  11 3D DB           .=.     LD     DE, $DB3D
0771  C3 0C DF           ...     JP     $DF0C
0774  3A 5D 00           :].     LD     A, ($005D)
0777  FE 20              .       CP     $20
0779  28 49              (I      JR     Z, $07C4
077B  AF                 .       XOR    A
077C  32 7C 00           2|.     LD     ($007C), A
077F  11 5C 00           .\.     LD     DE, $005C
0782  0E 0F              ..      LD     C, $0F
0784  CD 05 00           ...     CALL   $0005
0787  B7                 .       OR     A
0788  FA A5 E1           ...     JP     M $E1A5
078B  11 5C 00           .\.     LD     DE, $005C
078E  0E 14              ..      LD     C, $14
0790  CD 05 00           ...     CALL   $0005
0793  B7                 .       OR     A
0794  C0                 .       RET    NZ
0795  21 80 00           !..     LD     HL, $0080
0798  06 80              ..      LD     B, $80
.
079A  7E                 ~       LD     A, (HL)
079B  FE 1A              ..      CP     $1A
079D  C8                 .       RET    Z
079E  E5                 .       PUSH   HL
079F  C5                 .       PUSH   BC
07A0  5F                 _       LD     E, A
07A1  0E 02              ..      LD     C, $02
07A3  CD 05 00           ...     CALL   $0005
07A6  0E 0B              ..      LD     C, $0B
07A8  CD 05 00           ...     CALL   $0005
07AB  B7                 .       OR     A
07AC  CA 95 E1           ...     JP     Z $E195
07AF  0E 01              ..      LD     C, $01
07B1  CD 05 00           ...     CALL   $0005
07B4  FE 03              ..      CP     $03
07B6  CA 9D E1           ...     JP     Z $E19D
07B9  C1                 .       POP    BC
07BA  E1                 .       POP    HL
07BB  23                 #       INC    HL
07BC  10 DC              ..      DJNZ   $079A
07BE  C3 67 E1           .g.     JP     $E167
07C1  E1                 .       POP    HL
07C2  E1                 .       POP    HL
07C3  C9                 .       RET
.
07C4  21 7C DB           !|.     LD     HL, $DB7C
07C7  18 03              ..      JR     $07CC
07C9  21 6C DB           !l.     LD     HL, $DB6C
.
07CC  11 46 DB           .F.     LD     DE, $DB46
07CF  C3 0C DF           ...     JP     $DF0C
07D2  3A 5D 00           :].     LD     A, ($005D)
07D5  FE 20              .       CP     $20
07D7  28 25              (%      JR     Z, $07FE
07D9  2A 5D 00           *].     LD     HL, ($005D)
07DC  CD 1D DF           ...     CALL   $DF1D
07DF  38 22              8"      JR     C, $0803
07E1  FE 10              ..      CP     $10
07E3  30 1E              0.      JR     NC $0803
07E5  5F                 _       LD     E, A
07E6  CB 27              .'      SLA    A
07E8  CB 27              .'      SLA    A
07EA  CB 27              .'      SLA    A
07EC  CB 27              .'      SLA    A
07EE  47                 G       LD     B, A
07EF  3A 04 00           :..     LD     A, ($0004)
07F2  E6 0F              ..      AND    $0F
07F4  B0                 .       OR     B
07F5  32 04 00           2..     LD     ($0004), A
07F8  0E 20              .       LD     C, $20
07FA  CD 05 00           ...     CALL   $0005
07FD  C9                 .       RET
.
07FE  21 58 DB           !X.     LD     HL, $DB58
0801  18 03              ..      JR     $0806
.
0803  21 E1 DB           !..     LD     HL, $DBE1
.
0806  11 4F DB           .O.     LD     DE, $DB4F
0809  C3 0C DF           ...     JP     $DF0C
080C  00                 .       NOP
080D  00                 .       NOP
080E  00                 .       NOP
080F  00                 .       NOP
0810  00                 .       NOP
0811  00                 .       NOP
0812  00                 .       NOP
0813  00                 .       NOP
0814  00                 .       NOP
0815  00                 .       NOP
0816  00                 .       NOP
0817  00                 .       NOP
0818  00                 .       NOP
0819  00                 .       NOP
081A  00                 .       NOP
081B  00                 .       NOP
081C  00                 .       NOP
081D  00                 .       NOP
081E  00                 .       NOP
081F  00                 .       NOP
0820  00                 .       NOP
0821  00                 .       NOP
0822  00                 .       NOP
0823  00                 .       NOP
0824  30 31              01      JR     NC $0857
0826  2E 36              .6      LD     L, $36
0828  30 39              09      JR     NC $0863
082A  C3 28 E3           .(.     JP     $E328
082D  C9                 .       RET
082E  EF                 .       RST    28H
082F  AA                 .       XOR    D
0830  EF                 .       RST    28H
0831  AA                 .       XOR    D
0832  EF                 .       RST    28H
0833  AA                 .       XOR    D
0834  EF                 .       RST    28H
0835  00                 .       NOP
0836  00                 .       NOP
0837  00                 .       NOP
0838  00                 .       NOP
0839  00                 .       NOP
083A  00                 .       NOP
083B  00                 .       NOP
083C  00                 .       NOP
083D  00                 .       NOP
083E  00                 .       NOP
083F  00                 .       NOP
0840  00                 .       NOP
0841  00                 .       NOP
0842  00                 .       NOP
0843  FF                 .       RST    38H
0844  FF                 .       RST    38H
0845  83                 .       ADD    A, E
0846  E2 00 00           ...     JP     PO $0000
0849  00                 .       NOP
084A  00                 .       NOP
084B  00                 .       NOP
084C  00                 .       NOP
084D  00                 .       NOP
084E  00                 .       NOP
084F  00                 .       NOP
0850  00                 .       NOP
0851  00                 .       NOP
0852  00                 .       NOP
0853  00                 .       NOP
0854  00                 .       NOP
0855  00                 .       NOP
0856  00                 .       NOP
.
0857  00                 .       NOP
0858  00                 .       NOP
0859  00                 .       NOP
085A  00                 .       NOP
085B  00                 .       NOP
085C  00                 .       NOP
085D  00                 .       NOP
085E  00                 .       NOP
085F  00                 .       NOP
0860  00                 .       NOP
0861  00                 .       NOP
0862  00                 .       NOP
.
0863  00                 .       NOP
0864  00                 .       NOP
0865  00                 .       NOP
0866  00                 .       NOP
0867  00                 .       NOP
0868  00                 .       NOP
0869  00                 .       NOP
086A  00                 .       NOP
086B  00                 .       NOP
086C  00                 .       NOP
086D  00                 .       NOP
086E  00                 .       NOP
086F  00                 .       NOP
0870  00                 .       NOP
0871  00                 .       NOP
0872  00                 .       NOP
0873  00                 .       NOP
0874  00                 .       NOP
0875  00                 .       NOP
0876  00                 .       NOP
0877  00                 .       NOP
0878  00                 .       NOP
0879  00                 .       NOP
087A  00                 .       NOP
087B  00                 .       NOP
087C  00                 .       NOP
087D  00                 .       NOP
087E  00                 .       NOP
087F  00                 .       NOP
0880  00                 .       NOP
0881  00                 .       NOP
0882  00                 .       NOP
0883  00                 .       NOP
0884  00                 .       NOP
0885  00                 .       NOP
0886  00                 .       NOP
0887  00                 .       NOP
0888  00                 .       NOP
0889  00                 .       NOP
088A  00                 .       NOP
088B  00                 .       NOP
088C  00                 .       NOP
088D  00                 .       NOP
088E  00                 .       NOP
088F  00                 .       NOP
0890  00                 .       NOP
0891  00                 .       NOP
0892  00                 .       NOP
0893  00                 .       NOP
0894  00                 .       NOP
0895  00                 .       NOP
0896  00                 .       NOP
0897  00                 .       NOP
0898  00                 .       NOP
0899  00                 .       NOP
089A  00                 .       NOP
089B  00                 .       NOP
089C  00                 .       NOP
089D  00                 .       NOP
089E  00                 .       NOP
089F  00                 .       NOP
08A0  00                 .       NOP
08A1  00                 .       NOP
08A2  00                 .       NOP
08A3  00                 .       NOP
08A4  00                 .       NOP
08A5  00                 .       NOP
08A6  00                 .       NOP
08A7  00                 .       NOP
08A8  00                 .       NOP
08A9  00                 .       NOP
08AA  00                 .       NOP
08AB  00                 .       NOP
08AC  00                 .       NOP
08AD  00                 .       NOP
08AE  00                 .       NOP
08AF  00                 .       NOP
08B0  00                 .       NOP
08B1  00                 .       NOP
08B2  00                 .       NOP
08B3  00                 .       NOP
08B4  00                 .       NOP
08B5  00                 .       NOP
08B6  00                 .       NOP
08B7  00                 .       NOP
08B8  00                 .       NOP
08B9  00                 .       NOP
08BA  00                 .       NOP
08BB  00                 .       NOP
08BC  00                 .       NOP
08BD  00                 .       NOP
08BE  00                 .       NOP
08BF  00                 .       NOP
08C0  00                 .       NOP
08C1  00                 .       NOP
08C2  00                 .       NOP
08C3  00                 .       NOP
08C4  00                 .       NOP
08C5  00                 .       NOP
08C6  00                 .       NOP
08C7  00                 .       NOP
08C8  00                 .       NOP
08C9  00                 .       NOP
08CA  00                 .       NOP
08CB  00                 .       NOP
08CC  00                 .       NOP
08CD  00                 .       NOP
08CE  00                 .       NOP
08CF  00                 .       NOP
08D0  00                 .       NOP
08D1  00                 .       NOP
08D2  00                 .       NOP
08D3  00                 .       NOP
08D4  00                 .       NOP
08D5  00                 .       NOP
08D6  00                 .       NOP
08D7  00                 .       NOP
08D8  00                 .       NOP
08D9  00                 .       NOP
08DA  00                 .       NOP
08DB  00                 .       NOP
08DC  00                 .       NOP
08DD  00                 .       NOP
08DE  00                 .       NOP
08DF  00                 .       NOP
08E0  00                 .       NOP
08E1  00                 .       NOP
08E2  00                 .       NOP
08E3  00                 .       NOP
08E4  00                 .       NOP
08E5  00                 .       NOP
08E6  00                 .       NOP
08E7  00                 .       NOP
08E8  00                 .       NOP
08E9  00                 .       NOP
08EA  4E                 N       LD     C, (HL)
08EB  6F                 o       LD     L, A
08EC  20 64               d      JR     NZ $0952
08EE  72                 r       LD     (HL), D
08EF  69                 i       LD     L, C
08F0  76                 v       HALT
08F1  65                 e       LD     H, L
08F2  24                 $       INC    H
08F3  0D                 .       DEC    C
08F4  52                 R       LD     D, D
08F5  65                 e       LD     H, L
08F6  61                 a       LD     H, C
08F7  64                 d       LD     H, H
08F8  24                 $       INC    H
08F9  0D                 .       DEC    C
08FA  57                 W       LD     D, A
08FB  72                 r       LD     (HL), D
08FC  69                 i       LD     L, C
08FD  74                 t       LD     (HL), H
08FE  65                 e       LD     H, L
08FF  24                 $       INC    H
0900  44                 D       LD     B, H
0901  69                 i       LD     L, C
0902  73                 s       LD     (HL), E
0903  63                 c       LD     H, E
0904  20 52               R      JR     NZ $0958
0906  2F                 /       CPL
0907  4F                 O       LD     C, A
0908  24                 $       INC    H
0909  46                 F       LD     B, (HL)
090A  69                 i       LD     L, C
090B  6C                 l       LD     L, H
090C  65                 e       LD     H, L
090D  20 52               R      JR     NZ $0961
090F  2F                 /       CPL
0910  4F                 O       LD     C, A
0911  24                 $       INC    H
0912  20 65               e      JR     NZ $0979
0914  72                 r       LD     (HL), D
0915  72                 r       LD     (HL), D
0916  6F                 o       LD     L, A
0917  72                 r       LD     (HL), D
0918  20 6F               o      JR     NZ $0989
091A  6E                 n       LD     L, (HL)
091B  20 41               A      JR     NZ $095E
091D  3A 20 52           : R     LD     A, ($5220)
0920  29                 )       ADD    HL, HL
0921  65                 e       LD     H, L
0922  74                 t       LD     (HL), H
0923  72                 r       LD     (HL), D
0924  79                 y       LD     A, C
0925  2C                 ,       INC    L
0926  20 49               I      JR     NZ $0971
0928  29                 )       ADD    HL, HL
0929  67                 g       LD     H, A
092A  6E                 n       LD     L, (HL)
092B  6F                 o       LD     L, A
092C  72                 r       LD     (HL), D
092D  65                 e       LD     H, L
092E  20 6F               o      JR     NZ $099F
0930  72                 r       LD     (HL), D
0931  20 57               W      JR     NZ $098A
0933  29                 )       ADD    HL, HL
0934  61                 a       LD     H, C
0935  72                 r       LD     (HL), D
0936  6D                 m       LD     L, L
0937  20 62               b      JR     NZ $099B
0939  6F                 o       LD     L, A
093A  6F                 o       LD     L, A
093B  74                 t       LD     (HL), H
093C  3A 20 08           : .     LD     A, ($0820)
093F  24                 $       INC    H
0940  20 65               e      JR     NZ $09A7
0942  72                 r       LD     (HL), D
0943  72                 r       LD     (HL), D
0944  6F                 o       LD     L, A
0945  72                 r       LD     (HL), D
0946  20 6F               o      JR     NZ $09B7
0948  6E                 n       LD     L, (HL)
0949  20 00               .      JR     NZ $094B
.
094B  24                 $       INC    H
094C  3E 28              >(      LD     A, $28
094E  B9                 .       CP     C
094F  D8                 .       RET    C
0950  06 00              ..      LD     B, $00
.
0952  CB 21              .!      SLA    C
0954  ED 73 A2 E2        .s..    LD     ($E2A2), SP
.
0958  31 C6 E2           1..     LD     SP, $E2C6
095B  DD E5              ..      PUSH   IX
095D  FD E5              ..      PUSH   IY
095F  21 5E E3           !^.     LD     HL, $E35E
0962  09                 .       ADD    HL, BC
0963  7E                 ~       LD     A, (HL)
0964  23                 #       INC    HL
0965  66                 f       LD     H, (HL)
0966  6F                 o       LD     L, A
0967  4B                 K       LD     C, E
0968  CD 5D E3           .].     CALL   $E35D
096B  F5                 .       PUSH   AF
096C  C5                 .       PUSH   BC
096D  ED 4B 1D E2        .K..    LD     BC, ($E21D)
.
0971  CD 24 F0           .$.     CALL   $F024
0974  C1                 .       POP    BC
0975  F1                 .       POP    AF
0976  6F                 o       LD     L, A
0977  60                 `       LD     H, B
0978  FD E1              ..      POP    IY
097A  DD E1              ..      POP    IX
097C  ED 7B A2 E2        .{..    LD     SP, ($E2A2)
0980  C9                 .       RET
0981  E9                 .       JP     (HL)
0982  03                 .       INC    BC
0983  F0                 .       RET    P
0984  B0                 .       OR     B
0985  E3                 .       EX     (SP), HL
0986  D9                 .       EXX
0987  E3                 .       EX     (SP), HL
0988  15                 .       DEC    D
.
0989  F0                 .       RET    P
.
098A  12                 .       LD     (DE), A
098B  F0                 .       RET    P
098C  0F                 .       RCCA
098D  F0                 .       RET    P
098E  4B                 K       LD     C, E
098F  E4 5E E4           .^.     CALL   PO, $E45E
0992  62                 b       LD     H, D
0993  E4 67 E4           .g.     CALL   PO, $E467
0996  74                 t       LD     (HL), H
0997  E4 29 E4           .).     CALL   PO, $E429
099A  D6 E5              ..      SUB    $E5
099C  DC E5 F8           ...     CALL   C, $F8E5
.
099F  E5                 .       PUSH   HL
09A0  E1                 .       POP    HL
09A1  E6 4B              .K      AND    $4B
09A3  E7                 .       RST    20H
09A4  E4 E7 07           ...     CALL   PO, $07E7
.
09A7  E8                 .       RET    PE
09A8  22 E8 89           "..     LD     ($89E8), HL
09AB  E8                 .       RET    PE
09AC  C0                 .       RET    NZ
09AD  E8                 .       RET    PE
09AE  40                 @       LD     B, B
09AF  E9                 .       JP     (HL)
09B0  E0                 .       RET    PO
09B1  E9                 .       JP     (HL)
09B2  36 EA              6.      LD     (HL), $EA
09B4  3C                 <       INC    A
09B5  EA 40 EA           .@.     JP     PE $EA40
09B8  45                 E       LD     B, L
09B9  EA 52 EA           .R.     JP     PE $EA52
09BC  5F                 _       LD     E, A
09BD  EA 65 EA           .e.     JP     PE $EA65
09C0  6E                 n       LD     L, (HL)
09C1  EA 7B EA           .{.     JP     PE $EA7B
09C4  87                 .       ADD    A, A
09C5  EA D1 EA           ...     JP     PE $EAD1
09C8  80                 .       ADD    A, B
09C9  EB                 .       EX     DE, HL
09CA  E2 EB F4           ...     JP     PO $F4EB
09CD  EB                 .       EX     DE, HL
09CE  5C                 \       LD     E, H
09CF  E3                 .       EX     (SP), HL
09D0  5C                 \       LD     E, H
09D1  E3                 .       EX     (SP), HL
09D2  D5                 .       PUSH   DE
09D3  EA CD CE           ...     JP     PE $CECD
09D6  E3                 .       EX     (SP), HL
09D7  21 CA E3           !..     LD     HL, $E3CA
09DA  01 04 00           ...     LD     BC, $0004
09DD  ED B1              ..      CPIR
09DF  28 06              (.      JR     Z, $09E7
09E1  FE 20              .       CP     $20
09E3  D8                 .       RET    C
09E4  FE 7F              .      CP     $7F
09E6  C8                 .       RET    Z
.
09E7  F5                 .       PUSH   AF
09E8  5F                 _       LD     E, A
09E9  CD D9 E3           ...     CALL   $E3D9
09EC  F1                 .       POP    AF
09ED  C9                 .       RET
09EE  08                 .       EX     AF, AF\'
09EF  09                 .       ADD    HL, BC
09F0  0A                 .       LD     A, (BC)
09F1  0D                 .       DEC    C
09F2  21 11 E2           !..     LD     HL, $E211
09F5  7E                 ~       LD     A, (HL)
09F6  36 00              6.      LD     (HL), $00
09F8  B7                 .       OR     A
09F9  C0                 .       RET    NZ
09FA  C3 09 F0           ...     JP     $F009
09FD  D5                 .       PUSH   DE
09FE  3A 13 E2           :..     LD     A, ($E213)
0A01  4F                 O       LD     C, A
0A02  7B                 {       LD     A, E
0A03  FE 09              ..      CP     $09
0A05  28 19              (.      JR     Z, $0A20
0A07  FE 0D              ..      CP     $0D
0A09  28 28              ((      JR     Z, $0A33
0A0B  FE 08              ..      CP     $08
0A0D  28 28              ((      JR     Z, $0A37
0A0F  FE 20              .       CP     $20
0A11  38 05              8.      JR     C, $0A18
0A13  FE 7F              .      CP     $7F
0A15  28 01              (.      JR     Z, $0A18
0A17  0C                 .       INC    C
.
0A18  79                 y       LD     A, C
0A19  32 13 E2           2..     LD     ($E213), A
0A1C  C1                 .       POP    BC
0A1D  C3 16 E4           ...     JP     $E416
.
0A20  D1                 .       POP    DE
.
0A21  C5                 .       PUSH   BC
0A22  0E 20              .       LD     C, $20
0A24  CD 16 E4           ...     CALL   $E416
0A27  C1                 .       POP    BC
0A28  0C                 .       INC    C
0A29  79                 y       LD     A, C
0A2A  E6 07              ..      AND    $07
0A2C  20 F3               .      JR     NZ $0A21
0A2E  79                 y       LD     A, C
0A2F  32 13 E2           2..     LD     ($E213), A
0A32  C9                 .       RET
.
0A33  0E 00              ..      LD     C, $00
0A35  18 E1              ..      JR     $0A18
.
0A37  0D                 .       DEC    C
0A38  18 DE              ..      JR     $0A18
0A3A  C5                 .       PUSH   BC
0A3B  CD 29 E4           .).     CALL   $E429
0A3E  C1                 .       POP    BC
0A3F  3A 12 E2           :..     LD     A, ($E212)
0A42  B7                 .       OR     A
0A43  28 05              (.      JR     Z, $0A4A
0A45  C5                 .       PUSH   BC
0A46  CD 0F F0           ...     CALL   $F00F
0A49  C1                 .       POP    BC
.
0A4A  C3 0C F0           ...     JP     $F00C
0A4D  3A 11 E2           :..     LD     A, ($E211)
0A50  B7                 .       OR     A
0A51  20 19               .      JR     NZ $0A6C
0A53  CD 06 F0           ...     CALL   $F006
0A56  B7                 .       OR     A
0A57  C8                 .       RET    Z
0A58  CD 09 F0           ...     CALL   $F009
0A5B  FE 13              ..      CP     $13
0A5D  20 0A               .      JR     NZ $0A69
0A5F  CD 09 F0           ...     CALL   $F009
0A62  FE 03              ..      CP     $03
0A64  CA 00 00           ...     JP     Z $0000
0A67  AF                 .       XOR    A
0A68  C9                 .       RET
.
0A69  32 11 E2           2..     LD     ($E211), A
.
0A6C  3E FF              >.      LD     A, $FF
0A6E  C9                 .       RET
0A6F  79                 y       LD     A, C
0A70  3C                 <       INC    A
0A71  28 07              (.      JR     Z, $0A7A
0A73  3C                 <       INC    A
0A74  CA 06 F0           ...     JP     Z $F006
0A77  C3 0C F0           ...     JP     $F00C
.
0A7A  CD 06 F0           ...     CALL   $F006
0A7D  B7                 .       OR     A
0A7E  C4 09 F0           ...     CALL   NZ, $F009
0A81  C9                 .       RET
0A82  3A 03 00           :..     LD     A, ($0003)
0A85  C9                 .       RET
0A86  7B                 {       LD     A, E
0A87  32 03 00           2..     LD     ($0003), A
0A8A  C9                 .       RET
.
0A8B  1A                 .       LD     A, (DE)
0A8C  FE 24              .$      CP     $24
0A8E  C8                 .       RET    Z
0A8F  13                 .       INC    DE
0A90  D5                 .       PUSH   DE
0A91  5F                 _       LD     E, A
0A92  CD D9 E3           ...     CALL   $E3D9
0A95  D1                 .       POP    DE
0A96  18 F3              ..      JR     $0A8B
0A98  ED 53 14 E2        .S..    LD     ($E214), DE
0A9C  1A                 .       LD     A, (DE)
0A9D  13                 .       INC    DE
0A9E  13                 .       INC    DE
.
0A9F  ED 53 16 E2        .S..    LD     ($E216), DE
0AA3  32 18 E2           2..     LD     ($E218), A
0AA6  B7                 .       OR     A
0AA7  CA EB E4           ...     JP     Z $E4EB
0AAA  21 11 E2           !..     LD     HL, $E211
0AAD  7E                 ~       LD     A, (HL)
0AAE  36 00              6.      LD     (HL), $00
0AB0  B7                 .       OR     A
0AB1  CC 09 F0           ...     CALL   Z, $F009
0AB4  FE 03              ..      CP     $03
0AB6  CA FE E4           ...     JP     Z $E4FE
0AB9  FE 05              ..      CP     $05
0ABB  CA 08 E5           ...     JP     Z $E508
0ABE  FE 08              ..      CP     $08
0AC0  CA 15 E5           ...     JP     Z $E515
0AC3  FE 09              ..      CP     $09
0AC5  CA 48 E5           .H.     JP     Z $E548
0AC8  FE 0A              ..      CP     $0A
0ACA  CA EB E4           ...     JP     Z $E4EB
0ACD  FE 0D              ..      CP     $0D
0ACF  CA E6 E4           ...     JP     Z $E4E6
0AD2  FE 10              ..      CP     $10
0AD4  CA 59 E5           .Y.     JP     Z $E559
0AD7  FE 12              ..      CP     $12
0AD9  CA 64 E5           .d.     JP     Z $E564
0ADC  FE 15              ..      CP     $15
0ADE  CA 83 E5           ...     JP     Z $E583
0AE1  FE 18              ..      CP     $18
0AE3  CA 8D E5           ...     JP     Z $E58D
0AE6  FE 7F              .      CP     $7F
0AE8  CA 9C E5           ...     JP     Z $E59C
.
0AEB  FE 20              .       CP     $20
0AED  F5                 .       PUSH   AF
0AEE  30 09              0.      JR     NC $0AF9
0AF0  1E 5E              .^      LD     E, $5E
0AF2  CD D9 E3           ...     CALL   $E3D9
0AF5  F1                 .       POP    AF
0AF6  F5                 .       PUSH   AF
0AF7  C6 40              .@      ADD    A, $40
.
0AF9  5F                 _       LD     E, A
0AFA  CD D9 E3           ...     CALL   $E3D9
0AFD  F1                 .       POP    AF
0AFE  ED 5B 16 E2        .[..    LD     DE, ($E216)
0B02  12                 .       LD     (DE), A
0B03  13                 .       INC    DE
0B04  3A 18 E2           :..     LD     A, ($E218)
0B07  3D                 =       DEC    A
0B08  18 95              ..      JR     $0A9F
0B0A  1E 0D              ..      LD     E, $0D
0B0C  CD D9 E3           ...     CALL   $E3D9
0B0F  CD BE E5           ...     CALL   $E5BE
0B12  1B                 .       DEC    DE
0B13  12                 .       LD     (DE), A
0B14  C8                 .       RET    Z
0B15  47                 G       LD     B, A
0B16  3E 09              >.      LD     A, $09
0B18  EB                 .       EX     DE, HL
.
0B19  23                 #       INC    HL
0B1A  CB 7E              .~      BIT    7, (HL)
0B1C  28 01              (.      JR     Z, $0B1F
0B1E  77                 w       LD     (HL), A
.
0B1F  10 F8              ..      DJNZ   $0B19
0B21  C9                 .       RET
0B22  F5                 .       PUSH   AF
0B23  CD BE E5           ...     CALL   $E5BE
0B26  CA 03 F0           ...     JP     Z $F003
0B29  F1                 .       POP    AF
0B2A  18 BF              ..      JR     $0AEB
0B2C  11 12 E5           ...     LD     DE, $E512
0B2F  CD 67 E4           .g.     CALL   $E467
0B32  C3 86 E4           ...     JP     $E486
0B35  23                 #       INC    HL
0B36  0D                 .       DEC    C
0B37  0A                 .       LD     A, (BC)
0B38  24                 $       INC    H
0B39  CD 1B E5           ...     CALL   $E51B
0B3C  C3 86 E4           ...     JP     $E486
0B3F  CD BE E5           ...     CALL   $E5BE
0B42  C8                 .       RET    Z
0B43  ED 5B 16 E2        .[..    LD     DE, ($E216)
0B47  1B                 .       DEC    DE
0B48  04                 .       INC    B
0B49  ED 53 16 E2        .S..    LD     ($E216), DE
0B4D  78                 x       LD     A, B
0B4E  32 18 E2           2..     LD     ($E218), A
0B51  06 01              ..      LD     B, $01
0B53  1A                 .       LD     A, (DE)
0B54  CB 7F              .      BIT    7, A
0B56  28 05              (.      JR     Z, $0B5D
0B58  47                 G       LD     B, A
0B59  CB B8              ..      RES    7, B
0B5B  18 05              ..      JR     $0B62
.
0B5D  FE 20              .       CP     $20
0B5F  30 01              0.      JR     NC $0B62
0B61  04                 .       INC    B
.
0B62  C5                 .       PUSH   BC
0B63  1E 08              ..      LD     E, $08
0B65  CD D9 E3           ...     CALL   $E3D9
0B68  C1                 .       POP    BC
0B69  10 F7              ..      DJNZ   $0B62
0B6B  C9                 .       RET
0B6C  3A 13 E2           :..     LD     A, ($E213)
0B6F  E6 07              ..      AND    $07
0B71  D6 08              ..      SUB    $08
0B73  ED 44              .D      NEG
0B75  CB FF              ..      SET    7, A
0B77  F5                 .       PUSH   AF
0B78  3E 09              >.      LD     A, $09
0B7A  C3 D5 E4           ...     JP     $E4D5
0B7D  3A 12 E2           :..     LD     A, ($E212)
0B80  EE 01              ..      XOR    $01
0B82  32 12 E2           2..     LD     ($E212), A
0B85  C3 86 E4           ...     JP     $E486
0B88  CD D0 E5           ...     CALL   $E5D0
0B8B  CD BE E5           ...     CALL   $E5BE
0B8E  CA 86 E4           ...     JP     Z $E486
0B91  47                 G       LD     B, A
.
0B92  1A                 .       LD     A, (DE)
0B93  C5                 .       PUSH   BC
0B94  D5                 .       PUSH   DE
0B95  CB 7F              .      BIT    7, A
0B97  28 02              (.      JR     Z, $0B9B
0B99  3E 09              >.      LD     A, $09
.
0B9B  5F                 _       LD     E, A
0B9C  CD D9 E3           ...     CALL   $E3D9
0B9F  D1                 .       POP    DE
0BA0  C1                 .       POP    BC
0BA1  13                 .       INC    DE
0BA2  10 EE              ..      DJNZ   $0B92
0BA4  C3 86 E4           ...     JP     $E486
0BA7  CD D0 E5           ...     CALL   $E5D0
.
0BAA  ED 5B 14 E2        .[..    LD     DE, ($E214)
0BAE  C3 74 E4           .t.     JP     $E474
0BB1  CD BE E5           ...     CALL   $E5BE
0BB4  28 F4              (.      JR     Z, $0BAA
0BB6  47                 G       LD     B, A
.
0BB7  C5                 .       PUSH   BC
0BB8  CD 1B E5           ...     CALL   $E51B
0BBB  C1                 .       POP    BC
0BBC  10 F9              ..      DJNZ   $0BB7
0BBE  18 EA              ..      JR     $0BAA
0BC0  CD BE E5           ...     CALL   $E5BE
0BC3  CA 86 E4           ...     JP     Z $E486
0BC6  ED 5B 16 E2        .[..    LD     DE, ($E216)
0BCA  1B                 .       DEC    DE
0BCB  1A                 .       LD     A, (DE)
0BCC  CB 7F              .      BIT    7, A
0BCE  28 02              (.      JR     Z, $0BD2
0BD0  3E 09              >.      LD     A, $09
.
0BD2  04                 .       INC    B
0BD3  ED 53 16 E2        .S..    LD     ($E216), DE
0BD7  5F                 _       LD     E, A
0BD8  78                 x       LD     A, B
0BD9  32 18 E2           2..     LD     ($E218), A
0BDC  CD D9 E3           ...     CALL   $E3D9
0BDF  C3 86 E4           ...     JP     $E486
0BE2  2A 16 E2           *..     LD     HL, ($E216)
0BE5  ED 5B 14 E2        .[..    LD     DE, ($E214)
0BE9  3A 18 E2           :..     LD     A, ($E218)
0BEC  47                 G       LD     B, A
0BED  13                 .       INC    DE
0BEE  13                 .       INC    DE
0BEF  A7                 .       AND    A
0BF0  ED 52              .R      SBC    HL, DE
0BF2  7D                 }       LD     A, L
0BF3  C9                 .       RET
0BF4  11 11 E5           ...     LD     DE, $E511
0BF7  C3 67 E4           .g.     JP     $E467
0BFA  21 22 00           !".     LD     HL, $0022
0BFD  7D                 }       LD     A, L
0BFE  44                 D       LD     B, H
0BFF  C9                 .       RET
0C00  21 00 00           !..     LD     HL, $0000
0C03  22 19 E2           "..     LD     ($E219), HL
0C06  22 1B E2           "..     LD     ($E21B), HL
0C09  21 80 00           !..     LD     HL, $0080
0C0C  22 1D E2           "..     LD     ($E21D), HL
0C0F  3E FF              >.      LD     A, $FF
0C11  32 20 E2           2 .     LD     ($E220), A
0C14  32 1F E2           2..     LD     ($E21F), A
0C17  CD 18 F0           ...     CALL   $F018
0C1A  1E 00              ..      LD     E, $00
0C1C  7B                 {       LD     A, E
0C1D  32 1F E2           2..     LD     ($E21F), A
0C20  3A 20 E2           : .     LD     A, ($E220)
0C23  BB                 .       CP     E
0C24  C8                 .       RET    Z
0C25  7B                 {       LD     A, E
0C26  32 20 E2           2 .     LD     ($E220), A
0C29  21 85 E2           !..     LD     HL, $E285
0C2C  ED 5B 21 E2        .[!.    LD     DE, ($E221)
0C30  13                 .       INC    DE
0C31  13                 .       INC    DE
0C32  01 06 00           ...     LD     BC, $0006
0C35  ED B0              ..      LDIR
0C37  4F                 O       LD     C, A
0C38  CD 1B F0           ...     CALL   $F01B
0C3B  7C                 |       LD     A, H
0C3C  B5                 .       OR     L
0C3D  CA 88 EF           ...     JP     Z $EF88
0C40  22 21 E2           "!.     LD     ($E221), HL
0C43  11 83 E2           ...     LD     DE, $E283
0C46  01 10 00           ...     LD     BC, $0010
0C49  ED B0              ..      LDIR
0C4B  2A 8D E2           *..     LD     HL, ($E28D)
0C4E  01 0F 00           ...     LD     BC, $000F
0C51  ED B0              ..      LDIR
0C53  3A 20 E2           : .     LD     A, ($E220)
0C56  2A 19 E2           *..     LD     HL, ($E219)
0C59  CD 9F ED           ...     CALL   $ED9F
0C5C  D8                 .       RET    C
0C5D  22 19 E2           "..     LD     ($E219), HL
0C60  AF                 .       XOR    A
0C61  32 23 E2           2#.     LD     ($E223), A
0C64  CD D8 EC           ...     CALL   $ECD8
0C67  2A 8D E2           *..     LD     HL, ($E28D)
0C6A  11 93 E2           ...     LD     DE, $E293
0C6D  01 0F 00           ...     LD     BC, $000F
0C70  ED B0              ..      LDIR
0C72  2A 9A E2           *..     LD     HL, ($E29A)
0C75  CB 3C              .<      SRL    H
0C77  CB 1D              ..      RR     L
0C79  CB 3C              .<      SRL    H
0C7B  CB 1D              ..      RR     L
0C7D  3A 86 E2           :..     LD     A, ($E286)
0C80  BD                 .       CP     L
0C81  7D                 }       LD     A, L
0C82  38 03              8.      JR     C, $0C87
0C84  32 86 E2           2..     LD     ($E286), A
.
0C87  32 87 E2           2..     LD     ($E287), A
0C8A  3A 99 E2           :..     LD     A, ($E299)
0C8D  B7                 .       OR     A
0C8E  3E 00              >.      LD     A, $00
0C90  28 01              (.      JR     Z, $0C93
0C92  2F                 /       CPL
.
0C93  32 85 E2           2..     LD     ($E285), A
0C96  ED 4B 98 E2        .K..    LD     BC, ($E298)
0C9A  03                 .       INC    BC
0C9B  CB 38              .8      SRL    B
0C9D  CB 19              ..      RR     C
0C9F  CB 38              .8      SRL    B
0CA1  CB 19              ..      RR     C
0CA3  CB 38              .8      SRL    B
0CA5  CB 19              ..      RR     C
0CA7  2A 91 E2           *..     LD     HL, ($E291)
0CAA  ED 5B 9C E2        .[..    LD     DE, ($E29C)
0CAE  73                 s       LD     (HL), E
0CAF  23                 #       INC    HL
0CB0  72                 r       LD     (HL), D
0CB1  23                 #       INC    HL
0CB2  5D                 ]       LD     E, L
0CB3  54                 T       LD     D, H
0CB4  36 00              6.      LD     (HL), $00
0CB6  13                 .       INC    DE
0CB7  0B                 .       DEC    BC
0CB8  0B                 .       DEC    BC
0CB9  0B                 .       DEC    BC
0CBA  ED B0              ..      LDIR
0CBC  3A 98 E2           :..     LD     A, ($E298)
0CBF  3C                 <       INC    A
0CC0  E6 07              ..      AND    $07
0CC2  28 08              (.      JR     Z, $0CCC
0CC4  47                 G       LD     B, A
0CC5  3E FF              >.      LD     A, $FF
.
0CC7  CB 3F              .?      SRL    A
0CC9  10 FC              ..      DJNZ   $0CC7
0CCB  12                 .       LD     (DE), A
.
0CCC  AF                 .       XOR    A
0CCD  32 86 E2           2..     LD     ($E286), A
.
0CD0  32 23 E2           2#.     LD     ($E223), A
0CD3  CD D8 EC           ...     CALL   $ECD8
0CD6  CD 52 ED           .R.     CALL   $ED52
0CD9  38 01              8.      JR     C, $0CDC
0CDB  12                 .       LD     (DE), A
.
0CDC  CD B3 ED           ...     CALL   $EDB3
0CDF  3A 23 E2           :#.     LD     A, ($E223)
0CE2  38 08              8.      JR     C, $0CEC
0CE4  21 87 E2           !..     LD     HL, $E287
0CE7  BE                 .       CP     (HL)
0CE8  C8                 .       RET    Z
0CE9  3C                 <       INC    A
0CEA  18 E4              ..      JR     $0CD0
.
0CEC  3C                 <       INC    A
0CED  4F                 O       LD     C, A
0CEE  06 00              ..      LD     B, $00
0CF0  2A 9E E2           *..     LD     HL, ($E29E)
0CF3  7C                 |       LD     A, H
0CF4  B5                 .       OR     L
0CF5  C8                 .       RET    Z
0CF6  2A 8F E2           *..     LD     HL, ($E28F)
0CF9  09                 .       ADD    HL, BC
0CFA  3A 87 E2           :..     LD     A, ($E287)
.
0CFD  B9                 .       CP     C
0CFE  D8                 .       RET    C
0CFF  36 80              6.      LD     (HL), $80
0D01  23                 #       INC    HL
0D02  0C                 .       INC    C
0D03  18 F8              ..      JR     $0CFD
0D05  CD 64 EF           .d.     CALL   $EF64
0D08  21 00 80           !..     LD     HL, $8000
0D0B  22 5F E2           "_.     LD     ($E25F), HL
0D0E  CD F2 E6           ...     CALL   $E6F2
0D11  B7                 .       OR     A
0D12  F4 72 EF           .r.     CALL   P, $EF72
0D15  C9                 .       RET
0D16  21 52 E2           !R.     LD     HL, $E252
0D19  11 2E E2           ...     LD     DE, $E22E
0D1C  01 24 00           .$.     LD     BC, $0024
0D1F  ED B0              ..      LDIR
0D21  3A 5E E2           :^.     LD     A, ($E25E)
0D24  32 28 E2           2(.     LD     ($E228), A
0D27  CD 0B EC           ...     CALL   $EC0B
0D2A  B7                 .       OR     A
0D2B  F2 16 E7           ...     JP     P $E716
0D2E  21 2E E2           !..     LD     HL, $E22E
0D31  11 52 E2           .R.     LD     DE, $E252
0D34  01 24 00           .$.     LD     BC, $0024
0D37  ED B0              ..      LDIR
0D39  C9                 .       RET
0D3A  F5                 .       PUSH   AF
0D3B  CD 2F EF           ./.     CALL   $EF2F
0D3E  11 52 E2           .R.     LD     DE, $E252
0D41  01 1F 00           ...     LD     BC, $001F
0D44  13                 .       INC    DE
0D45  23                 #       INC    HL
0D46  ED B0              ..      LDIR
0D48  DD 21 52 E2        .!R.    LD     IX, $E252
0D4C  DD 36 0D 00        .6..    
0D50  DD CB              ..      ****BUG****			DD CB 05 FE   SET 7,(IX+05)
0D52  0E FE              ..      LD     C, $FE
0D54  3A 28 E2           :(.     LD     A, ($E228)
0D57  DD BE 0C           ...     CP     (IX+$0C)
0D5A  28 0F              (.      JR     Z, $0D6B
.
0D5C  32 5E E2           2^.     LD     ($E25E), A
0D5F  38 06              8.      JR     C, $0D67
0D61  DD 36 0F 00        .6..    
0D65  18 04              ..      JR     $0D6B
.
0D67  DD 36 0F 80        .6..    
.
0D6B  F1                 .       POP    AF
0D6C  06 00              ..      LD     B, $00
0D6E  C9                 .       RET
0D6F  CD 64 EF           .d.     CALL   $EF64
0D72  DD 21 52 E2        .!R.    LD     IX, $E252
0D76  DD CB              ..      ****BUG****			DD CB 05 FE   SET 7,(IX+05)
0D78  0E 7E              .~      LD     C, $7E
0D7A  28 06              (.      JR     Z, $0D82
0D7C  CD D8 EC           ...     CALL   $ECD8
0D7F  AF                 .       XOR    A
0D80  47                 G       LD     B, A
0D81  C9                 .       RET
.
0D82  AF                 .       XOR    A
0D83  32 5F E2           2_.     LD     ($E25F), A
0D86  CD 3A EF           .:.     CALL   $EF3A
0D89  CD 0B EC           ...     CALL   $EC0B
0D8C  B7                 .       OR     A
0D8D  06 00              ..      LD     B, $00
0D8F  F8                 .       RET    M
0D90  32 29 E2           2).     LD     ($E229), A
0D93  CD 2F EF           ./.     CALL   $EF2F
0D96  E5                 .       PUSH   HL
0D97  DD 21 52 E2        .!R.    LD     IX, $E252
0D9B  CD D3 EE           ...     CALL   $EED3
0D9E  EB                 .       EX     DE, HL
0D9F  DD E1              ..      POP    IX
0DA1  CD D3 EE           ...     CALL   $EED3
0DA4  AF                 .       XOR    A
0DA5  EB                 .       EX     DE, HL
0DA6  ED 52              .R      SBC    HL, DE
0DA8  38 12              8.      JR     C, $0DBC
0DAA  3A 5E E2           :^.     LD     A, ($E25E)
0DAD  DD 77 0C           .w.     LD     (IX+$0C), A
0DB0  3A 60 E2           :`.     LD     A, ($E260)
0DB3  DD 77 0E           .w.     LD     (IX+$0E), A
0DB6  3A 61 E2           :a.     LD     A, ($E261)
0DB9  DD 77 0F           .w.     LD     (IX+$0F), A
.
0DBC  DD E5              ..      PUSH   IX
0DBE  E1                 .       POP    HL
0DBF  11 52 E2           .R.     LD     DE, $E252
0DC2  01 10 00           ...     LD     BC, $0010
0DC5  09                 .       ADD    HL, BC
0DC6  EB                 .       EX     DE, HL
0DC7  09                 .       ADD    HL, BC
0DC8  D5                 .       PUSH   DE
0DC9  3A 97 E2           :..     LD     A, ($E297)
0DCC  3C                 <       INC    A
0DCD  06 05              ..      LD     B, $05
0DCF  0E 00              ..      LD     C, $00
.
0DD1  1F                 .       RRA
0DD2  CB 11              ..      RL     C
0DD4  10 FB              ..      DJNZ   $0DD1
0DD6  3A 5E E2           :^.     LD     A, ($E25E)
0DD9  47                 G       LD     B, A
0DDA  3A 97 E2           :..     LD     A, ($E297)
0DDD  A0                 .       AND    B
0DDE  06 00              ..      LD     B, $00
0DE0  3C                 <       INC    A
.
0DE1  3D                 =       DEC    A
0DE2  28 06              (.      JR     Z, $0DEA
0DE4  09                 .       ADD    HL, BC
0DE5  EB                 .       EX     DE, HL
0DE6  09                 .       ADD    HL, BC
0DE7  EB                 .       EX     DE, HL
0DE8  18 F7              ..      JR     $0DE1
.
0DEA  ED B0              ..      LDIR
0DEC  D1                 .       POP    DE
0DED  2A 24 E2           *$.     LD     HL, ($E224)
0DF0  01 10 00           ...     LD     BC, $0010
0DF3  09                 .       ADD    HL, BC
0DF4  EB                 .       EX     DE, HL
0DF5  ED B0              ..      LDIR
0DF7  CD 52 ED           .R.     CALL   $ED52
0DFA  38 01              8.      JR     C, $0DFD
0DFC  12                 .       LD     (DE), A
.
0DFD  0E 01              ..      LD     C, $01
0DFF  CD 05 ED           ...     CALL   $ED05
0E02  3A 29 E2           :).     LD     A, ($E229)
0E05  06 00              ..      LD     B, $00
0E07  C9                 .       RET
0E08  ED 53 26 E2        .S&.    LD     ($E226), DE
0E0C  CD 64 EF           .d.     CALL   $EF64
0E0F  21 5F E2           !_.     LD     HL, $E25F
0E12  36 00              6.      LD     (HL), $00
0E14  3A 52 E2           :R.     LD     A, ($E252)
0E17  FE 3F              .?      CP     $3F
0E19  28 08              (.      JR     Z, $0E23
0E1B  23                 #       INC    HL
0E1C  7E                 ~       LD     A, (HL)
0E1D  FE 3F              .?      CP     $3F
0E1F  28 02              (.      JR     Z, $0E23
0E21  36 00              6.      LD     (HL), $00
.
0E23  CD 72 EF           .r.     CALL   $EF72
0E26  CD 0B EC           ...     CALL   $EC0B
0E29  18 0A              ..      JR     $0E35
0E2B  ED 5B 26 E2        .[&.    LD     DE, ($E226)
0E2F  CD 64 EF           .d.     CALL   $EF64
0E32  CD 16 EC           ...     CALL   $EC16
.
0E35  B7                 .       OR     A
0E36  06 00              ..      LD     B, $00
0E38  F8                 .       RET    M
0E39  2A 8B E2           *..     LD     HL, ($E28B)
0E3C  ED 5B 1D E2        .[..    LD     DE, ($E21D)
0E40  01 80 00           ...     LD     BC, $0080
0E43  ED B0              ..      LDIR
0E45  C9                 .       RET
0E46  CD 64 EF           .d.     CALL   $EF64
0E49  3E 3F              >?      LD     A, $3F
0E4B  32 5E E2           2^.     LD     ($E25E), A
0E4E  32 60 E2           2`.     LD     ($E260), A
0E51  AF                 .       XOR    A
0E52  32 5F E2           2_.     LD     ($E25F), A
0E55  CD 0B EC           ...     CALL   $EC0B
0E58  B7                 .       OR     A
0E59  06 00              ..      LD     B, $00
0E5B  F8                 .       RET    M
0E5C  F5                 .       PUSH   AF
0E5D  CD 2F EF           ./.     CALL   $EF2F
0E60  E5                 .       PUSH   HL
0E61  DD E1              ..      POP    IX
0E63  DD CB              ..      ****BUG****			DD CB 05 FE   SET 7,(IX+05)
0E65  09                 .       ADD    HL, BC
0E66  7E                 ~       LD     A, (HL)
0E67  C2 A3 EF           ...     JP     NZ $EFA3
0E6A  36 E5              6.      LD     (HL), $E5
0E6C  E5                 .       PUSH   HL
0E6D  CD 52 ED           .R.     CALL   $ED52
0E70  38 01              8.      JR     C, $0E73
0E72  12                 .       LD     (DE), A
.
0E73  FD 21 10 00        .!..    LD     IY, $0010
0E77  D1                 .       POP    DE
0E78  FD 19              ..      ADD    IY, DE	
0E7A  3A 85 E2           :..     LD     A, ($E285)
0E7D  06 10              ..      LD     B, $10
0E7F  B7                 .       OR     A
0E80  28 02              (.      JR     Z, $0E84
0E82  CB 38              .8      SRL    B
.
0E84  C5                 .       PUSH   BC
0E85  FD 4E 00           .N.     LD     C, (IY+$00)
0E88  FD A6 01           ...     AND    (IY+$01)
0E8B  47                 G       LD     B, A
0E8C  B1                 .       OR     C
0E8D  C4 0E EE           ...     CALL   NZ, $EE0E
0E90  3A 85 E2           :..     LD     A, ($E285)
0E93  FD 23              .#      INC    IY
0E95  B7                 .       OR     A
0E96  28 02              (.      JR     Z, $0E9A
0E98  FD 23              .#      INC    IY
.
0E9A  C1                 .       POP    BC
0E9B  10 E7              ..      DJNZ   $0E84
0E9D  0E 01              ..      LD     C, $01
0E9F  CD 05 ED           ...     CALL   $ED05
0EA2  CD 16 EC           ...     CALL   $EC16
0EA5  B7                 .       OR     A
0EA6  F2 39 E8           .9.     JP     P $E839
0EA9  F1                 .       POP    AF
0EAA  06 00              ..      LD     B, $00
0EAC  C9                 .       RET
0EAD  CD 64 EF           .d.     CALL   $EF64
0EB0  3A 72 E2           :r.     LD     A, ($E272)
0EB3  FE 80              ..      CP     $80
0EB5  20 0B               .      JR     NZ $0EC2
0EB7  CD E5 EE           ...     CALL   $EEE5
0EBA  06 00              ..      LD     B, $00
0EBC  C0                 .       RET    NZ
0EBD  32 72 E2           2r.     LD     ($E272), A
0EC0  18 03              ..      JR     $0EC5
.
0EC2  CD 3A EF           .:.     CALL   $EF3A
.
0EC5  21 61 E2           !a.     LD     HL, $E261
0EC8  3A 72 E2           :r.     LD     A, ($E272)
0ECB  BE                 .       CP     (HL)
0ECC  3E 01              >.      LD     A, $01
0ECE  06 00              ..      LD     B, $00
0ED0  D0                 .       RET    NC
0ED1  CD 7F EE           ..     CALL   $EE7F
0ED4  ED 44              .D      NEG
0ED6  06 00              ..      LD     B, $00
0ED8  C0                 .       RET    NZ
0ED9  EB                 .       EX     DE, HL
0EDA  CD E7 EC           ...     CALL   $ECE7
0EDD  21 72 E2           !r.     LD     HL, $E272
0EE0  34                 4       INC    (HL)
0EE1  C3 72 EF           .r.     JP     $EF72
0EE4  CD 64 EF           .d.     CALL   $EF64
0EE7  CD 80 EF           ...     CALL   $EF80
0EEA  3A 72 E2           :r.     LD     A, ($E272)
0EED  FE 80              ..      CP     $80
0EEF  20 1C               .      JR     NZ $0F0D
0EF1  CD E5 EE           ...     CALL   $EEE5
0EF4  28 11              (.      JR     Z, $0F07
0EF6  FE 03              ..      CP     $03
0EF8  06 00              ..      LD     B, $00
0EFA  C8                 .       RET    Z
0EFB  11 52 E2           .R.     LD     DE, $E252
0EFE  CD 49 E9           .I.     CALL   $E949
0F01  B7                 .       OR     A
0F02  3E 05              >.      LD     A, $05
0F04  06 00              ..      LD     B, $00
0F06  F8                 .       RET    M
.
0F07  AF                 .       XOR    A
0F08  32 72 E2           2r.     LD     ($E272), A
0F0B  18 03              ..      JR     $0F10
.
0F0D  CD 3A EF           .:.     CALL   $EF3A
.
0F10  AF                 .       XOR    A
0F11  32 2A E2           2*.     LD     ($E22A), A
0F14  CD 7F EE           ..     CALL   $EE7F
0F17  F2 16 E9           ...     JP     P $E916
0F1A  E5                 .       PUSH   HL
0F1B  CD 31 EE           .1.     CALL   $EE31
0F1E  3E 02              >.      LD     A, $02
0F20  DD E1              ..      POP    IX
0F22  06 00              ..      LD     B, $00
0F24  F8                 .       RET    M
0F25  DD 75 00           .u.     LD     (IX+$00), L
0F28  3A 85 E2           :..     LD     A, ($E285)
0F2B  B7                 .       OR     A
0F2C  28 03              (.      JR     Z, $0F31
0F2E  DD 74 01           .t.     LD     (IX+$01), H
.
0F31  EB                 .       EX     DE, HL
0F32  CD B8 EE           ...     CALL   $EEB8
0F35  3E 02              >.      LD     A, $02
0F37  32 2A E2           2*.     LD     ($E22A), A
0F3A  E5                 .       PUSH   HL
0F3B  ED 4B 1D E2        .K..    LD     BC, ($E21D)
0F3F  CD 24 F0           .$.     CALL   $F024
0F42  D1                 .       POP    DE
0F43  3A 2A E2           :*.     LD     A, ($E22A)
0F46  4F                 O       LD     C, A
0F47  CD FF EC           ...     CALL   $ECFF
0F4A  21 72 E2           !r.     LD     HL, $E272
0F4D  34                 4       INC    (HL)
0F4E  3A 61 E2           :a.     LD     A, ($E261)
0F51  4F                 O       LD     C, A
0F52  7E                 ~       LD     A, (HL)
0F53  B9                 .       CP     C
0F54  38 0A              8.      JR     C, $0F60
0F56  32 61 E2           2a.     LD     ($E261), A
0F59  E5                 .       PUSH   HL
0F5A  21 60 E2           !`.     LD     HL, $E260
0F5D  CB BE              ..      RES    7, (HL)
0F5F  E1                 .       POP    HL
.
0F60  AF                 .       XOR    A
0F61  C3 72 EF           .r.     JP     $EF72
0F64  21 0D 00           !..     LD     HL, $000D
0F67  19                 .       ADD    HL, DE
0F68  36 00              6.      LD     (HL), $00
0F6A  23                 #       INC    HL
0F6B  36 00              6.      LD     (HL), $00
0F6D  ED 53 2B E2        .S+.    LD     ($E22B), DE
0F71  21 2E E2           !..     LD     HL, $E22E
0F74  EB                 .       EX     DE, HL
0F75  01 24 00           .$.     LD     BC, $0024
0F78  ED B0              ..      LDIR
0F7A  3A 1F E2           :..     LD     A, ($E21F)
0F7D  32 2D E2           2-.     LD     ($E22D), A
0F80  3A 2E E2           :..     LD     A, ($E22E)
0F83  3D                 =       DEC    A
0F84  FA 66 E9           .f.     JP     M $E966
0F87  32 1F E2           2..     LD     ($E21F), A
0F8A  21 52 E2           !R.     LD     HL, $E252
0F8D  11 53 E2           .S.     LD     DE, $E253
0F90  36 3F              6?      LD     (HL), $3F
0F92  01 0E 00           ...     LD     BC, $000E
0F95  ED B0              ..      LDIR
0F97  CD 0B EC           ...     CALL   $EC0B
.
0F9A  B7                 .       OR     A
0F9B  FA C7 E9           ...     JP     M $E9C7
0F9E  F5                 .       PUSH   AF
0F9F  CD 2F EF           ./.     CALL   $EF2F
0FA2  3E E5              >.      LD     A, $E5
0FA4  BE                 .       CP     (HL)
0FA5  28 06              (.      JR     Z, $0FAD
0FA7  F1                 .       POP    AF
0FA8  CD 16 EC           ...     CALL   $EC16
0FAB  18 ED              ..      JR     $0F9A
.
0FAD  AF                 .       XOR    A
0FAE  32 3B E2           2;.     LD     ($E23B), A
0FB1  3A 76 E2           :v.     LD     A, ($E276)
0FB4  77                 w       LD     (HL), A
0FB5  11 2F E2           ./.     LD     DE, $E22F
0FB8  23                 #       INC    HL
0FB9  01 0E 00           ...     LD     BC, $000E
0FBC  EB                 .       EX     DE, HL
0FBD  ED B0              ..      LDIR
0FBF  01 11 00           ...     LD     BC, $0011
0FC2  36 00              6.      LD     (HL), $00
0FC4  ED A0              ..      LDI
0FC6  EA 9E E9           ...     JP     PE $E99E
0FC9  CD 52 ED           .R.     CALL   $ED52
0FCC  38 01              8.      JR     C, $0FCF
0FCE  12                 .       LD     (DE), A
.
0FCF  0E 01              ..      LD     C, $01
0FD1  CD 05 ED           ...     CALL   $ED05
0FD4  21 2E E2           !..     LD     HL, $E22E
0FD7  ED 5B 2B E2        .[+.    LD     DE, ($E22B)
0FDB  01 24 00           .$.     LD     BC, $0024
0FDE  ED B0              ..      LDIR
0FE0  DD 2A 2B E2        .*+.    LD     IX, ($E22B)
0FE4  DD CB              ..      ****BUG****			DD CB 05 FE   SET 7,(IX+05)
0FE6  0E FE              ..      LD     C, $FE
0FE8  F1                 .       POP    AF
0FE9  18 0E              ..      JR     $0FF9
0FEB  3E FF              >.      LD     A, $FF
0FED  21 2E E2           !..     LD     HL, $E22E
0FF0  ED 5B 2B E2        .[+.    LD     DE, ($E22B)
0FF4  01 24 00           .$.     LD     BC, $0024
0FF7  ED B0              ..      LDIR
.
0FF9  47                 G       LD     B, A
0FFA  3A 2D E2           :-.     LD     A, ($E22D)
0FFD  32 1F E2           2..     LD     ($E21F), A
1000  78                 x       LD     A, B
1001  06 00              ..      LD     B, $00
1003  C9                 .       RET
1004  CD 64 EF           .d.     CALL   $EF64
1007  01 11 00           ...     LD     BC, $0011
100A  ED 43 80 E2        .C..    LD     ($E280), BC
100E  3E 3F              >?      LD     A, $3F
1010  32 5E E2           2^.     LD     ($E25E), A
1013  32 60 E2           2`.     LD     ($E260), A
1016  AF                 .       XOR    A
1017  32 5F E2           2_.     LD     ($E25F), A
101A  CD 0B EC           ...     CALL   $EC0B
101D  B7                 .       OR     A
101E  06 00              ..      LD     B, $00
1020  F8                 .       RET    M
1021  F5                 .       PUSH   AF
1022  CD 2F EF           ./.     CALL   $EF2F
1025  3A 80 E2           :..     LD     A, ($E280)
1028  3D                 =       DEC    A
1029  28 0A              (.      JR     Z, $1035
102B  E5                 .       PUSH   HL
102C  DD E1              ..      POP    IX
102E  DD CB              ..      ****BUG****			DD CB 05 FE   SET 7,(IX+05)
1030  09                 .       ADD    HL, BC
1031  7E                 ~       LD     A, (HL)
1032  C2 A3 EF           ...     JP     NZ $EFA3
.
1035  11 52 E2           .R.     LD     DE, $E252
1038  ED 4B 80 E2        .K..    LD     BC, ($E280)
103C  EB                 .       EX     DE, HL
103D  09                 .       ADD    HL, BC
103E  13                 .       INC    DE
103F  01 0B 00           ...     LD     BC, $000B
1042  ED B0              ..      LDIR
1044  CD 52 ED           .R.     CALL   $ED52
1047  38 01              8.      JR     C, $104A
1049  12                 .       LD     (DE), A
.
104A  0E 01              ..      LD     C, $01
104C  CD 05 ED           ...     CALL   $ED05
104F  CD 16 EC           ...     CALL   $EC16
1052  B7                 .       OR     A
1053  F2 FE E9           ...     JP     P $E9FE
1056  F1                 .       POP    AF
1057  06 00              ..      LD     B, $00
1059  C9                 .       RET
105A  2A 19 E2           *..     LD     HL, ($E219)
105D  7D                 }       LD     A, L
105E  44                 D       LD     B, H
105F  C9                 .       RET
1060  3A 1F E2           :..     LD     A, ($E21F)
1063  C9                 .       RET
1064  ED 53 1D E2        .S..    LD     ($E21D), DE
1068  C9                 .       RET
1069  3A 1F E2           :..     LD     A, ($E21F)
106C  5F                 _       LD     E, A
106D  CD FC E5           ...     CALL   $E5FC
1070  2A 91 E2           *..     LD     HL, ($E291)
1073  7D                 }       LD     A, L
1074  44                 D       LD     B, H
1075  C9                 .       RET
1076  2A 1B E2           *..     LD     HL, ($E21B)
1079  3A 1F E2           :..     LD     A, ($E21F)
107C  CD 9F ED           ...     CALL   $ED9F
107F  22 1B E2           "..     LD     ($E21B), HL
1082  C9                 .       RET
1083  2A 1B E2           *..     LD     HL, ($E21B)
1086  7D                 }       LD     A, L
1087  44                 D       LD     B, H
1088  C9                 .       RET
1089  CD 64 EF           .d.     CALL   $EF64
108C  01 01 00           ...     LD     BC, $0001
108F  C3 E6 E9           ...     JP     $E9E6
1092  3A 1F E2           :..     LD     A, ($E21F)
1095  5F                 _       LD     E, A
1096  CD FC E5           ...     CALL   $E5FC
1099  2A 8D E2           *..     LD     HL, ($E28D)
109C  7D                 }       LD     A, L
109D  44                 D       LD     B, H
109E  C9                 .       RET
109F  7B                 {       LD     A, E
10A0  E6 1F              ..      AND    $1F
10A2  21 76 E2           !v.     LD     HL, $E276
10A5  1C                 .       INC    E
10A6  20 01               .      JR     NZ $10A9
10A8  7E                 ~       LD     A, (HL)
.
10A9  77                 w       LD     (HL), A
10AA  C9                 .       RET
10AB  CD 64 EF           .d.     CALL   $EF64
10AE  CD 3A EF           .:.     CALL   $EF3A
10B1  CD 48 EF           .H.     CALL   $EF48
10B4  CD 06 EF           ...     CALL   $EF06
10B7  F5                 .       PUSH   AF
10B8  FE 04              ..      CP     $04
10BA  20 10               .      JR     NZ $10CC
10BC  11 52 E2           .R.     LD     DE, $E252
10BF  CD 49 E9           .I.     CALL   $E949
10C2  B7                 .       OR     A
10C3  F2 A8 EA           ...     JP     P $EAA8
10C6  F1                 .       POP    AF
10C7  3E 05              >.      LD     A, $05
10C9  06 00              ..      LD     B, $00
10CB  C9                 .       RET
.
10CC  3A 79 E2           :y.     LD     A, ($E279)
10CF  32 72 E2           2r.     LD     ($E272), A
10D2  CD 72 EF           .r.     CALL   $EF72
10D5  F1                 .       POP    AF
10D6  C0                 .       RET    NZ
10D7  CD 7F EE           ..     CALL   $EE7F
10DA  3E 01              >.      LD     A, $01
10DC  06 00              ..      LD     B, $00
10DE  C0                 .       RET    NZ
10DF  3A 61 E2           :a.     LD     A, ($E261)
10E2  47                 G       LD     B, A
10E3  3A 72 E2           :r.     LD     A, ($E272)
10E6  B8                 .       CP     B
10E7  3E 01              >.      LD     A, $01
10E9  06 00              ..      LD     B, $00
10EB  D0                 .       RET    NC
10EC  EB                 .       EX     DE, HL
10ED  CD E7 EC           ...     CALL   $ECE7
10F0  CD 72 EF           .r.     CALL   $EF72
10F3  AF                 .       XOR    A
10F4  C9                 .       RET
10F5  3E 02              >.      LD     A, $02
10F7  18 01              ..      JR     $10FA
10F9  AF                 .       XOR    A
.
10FA  32 82 E2           2..     LD     ($E282), A
10FD  CD 64 EF           .d.     CALL   $EF64
1100  CD 80 EF           ...     CALL   $EF80
1103  CD 3A EF           .:.     CALL   $EF3A
1106  CD 48 EF           .H.     CALL   $EF48
1109  CD 06 EF           ...     CALL   $EF06
110C  28 11              (.      JR     Z, $111F
110E  FE 03              ..      CP     $03
1110  06 00              ..      LD     B, $00
1112  C8                 .       RET    Z
1113  11 52 E2           .R.     LD     DE, $E252
1116  CD 49 E9           .I.     CALL   $E949
1119  B7                 .       OR     A
111A  3E 05              >.      LD     A, $05
111C  06 00              ..      LD     B, $00
111E  F8                 .       RET    M
.
111F  3A 61 E2           :a.     LD     A, ($E261)
1122  4F                 O       LD     C, A
1123  3A 79 E2           :y.     LD     A, ($E279)
1126  32 72 E2           2r.     LD     ($E272), A
1129  3C                 <       INC    A
112A  B9                 .       CP     C
112B  38 08              8.      JR     C, $1135
112D  32 61 E2           2a.     LD     ($E261), A
1130  21 60 E2           !`.     LD     HL, $E260
1133  CB BE              ..      RES    7, (HL)
.
1135  CD 7F EE           ..     CALL   $EE7F
1138  28 54              (T      JR     Z, $118E
113A  E5                 .       PUSH   HL
113B  CD 31 EE           .1.     CALL   $EE31
113E  3E 06              >.      LD     A, $06
1140  D1                 .       POP    DE
1141  06 00              ..      LD     B, $00
1143  F8                 .       RET    M
1144  EB                 .       EX     DE, HL
1145  73                 s       LD     (HL), E
1146  3A 85 E2           :..     LD     A, ($E285)
1149  B7                 .       OR     A
114A  28 02              (.      JR     Z, $114E
114C  23                 #       INC    HL
114D  72                 r       LD     (HL), D
.
114E  CD B8 EE           ...     CALL   $EEB8
1151  C5                 .       PUSH   BC
1152  3A 82 E2           :..     LD     A, ($E282)
1155  B7                 .       OR     A
1156  20 2E               .      JR     NZ $1186
1158  E5                 .       PUSH   HL
1159  D5                 .       PUSH   DE
115A  2A 8B E2           *..     LD     HL, ($E28B)
115D  E5                 .       PUSH   HL
115E  06 80              ..      LD     B, $80
.
1160  36 00              6.      LD     (HL), $00
1162  23                 #       INC    HL
1163  10 FB              ..      DJNZ   $1160
1165  C1                 .       POP    BC
1166  CD 24 F0           .$.     CALL   $F024
1169  3A 95 E2           :..     LD     A, ($E295)
116C  47                 G       LD     B, A
116D  AF                 .       XOR    A
116E  3C                 <       INC    A
.
116F  17                 .       RLA
1170  10 FD              ..      DJNZ   $116F
1172  D1                 .       POP    DE
1173  0E 02              ..      LD     C, $02
.
1175  D5                 .       PUSH   DE
1176  F5                 .       PUSH   AF
1177  CD FF EC           ...     CALL   $ECFF
117A  F1                 .       POP    AF
117B  D1                 .       POP    DE
117C  0E 00              ..      LD     C, $00
117E  13                 .       INC    DE
117F  3D                 =       DEC    A
1180  20 F3               .      JR     NZ $1175
1182  CD D8 EC           ...     CALL   $ECD8
1185  E1                 .       POP    HL
.
1186  C1                 .       POP    BC
1187  78                 x       LD     A, B
1188  B1                 .       OR     C
1189  3E 02              >.      LD     A, $02
118B  28 01              (.      JR     Z, $118E
118D  AF                 .       XOR    A
.
118E  F5                 .       PUSH   AF
118F  E5                 .       PUSH   HL
1190  ED 4B 1D E2        .K..    LD     BC, ($E21D)
1194  CD 24 F0           .$.     CALL   $F024
1197  D1                 .       POP    DE
1198  F1                 .       POP    AF
1199  4F                 O       LD     C, A
119A  CD FF EC           ...     CALL   $ECFF
119D  CD 72 EF           .r.     CALL   $EF72
11A0  AF                 .       XOR    A
11A1  06 00              ..      LD     B, $00
11A3  C9                 .       RET
11A4  CD 64 EF           .d.     CALL   $EF64
11A7  3E 3F              >?      LD     A, $3F
11A9  32 5E E2           2^.     LD     ($E25E), A
11AC  32 60 E2           2`.     LD     ($E260), A
11AF  21 00 00           !..     LD     HL, $0000
11B2  22 7A E2           "z.     LD     ($E27A), HL
11B5  32 7C E2           2|.     LD     ($E27C), A
11B8  CD 0B EC           ...     CALL   $EC0B
11BB  B7                 .       OR     A
11BC  06 00              ..      LD     B, $00
11BE  F8                 .       RET    M
11BF  CD 2F EF           ./.     CALL   $EF2F
11C2  E5                 .       PUSH   HL
11C3  DD E1              ..      POP    IX
11C5  CD D3 EE           ...     CALL   $EED3
11C8  ED 5B 7A E2        .[z.    LD     DE, ($E27A)
11CC  AF                 .       XOR    A
11CD  ED 52              .R      SBC    HL, DE
11CF  38 0A              8.      JR     C, $11DB
11D1  19                 .       ADD    HL, DE
11D2  22 7A E2           "z.     LD     ($E27A), HL
11D5  DD 7E 0F           .~.     LD     A, (IX+$0F)
11D8  32 7C E2           2|.     LD     ($E27C), A
.
11DB  CD 16 EC           ...     CALL   $EC16
11DE  B7                 .       OR     A
11DF  F2 9B EB           ...     JP     P $EB9B
11E2  2A 7A E2           *z.     LD     HL, ($E27A)
.
11E5  7D                 }       LD     A, L
11E6  2E 00              ..      LD     L, $00
11E8  45                 E       LD     B, L
11E9  CB 3C              .<      SRL    H
11EB  1F                 .       RRA
11EC  67                 g       LD     H, A
11ED  CB 1D              ..      RR     L
11EF  3A 7C E2           :|.     LD     A, ($E27C)
11F2  4F                 O       LD     C, A
11F3  09                 .       ADD    HL, BC
11F4  CB 10              ..      RL     B
11F6  DD 2A 24 E2        .*$.    LD     IX, ($E224)
11FA  DD 75 21           .u!     LD     (IX+$21), L
11FD  DD 74 22           .t"     LD     (IX+$22), H
1200  DD 70 23           .p#     LD     (IX+$23), B
1203  AF                 .       XOR    A
1204  47                 G       LD     B, A
1205  C9                 .       RET
1206  CD 64 EF           .d.     CALL   $EF64
1209  DD 21 52 E2        .!R.    LD     IX, $E252
120D  CD D3 EE           ...     CALL   $EED3
1210  3A 72 E2           :r.     LD     A, ($E272)
1213  32 7C E2           2|.     LD     ($E27C), A
1216  18 CD              ..      JR     $11E5
1218  21 FF FF           !..     LD     HL, $FFFF
121B  AF                 .       XOR    A
121C  ED 52              .R      SBC    HL, DE
121E  11 19 E2           ...     LD     DE, $E219
1221  CD 03 EC           ...     CALL   $EC03
1224  11 1B E2           ...     LD     DE, $E21B
1227  1A                 .       LD     A, (DE)
1228  A5                 .       AND    L
1229  12                 .       LD     (DE), A
122A  13                 .       INC    DE
122B  1A                 .       LD     A, (DE)
122C  A4                 .       AND    H
122D  12                 .       LD     (DE), A
122E  C9                 .       RET
122F  AF                 .       XOR    A
1230  32 7E E2           2~.     LD     ($E27E), A
1233  3D                 =       DEC    A
1234  32 7D E2           2}.     LD     ($E27D), A
1237  CD 18 F0           ...     CALL   $F018
123A  3A 52 E2           :R.     LD     A, ($E252)
123D  FE 3F              .?      CP     $3F
123F  20 06               .      JR     NZ $1247
1241  3A 1F E2           :..     LD     A, ($E21F)
1244  C3 41 EC           .A.     JP     $EC41
.
1247  3D                 =       DEC    A
1248  F2 2A EC           .*.     JP     P $EC2A
124B  3A 1F E2           :..     LD     A, ($E21F)
124E  CD 41 EC           .A.     CALL   $EC41
1251  B7                 .       OR     A
1252  F8                 .       RET    M
1253  F5                 .       PUSH   AF
1254  CD 2F EF           ./.     CALL   $EF2F
1257  3A 76 E2           :v.     LD     A, ($E276)
125A  BE                 .       CP     (HL)
125B  20 02               .      JR     NZ $125F
125D  F1                 .       POP    AF
125E  C9                 .       RET
.
125F  F1                 .       POP    AF
1260  3A 52 E2           :R.     LD     A, ($E252)
1263  18 E2              ..      JR     $1247
1265  5F                 _       LD     E, A
1266  CD FC E5           ...     CALL   $E5FC
1269  3A 52 E2           :R.     LD     A, ($E252)
126C  FE 3F              .?      CP     $3F
126E  3A 86 E2           :..     LD     A, ($E286)
1271  20 03               .      JR     NZ $1276
1273  3A 87 E2           :..     LD     A, ($E287)
.
1276  32 7F E2           2.     LD     ($E27F), A
1279  3A 7E E2           :~.     LD     A, ($E27E)
127C  32 23 E2           2#.     LD     ($E223), A
127F  3A 7D E2           :}.     LD     A, ($E27D)
1282  FE 03              ..      CP     $03
1284  28 0E              (.      JR     Z, $1294
1286  CD D8 EC           ...     CALL   $ECD8
1289  CD 71 ED           .q.     CALL   $ED71
.
128C  3A 7D E2           :}.     LD     A, ($E27D)
128F  3C                 <       INC    A
1290  FE 04              ..      CP     $04
1292  20 17               .      JR     NZ $12AB
.
1294  21 7E E2           !~.     LD     HL, $E27E
1297  34                 4       INC    (HL)
1298  28 59              (Y      JR     Z, $12F3
129A  3A 7F E2           :.     LD     A, ($E27F)
129D  BE                 .       CP     (HL)
129E  38 53              8S      JR     C, $12F3
12A0  7E                 ~       LD     A, (HL)
12A1  32 23 E2           2#.     LD     ($E223), A
12A4  CD D8 EC           ...     CALL   $ECD8
12A7  CD 71 ED           .q.     CALL   $ED71
12AA  AF                 .       XOR    A
.
12AB  32 7D E2           2}.     LD     ($E27D), A
12AE  CD 2F EF           ./.     CALL   $EF2F
12B1  06 0B              ..      LD     B, $0B
12B3  11 52 E2           .R.     LD     DE, $E252
.
12B6  13                 .       INC    DE
12B7  23                 #       INC    HL
12B8  1A                 .       LD     A, (DE)
12B9  E6 7F              .      AND    $7F
12BB  FE 3F              .?      CP     $3F
12BD  28 06              (.      JR     Z, $12C5
12BF  4E                 N       LD     C, (HL)
12C0  CB B9              ..      RES    7, C
12C2  B9                 .       CP     C
12C3  20 C7               .      JR     NZ $128C
.
12C5  10 EF              ..      DJNZ   $12B6
12C7  13                 .       INC    DE
12C8  23                 #       INC    HL
12C9  1A                 .       LD     A, (DE)
12CA  FE 3F              .?      CP     $3F
12CC  28 09              (.      JR     Z, $12D7
12CE  AE                 .       XOR    (HL)
12CF  47                 G       LD     B, A
12D0  3A 97 E2           :..     LD     A, ($E297)
12D3  2F                 /       CPL
12D4  A0                 .       AND    B
12D5  20 B5               .      JR     NZ $128C
.
12D7  23                 #       INC    HL
12D8  23                 #       INC    HL
12D9  13                 .       INC    DE
12DA  13                 .       INC    DE
12DB  1A                 .       LD     A, (DE)
12DC  E6 7F              .      AND    $7F
12DE  FE 3F              .?      CP     $3F
12E0  28 03              (.      JR     Z, $12E5
12E2  BE                 .       CP     (HL)
12E3  20 A7               .      JR     NZ $128C
.
12E5  21 86 E2           !..     LD     HL, $E286
12E8  3A 7E E2           :~.     LD     A, ($E27E)
12EB  BE                 .       CP     (HL)
12EC  38 01              8.      JR     C, $12EF
12EE  77                 w       LD     (HL), A
.
12EF  3A 7D E2           :}.     LD     A, ($E27D)
12F2  C9                 .       RET
.
12F3  AF                 .       XOR    A
12F4  32 7E E2           2~.     LD     ($E27E), A
12F7  3D                 =       DEC    A
12F8  32 7D E2           2}.     LD     ($E27D), A
12FB  C9                 .       RET
12FC  ED 4B 8B E2        .K..    LD     BC, ($E28B)
1300  CD 24 F0           .$.     CALL   $F024
1303  3A 23 E2           :#.     LD     A, ($E223)
1306  5F                 _       LD     E, A
1307  16 00              ..      LD     D, $00
1309  18 0B              ..      JR     $1316
130B  D5                 .       PUSH   DE
130C  ED 4B 1D E2        .K..    LD     BC, ($E21D)
1310  CD 24 F0           .$.     CALL   $F024
1313  D1                 .       POP    DE
1314  0E 00              ..      LD     C, $00
.
1316  CD 1D ED           ...     CALL   $ED1D
.
1319  CD 27 F0           .'.     CALL   $F027
131C  B7                 .       OR     A
131D  C4 90 EF           ...     CALL   NZ, $EF90
1320  20 F7               .      JR     NZ $1319
1322  C9                 .       RET
1323  C5                 .       PUSH   BC
1324  CD 1D ED           ...     CALL   $ED1D
1327  18 01              ..      JR     $132A
1329  C5                 .       PUSH   BC
.
132A  3A 20 E2           : .     LD     A, ($E220)
132D  2A 1B E2           *..     LD     HL, ($E21B)
1330  CD 9F ED           ...     CALL   $ED9F
1333  C1                 .       POP    BC
1334  DA 9C EF           ...     JP     C $EF9C
.
1337  CD 2A F0           .*.     CALL   $F02A
133A  B7                 .       OR     A
133B  C4 95 EF           ...     CALL   NZ, $EF95
133E  20 F7               .      JR     NZ $1337
1340  C9                 .       RET
1341  4B                 K       LD     C, E
1342  7A                 z       LD     A, D
1343  ED 5B 93 E2        .[..    LD     DE, ($E293)
1347  21 00 00           !..     LD     HL, $0000
134A  06 10              ..      LD     B, $10
.
134C  CB 11              ..      RL     C
134E  17                 .       RLA
134F  ED 6A              .j      ADC    HL, HL
1351  ED 52              .R      SBC    HL, DE
1353  30 01              0.      JR     NC $1356
1355  19                 .       ADD    HL, DE
.
1356  3F                 ?       CCF
1357  10 F3              ..      DJNZ   $134C
1359  CB 11              ..      RL     C
135B  17                 .       RLA
135C  47                 G       LD     B, A
135D  C5                 .       PUSH   BC
135E  4D                 M       LD     C, L
135F  44                 D       LD     B, H
1360  ED 5B 83 E2        .[..    LD     DE, ($E283)
1364  CD 30 F0           .0.     CALL   $F030
1367  4D                 M       LD     C, L
1368  44                 D       LD     B, H
1369  CD 21 F0           .!.     CALL   $F021
136C  C1                 .       POP    BC
136D  2A A0 E2           *..     LD     HL, ($E2A0)
1370  09                 .       ADD    HL, BC
1371  4D                 M       LD     C, L
1372  44                 D       LD     B, H
1373  C3 1E F0           ...     JP     $F01E
1376  ED 5B 9E E2        .[..    LD     DE, ($E29E)
137A  7B                 {       LD     A, E
137B  B2                 .       OR     D
137C  37                 7       SCF
137D  C8                 .       RET    Z
137E  3A 23 E2           :#.     LD     A, ($E223)
1381  2A 8F E2           *..     LD     HL, ($E28F)
1384  5F                 _       LD     E, A
1385  16 00              ..      LD     D, $00
1387  19                 .       ADD    HL, DE
1388  EB                 .       EX     DE, HL
1389  2A 8B E2           *..     LD     HL, ($E28B)
138C  AF                 .       XOR    A
138D  06 80              ..      LD     B, $80
.
138F  86                 .       ADD    A, (HL)
1390  23                 #       INC    HL
1391  10 FC              ..      DJNZ   $138F
1393  A7                 .       AND    A
1394  C9                 .       RET
1395  CD 52 ED           .R.     CALL   $ED52
1398  D8                 .       RET    C
1399  EB                 .       EX     DE, HL
139A  BE                 .       CP     (HL)
139B  C8                 .       RET    Z
139C  2A 8D E2           *..     LD     HL, ($E28D)
139F  11 93 E2           ...     LD     DE, $E293
13A2  01 0F 00           ...     LD     BC, $000F
13A5  ED B0              ..      LDIR
13A7  3A 23 E2           :#.     LD     A, ($E223)
13AA  CD D8 EC           ...     CALL   $ECD8
13AD  3A 87 E2           :..     LD     A, ($E287)
13B0  32 86 E2           2..     LD     ($E286), A
13B3  32 7F E2           2.     LD     ($E27F), A
13B6  2A 1B E2           *..     LD     HL, ($E21B)
13B9  3A 20 E2           : .     LD     A, ($E220)
13BC  CD 9F ED           ...     CALL   $ED9F
13BF  22 1B E2           "..     LD     ($E21B), HL
13C2  C9                 .       RET
13C3  3C                 <       INC    A
13C4  47                 G       LD     B, A
13C5  A7                 .       AND    A
.
13C6  CB 1C              ..      RR     H
13C8  CB 1D              ..      RR     L
13CA  10 FA              ..      DJNZ   $13C6
13CC  F5                 .       PUSH   AF
13CD  47                 G       LD     B, A
13CE  37                 7       SCF
.
13CF  CB 15              ..      RL     L
13D1  CB 14              ..      RL     H
13D3  10 FA              ..      DJNZ   $13CF
13D5  F1                 .       POP    AF
13D6  C9                 .       RET
13D7  FD 2A 8B E2        .*..    LD     IY, ($E28B)
13DB  3A 85 E2           :..     LD     A, ($E285)
13DE  06 10              ..      LD     B, $10
13E0  B7                 .       OR     A
13E1  28 02              (.      JR     Z, $13E5
13E3  CB 38              .8      SRL    B
.
13E5  0E 04              ..      LD     C, $04
.
13E7  C5                 .       PUSH   BC
13E8  FD 7E 0F           .~.     LD     A, (IY+$0F)
13EB  FE E5              ..      CP     $E5
13ED  20 03               .      JR     NZ $13F2
13EF  37                 7       SCF
13F0  C1                 .       POP    BC
13F1  C9                 .       RET
.
13F2  FD 7E 00           .~.     LD     A, (IY+$00)
13F5  FE E5              ..      CP     $E5
13F7  28 29              ()      JR     Z, $1422
13F9  3A 23 E2           :#.     LD     A, ($E223)
13FC  32 86 E2           2..     LD     ($E286), A
13FF  11 10 00           ...     LD     DE, $0010
1402  FD 19              ..      ADD    IY, DE	
.
1404  C5                 .       PUSH   BC
1405  FD 4E 00           .N.     LD     C, (IY+$00)
1408  3A 85 E2           :..     LD     A, ($E285)
140B  FD A6 01           ...     AND    (IY+$01)
140E  47                 G       LD     B, A
140F  B1                 .       OR     C
1410  C4 08 EE           ...     CALL   NZ, $EE08
1413  FD 23              .#      INC    IY
1415  3A 85 E2           :..     LD     A, ($E285)
1418  B7                 .       OR     A
1419  28 02              (.      JR     Z, $141D
141B  FD 23              .#      INC    IY
.
141D  C1                 .       POP    BC
141E  10 E4              ..      DJNZ   $1404
1420  18 05              ..      JR     $1427
.
1422  11 20 00           . .     LD     DE, $0020
1425  FD 19              ..      ADD    IY, DE	
.
1427  C1                 .       POP    BC
1428  0D                 .       DEC    C
1429  20 BC               .      JR     NZ $13E7
142B  C9                 .       RET
142C  CD 15 EE           ...     CALL   $EE15
142F  B6                 .       OR     (HL)
1430  77                 w       LD     (HL), A
1431  C9                 .       RET
1432  CD 15 EE           ...     CALL   $EE15
1435  2F                 /       CPL
1436  A6                 .       AND    (HL)
1437  77                 w       LD     (HL), A
1438  C9                 .       RET
1439  59                 Y       LD     E, C
143A  CB 38              .8      SRL    B
143C  CB 19              ..      RR     C
143E  CB 38              .8      SRL    B
1440  CB 19              ..      RR     C
1442  CB 38              .8      SRL    B
1444  CB 19              ..      RR     C
1446  2A 91 E2           *..     LD     HL, ($E291)
1449  09                 .       ADD    HL, BC
144A  7B                 {       LD     A, E
144B  E6 07              ..      AND    $07
144D  47                 G       LD     B, A
144E  04                 .       INC    B
144F  3E 01              >.      LD     A, $01
.
1451  0F                 .       RCCA
1452  10 FD              ..      DJNZ   $1451
1454  C9                 .       RET
1455  2A 98 E2           *..     LD     HL, ($E298)
1458  11 07 00           ...     LD     DE, $0007
145B  19                 .       ADD    HL, DE
145C  06 03              ..      LD     B, $03
.
145E  CB 3C              .<      SRL    H
1460  CB 1D              ..      RR     L
1462  10 FA              ..      DJNZ   $145E
1464  4D                 M       LD     C, L
1465  44                 D       LD     B, H
1466  2A 91 E2           *..     LD     HL, ($E291)
1469  3E FF              >.      LD     A, $FF
146B  ED A1              ..      CPI
146D  20 05               .      JR     NZ $1474
146F  EA 47 EE           .G.     JP     PE $EE47
1472  B7                 .       OR     A
1473  C9                 .       RET
.
1474  EB                 .       EX     DE, HL
1475  21 60 E2           !`.     LD     HL, $E260
1478  CB BE              ..      RES    7, (HL)
147A  1B                 .       DEC    DE
147B  1A                 .       LD     A, (DE)
147C  06 08              ..      LD     B, $08
147E  CB 27              .'      SLA    A
.
1480  30 04              0.      JR     NC $1486
1482  CB 17              ..      RL     A
1484  10 FA              ..      DJNZ   $1480
.
1486  37                 7       SCF
1487  48                 H       LD     C, B
.
1488  CB 17              ..      RL     A
148A  10 FC              ..      DJNZ   $1488
148C  12                 .       LD     (DE), A
148D  3E 08              >.      LD     A, $08
148F  91                 .       SUB    C
1490  4F                 O       LD     C, A
1491  2A 91 E2           *..     LD     HL, ($E291)
1494  AF                 .       XOR    A
1495  EB                 .       EX     DE, HL
1496  ED 52              .R      SBC    HL, DE
1498  06 03              ..      LD     B, $03
.
149A  CB 25              .%      SLA    L
149C  CB 14              ..      RL     H
149E  10 FA              ..      DJNZ   $149A
14A0  09                 .       ADD    HL, BC
14A1  B7                 .       OR     A
14A2  C9                 .       RET
14A3  3A 5E E2           :^.     LD     A, ($E25E)
14A6  47                 G       LD     B, A
14A7  3A 97 E2           :..     LD     A, ($E297)
14AA  A0                 .       AND    B
14AB  4F                 O       LD     C, A
14AC  3A 85 E2           :..     LD     A, ($E285)
14AF  47                 G       LD     B, A
14B0  3A 95 E2           :..     LD     A, ($E295)
14B3  80                 .       ADD    A, B
14B4  3C                 <       INC    A
14B5  47                 G       LD     B, A
14B6  28 04              (.      JR     Z, $14BC
.
14B8  CB 09              ..      RRC    C
14BA  10 FC              ..      DJNZ   $14B8
.
14BC  21 62 E2           !b.     LD     HL, $E262
14BF  09                 .       ADD    HL, BC
14C0  3A 95 E2           :..     LD     A, ($E295)
14C3  47                 G       LD     B, A
14C4  3A 72 E2           :r.     LD     A, ($E272)
.
14C7  CB 3F              .?      SRL    A
14C9  10 FC              ..      DJNZ   $14C7
14CB  4F                 O       LD     C, A
14CC  3A 85 E2           :..     LD     A, ($E285)
14CF  B7                 .       OR     A
14D0  28 02              (.      JR     Z, $14D4
14D2  CB 21              .!      SLA    C
.
14D4  09                 .       ADD    HL, BC
14D5  5E                 ^       LD     E, (HL)
14D6  23                 #       INC    HL
14D7  A6                 .       AND    (HL)
14D8  57                 W       LD     D, A
14D9  B3                 .       OR     E
14DA  28 16              (.      JR     Z, $14F2
14DC  3A 95 E2           :..     LD     A, ($E295)
14DF  47                 G       LD     B, A
14E0  EB                 .       EX     DE, HL
.
14E1  29                 )       ADD    HL, HL
14E2  10 FD              ..      DJNZ   $14E1
14E4  5D                 ]       LD     E, L
14E5  54                 T       LD     D, H
14E6  3A 72 E2           :r.     LD     A, ($E272)
14E9  4F                 O       LD     C, A
14EA  3A 96 E2           :..     LD     A, ($E296)
14ED  A1                 .       AND    C
14EE  4F                 O       LD     C, A
14EF  09                 .       ADD    HL, BC
14F0  AF                 .       XOR    A
14F1  C9                 .       RET
.
14F2  2B                 +       DEC    HL
14F3  3E FF              >.      LD     A, $FF
14F5  B7                 .       OR     A
14F6  C9                 .       RET
14F7  DD 66 0E           .f.     LD     H, (IX+$0E)
14FA  AF                 .       XOR    A
14FB  CB BC              ..      RES    7, H
14FD  06 03              ..      LD     B, $03
.
14FF  CB 1C              ..      RR     H
1501  1F                 .       RRA
1502  10 FB              ..      DJNZ   $14FF
1504  DD B6 0C           ...     OR     (IX+$0C)
1507  6F                 o       LD     L, A
1508  C9                 .       RET
1509  CD 4E E7           .N.     CALL   $E74E
150C  B7                 .       OR     A
150D  3E 03              >.      LD     A, $03
150F  F8                 .       RET    M
1510  21 5E E2           !^.     LD     HL, $E25E
1513  34                 4       INC    (HL)
1514  CB 6E              .n      BIT    5, (HL)
1516  28 09              (.      JR     Z, $1521
1518  36 00              6.      LD     (HL), $00
151A  23                 #       INC    HL
151B  23                 #       INC    HL
151C  34                 4       INC    (HL)
151D  87                 .       ADD    A, A
151E  CB 66              .f      BIT    4, (HL)
1520  C0                 .       RET    NZ
.
1521  CD F2 E6           ...     CALL   $E6F2
1524  B7                 .       OR     A
1525  3E 04              >.      LD     A, $04
1527  F8                 .       RET    M
1528  AF                 .       XOR    A
1529  C9                 .       RET
152A  DD 21 52 E2        .!R.    LD     IX, $E252
152E  CD D3 EE           ...     CALL   $EED3
1531  ED 5B 77 E2        .[w.    LD     DE, ($E277)
1535  AF                 .       XOR    A
1536  ED 52              .R      SBC    HL, DE
1538  C8                 .       RET    Z
1539  CD 4E E7           .N.     CALL   $E74E
153C  B7                 .       OR     A
153D  3E 03              >.      LD     A, $03
153F  F8                 .       RET    M
1540  2A 77 E2           *w.     LD     HL, ($E277)
1543  7D                 }       LD     A, L
1544  E6 1F              ..      AND    $1F
1546  32 5E E2           2^.     LD     ($E25E), A
1549  29                 )       ADD    HL, HL
154A  29                 )       ADD    HL, HL
154B  29                 )       ADD    HL, HL
154C  7C                 |       LD     A, H
154D  32 60 E2           2`.     LD     ($E260), A
1550  C3 FD EE           ...     JP     $EEFD
1553  0F                 .       RCCA
1554  0F                 .       RCCA
1555  0F                 .       RCCA
1556  4F                 O       LD     C, A
1557  06 00              ..      LD     B, $00
1559  2A 8B E2           *..     LD     HL, ($E28B)
155C  09                 .       ADD    HL, BC
155D  C9                 .       RET
155E  3A 52 E2           :R.     LD     A, ($E252)
1561  3D                 =       DEC    A
1562  F2 44 EF           .D.     JP     P $EF44
1565  3A 1F E2           :..     LD     A, ($E21F)
1568  5F                 _       LD     E, A
1569  C3 FC E5           ...     JP     $E5FC
156C  3A 73 E2           :s.     LD     A, ($E273)
156F  4F                 O       LD     C, A
1570  CB BF              ..      RES    7, A
1572  32 79 E2           2y.     LD     ($E279), A
1575  3A 74 E2           :t.     LD     A, ($E274)
1578  CB 21              .!      SLA    C
157A  CB 17              ..      RL     A
157C  4F                 O       LD     C, A
157D  3A 75 E2           :u.     LD     A, ($E275)
1580  CB 17              ..      RL     A
1582  47                 G       LD     B, A
1583  ED 43 77 E2        .Cw.    LD     ($E277), BC
1587  C9                 .       RET
1588  21 52 E2           !R.     LD     HL, $E252
158B  ED 53 24 E2        .S$.    LD     ($E224), DE
158F  EB                 .       EX     DE, HL
1590  01 24 00           .$.     LD     BC, $0024
1593  ED B0              ..      LDIR
1595  C9                 .       RET
1596  21 52 E2           !R.     LD     HL, $E252
1599  ED 5B 24 E2        .[$.    LD     DE, ($E224)
159D  01 21 00           .!.     LD     BC, $0021
15A0  ED B0              ..      LDIR
15A2  AF                 .       XOR    A
15A3  C9                 .       RET
15A4  3A 5B E2           :[.     LD     A, ($E25B)
15A7  CB 7F              .      BIT    7, A
15A9  C8                 .       RET    Z
15AA  18 1B              ..      JR     $15C7
15AC  D1                 .       POP    DE
15AD  11 C6 E2           ...     LD     DE, $E2C6
15B0  2A 0B E2           *..     LD     HL, ($E20B)
15B3  E9                 .       JP     (HL)
15B4  11 CF E2           ...     LD     DE, $E2CF
15B7  18 03              ..      JR     $15BC
15B9  11 D5 E2           ...     LD     DE, $E2D5
.
15BC  2A 09 E2           *..     LD     HL, ($E209)
15BF  E9                 .       JP     (HL)
15C0  11 DC E2           ...     LD     DE, $E2DC
15C3  2A 0D E2           *..     LD     HL, ($E20D)
15C6  E9                 .       JP     (HL)
.
15C7  11 E5 E2           ...     LD     DE, $E2E5
15CA  2A 0F E2           *..     LD     HL, ($E20F)
15CD  E9                 .       JP     (HL)
15CE  D5                 .       PUSH   DE
15CF  11 12 E5           ...     LD     DE, $E512
15D2  CD 67 E4           .g.     CALL   $E467
15D5  D1                 .       POP    DE
15D6  CD 67 E4           .g.     CALL   $E467
15D9  3A 20 E2           : .     LD     A, ($E220)
15DC  C6 41              .A      ADD    A, $41
15DE  32 26 E3           2&.     LD     ($E326), A
15E1  11 1C E3           ...     LD     DE, $E31C
15E4  CD 67 E4           .g.     CALL   $E467
15E7  CD B0 E3           ...     CALL   $E3B0
15EA  C3 03 F0           ...     JP     $F003
15ED  3A 20 E2           : .     LD     A, ($E220)
15F0  C6 41              .A      ADD    A, $41
15F2  32 F8 E2           2..     LD     ($E2F8), A
15F5  CD 67 E4           .g.     CALL   $E467
15F8  11 EE E2           ...     LD     DE, $E2EE
15FB  CD 67 E4           .g.     CALL   $E467
.
15FE  CD B0 E3           ...     CALL   $E3B0
1601  E6 DF              ..      AND    $DF
1603  FE 49              .I      CP     $49
1605  C8                 .       RET    Z
1606  FE 52              .R      CP     $52
1608  20 02               .      JR     NZ $160C
160A  B7                 .       OR     A
160B  C9                 .       RET
.
160C  FE 57              .W      CP     $57
160E  20 EE               .      JR     NZ $15FE
1610  C3 03 F0           ...     JP     $F003
1613  00                 .       NOP
1614  FF                 .       RST    38H
1615  FF                 .       RST    38H
1616  FF                 .       RST    38H
1617  FF                 .       RST    38H
1618  00                 .       NOP
1619  00                 .       NOP
161A  00                 .       NOP
161B  00                 .       NOP
161C  FF                 .       RST    38H
161D  FF                 .       RST    38H
161E  FF                 .       RST    38H
161F  FF                 .       RST    38H
1620  00                 .       NOP
1621  00                 .       NOP
1622  00                 .       NOP
1623  00                 .       NOP
1624  C3 80 F0           ...     JP     $F080
1627  C3 28 F1           .(.     JP     $F128
162A  C3 8B F1           ...     JP     $F18B
162D  C3 C8 F1           ...     JP     $F1C8
1630  C3 EB F1           ...     JP     $F1EB
1633  C3 25 F2           .%.     JP     $F225
1636  C3 42 F2           .B.     JP     $F242
1639  C3 0B F2           ...     JP     $F20B
163C  C3 9A F2           ...     JP     $F29A
163F  C3 79 F2           .y.     JP     $F279
1642  C3 5F F2           ._.     JP     $F25F
1645  C3 69 F2           .i.     JP     $F269
1648  C3 73 F2           .s.     JP     $F273
164B  C3 A8 F2           ...     JP     $F2A8
164E  C3 C6 F2           ...     JP     $F2C6
1651  C3 A3 F2           ...     JP     $F2A3
1654  C3 A0 F2           ...     JP     $F2A0
1657  C3 00 00           ...     JP     $0000
165A  C3 00 00           ...     JP     $0000
165D  C3 00 00           ...     JP     $0000
1660  00                 .       NOP
1661  00                 .       NOP
1662  00                 .       NOP
1663  00                 .       NOP
1664  00                 .       NOP
1665  00                 .       NOP
1666  00                 .       NOP
1667  00                 .       NOP
.
1668  98                 .       SBC    B
1669  F7                 .       RST    30H
166A  6D                 m       LD     L, L
166B  F7                 .       RST    30H
166C  AC                 .       XOR    H
166D  F9                 .       LD     SP, HL
166E  18 F8              ..      JR     $1668
1670  00                 .       NOP
1671  00                 .       NOP
1672  00                 .       NOP
1673  00                 .       NOP
1674  00                 .       NOP
1675  00                 .       NOP
1676  00                 .       NOP
1677  00                 .       NOP
1678  98                 .       SBC    B
1679  F7                 .       RST    30H
167A  7C                 |       LD     A, H
167B  F7                 .       RST    30H
167C  ED                 #.      ...
167C  F9                 $.      ...
167E  7D                 }       LD     A, L
167F  F8                 .       RET    M
1680  00                 .       NOP
1681  00                 .       NOP
1682  00                 .       NOP
1683  00                 .       NOP
1684  00                 .       NOP
1685  00                 .       NOP
1686  00                 .       NOP
1687  00                 .       NOP
1688  98                 .       SBC    B
1689  F7                 .       RST    30H
168A  6D                 m       LD     L, L
168B  F7                 .       RST    30H
168C  2E FA              ..      LD     L, $FA
168E  E2 F8 00           ...     JP     PO $00F8
1691  00                 .       NOP
1692  00                 .       NOP
1693  00                 .       NOP
1694  00                 .       NOP
1695  00                 .       NOP
1696  00                 .       NOP
1697  00                 .       NOP
1698  98                 .       SBC    B
1699  F7                 .       RST    30H
169A  7C                 |       LD     A, H
169B  F7                 .       RST    30H
169C  6F                 o       LD     L, A
169D  FA 47 F9           .G.     JP     M $F947
16A0  50                 P       LD     D, B
16A1  49                 I       LD     C, C
16A2  4E                 N       LD     C, (HL)
16A3  4E                 N       LD     C, (HL)
16A4  AF                 .       XOR    A
16A5  D3 80              ..      OUT    ($80), A
16A7  32 04 00           2..     LD     ($0004), A
16AA  3E 81              >.      LD     A, $81
16AC  32 03 00           2..     LD     ($0003), A
16AF  C3 37 F1           .7.     JP     $F137
16B2  D3 00              ..      OUT    ($00), A
16B4  DB 00              ..      IN     A, ($00)
16B6  5F                 _       LD     E, A
16B7  DB 00              ..      IN     A, ($00)
16B9  BB                 .       CP     E
16BA  C2 90 F0           ...     JP     NZ $F090
16BD  B7                 .       OR     A
16BE  F2 90 F0           ...     JP     P $F090
16C1  AF                 .       XOR    A
16C2  D3 00              ..      OUT    ($00), A
16C4  C9                 .       RET
16C5  DB 00              ..      IN     A, ($00)
16C7  5F                 _       LD     E, A
16C8  DB 00              ..      IN     A, ($00)
16CA  BB                 .       CP     E
16CB  C2 A1 F0           ...     JP     NZ $F0A1
16CE  B7                 .       OR     A
16CF  FA A1 F0           ...     JP     M $F0A1
16D2  CB 47              .G      BIT    0, A
16D4  C8                 .       RET    Z
16D5  F5                 .       PUSH   AF
16D6  AF                 .       XOR    A
16D7  D3 01              ..      OUT    ($01), A
16D9  3E 81              >.      LD     A, $81
16DB  CD 8E F0           ...     CALL   $F08E
16DE  F1                 .       POP    AF
16DF  C3 FD FF           ...     JP     $FFFD
16E2  0E 09              ..      LD     C, $09
16E4  11 C9 F0           ...     LD     DE, $F0C9
16E7  CD 05 00           ...     CALL   $0005
16EA  C3 00 00           ...     JP     $0000
16ED  0D                 .       DEC    C
16EE  0A                 .       LD     A, (BC)
16EF  55                 U       LD     D, L
16F0  6E                 n       LD     L, (HL)
16F1  69                 i       LD     L, C
16F2  6D                 m       LD     L, L
16F3  70                 p       LD     (HL), B
16F4  6C                 l       LD     L, H
16F5  65                 e       LD     H, L
16F6  6D                 m       LD     L, L
16F7  65                 e       LD     H, L
16F8  6E                 n       LD     L, (HL)
16F9  74                 t       LD     (HL), H
16FA  65                 e       LD     H, L
16FB  64                 d       LD     H, H
16FC  20 4F               O      JR     NZ $174D
16FE  53                 S       LD     D, E
16FF  20 63               c      JR     NZ $1764
1701  61                 a       LD     H, C
1702  6C                 l       LD     L, H
1703  6C                 l       LD     L, H
1704  2E 0D              ..      LD     L, $0D
1706  0A                 .       LD     A, (BC)
1707  24                 $       INC    H
1708  C3 BE F0           ...     JP     $F0BE
170B  C3 39 F7           .9.     JP     $F739
170E  C3 BE F0           ...     JP     $F0BE
1711  C3 36 F7           .6.     JP     $F736
1714  C3 33 F7           .3.     JP     $F733
1717  C3 30 F7           .0.     JP     $F730
171A  C3 C6 F3           ...     JP     $F3C6
171D  C3 9A F3           ...     JP     $F39A
1720  C3 6E F5           .n.     JP     $F56E
1723  C3 BE F0           ...     JP     $F0BE
1726  C3 45 F5           .E.     JP     $F545
1729  C3 5C F5           .\.     JP     $F55C
172C  C3 8E F5           ...     JP     $F58E
172F  C3 BE F0           ...     JP     $F0BE
1732  C3 87 F3           ...     JP     $F387
1735  C3 A2 F3           ...     JP     $F3A2
1738  00                 .       NOP
1739  C3 B4 F3           ...     JP     $F3B4
173C  00                 .       NOP
173D  C3 BE F0           ...     JP     $F0BE
1740  C3 C1 F3           ...     JP     $F3C1
1743  C3 CB F3           ...     JP     $F3CB
1746  C3 DA F4           ...     JP     $F4DA
1749  C3 16 F5           ...     JP     $F516
174C  DB 81              ..      IN     A, ($81)
174E  21 24 00           !$.     LD     HL, $0024
1751  11 00 DA           ...     LD     DE, $DA00
1754  01 61 1D           .a.     LD     BC, $1D61
1757  ED B0              ..      LDIR
1759  D3 81              ..      OUT    ($81), A
175B  21 E4 F0           !..     LD     HL, $F0E4
175E  11 B6 FF           ...     LD     DE, $FFB6
1761  01 44 00           .D.     LD     BC, $0044
.
1764  ED B0              ..      LDIR
1766  31 80 00           1..     LD     SP, $0080
1769  3E C3              >.      LD     A, $C3
176B  32 FD FF           2..     LD     ($FFFD), A
176E  21 E1 F2           !..     LD     HL, $F2E1
1771  22 FE FF           "..     LD     ($FFFE), HL
1774  CD A1 F0           ...     CALL   $F0A1
1777  AF                 .       XOR    A
1778  32 80 FF           2..     LD     ($FF80), A
177B  06 1E              ..      LD     B, $1E
177D  21 6D F7           !m.     LD     HL, $F76D
.
1780  3E BA              >.      LD     A, $BA
1782  CD 8E F0           ...     CALL   $F08E
1785  CD A1 F0           ...     CALL   $F0A1
1788  DB 01              ..      IN     A, ($01)
178A  77                 w       LD     (HL), A
178B  23                 #       INC    HL
178C  10 F2              ..      DJNZ   $1780
178E  3E C3              >.      LD     A, $C3
1790  32 00 00           2..     LD     ($0000), A
1793  21 03 F0           !..     LD     HL, $F003
1796  22 01 00           "..     LD     ($0001), HL
1799  32 05 00           2..     LD     ($0005), A
179C  21 06 E2           !..     LD     HL, $E206
179F  22 06 00           "..     LD     ($0006), HL
17A2  01 80 00           ...     LD     BC, $0080
17A5  CD 73 F2           .s.     CALL   $F273
17A8  3A 04 00           :..     LD     A, ($0004)
17AB  4F                 O       LD     C, A
17AC  C3 00 DA           ...     JP     $DA00
17AF  3A 03 00           :..     LD     A, ($0003)
17B2  E6 03              ..      AND    $03
17B4  06 85              ..      LD     B, $85
17B6  28 23              (#      JR     Z, $17DB
17B8  FE 01              ..      CP     $01
17BA  06 86              ..      LD     B, $86
17BC  28 1D              (.      JR     Z, $17DB
17BE  FE 02              ..      CP     $02
17C0  28 02              (.      JR     Z, $17C4
17C2  AF                 .       XOR    A
17C3  C9                 .       RET
.
17C4  3A 03 00           :..     LD     A, ($0003)
17C7  E6 0C              ..      AND    $0C
17C9  06 85              ..      LD     B, $85
17CB  28 0E              (.      JR     Z, $17DB
17CD  FE 04              ..      CP     $04
17CF  06 95              ..      LD     B, $95
17D1  28 08              (.      JR     Z, $17DB
17D3  FE 08              ..      CP     $08
17D5  06 96              ..      LD     B, $96
17D7  28 02              (.      JR     Z, $17DB
17D9  06 97              ..      LD     B, $97
.
17DB  CD A1 F0           ...     CALL   $F0A1
17DE  78                 x       LD     A, B
17DF  CD 8E F0           ...     CALL   $F08E
17E2  CD A1 F0           ...     CALL   $F0A1
17E5  CB 6F              .o      BIT    5, A
17E7  3E FF              >.      LD     A, $FF
17E9  C8                 .       RET    Z
17EA  AF                 .       XOR    A
17EB  C9                 .       RET
17EC  3A 03 00           :..     LD     A, ($0003)
17EF  E6 03              ..      AND    $03
17F1  06 82              ..      LD     B, $82
17F3  28 0D              (.      JR     Z, $1802
17F5  FE 01              ..      CP     $01
17F7  06 80              ..      LD     B, $80
17F9  28 07              (.      JR     Z, $1802
17FB  FE 02              ..      CP     $02
17FD  CA 0B F2           ...     JP     Z $F20B
1800  06 81              ..      LD     B, $81
.
1802  CD A1 F0           ...     CALL   $F0A1
1805  78                 x       LD     A, B
1806  CD 8E F0           ...     CALL   $F08E
1809  CD A1 F0           ...     CALL   $F0A1
180C  DB 01              ..      IN     A, ($01)
180E  C9                 .       RET
180F  3A 03 00           :..     LD     A, ($0003)
1812  E6 03              ..      AND    $03
1814  06 8A              ..      LD     B, $8A
1816  28 0D              (.      JR     Z, $1825
1818  FE 01              ..      CP     $01
181A  06 8D              ..      LD     B, $8D
181C  28 07              (.      JR     Z, $1825
181E  FE 02              ..      CP     $02
1820  CA 25 F2           .%.     JP     Z $F225
1823  06 89              ..      LD     B, $89
.
1825  CD A1 F0           ...     CALL   $F0A1
1828  79                 y       LD     A, C
1829  D3 01              ..      OUT    ($01), A
182B  78                 x       LD     A, B
182C  C3 8E F0           ...     JP     $F08E
182F  3A 03 00           :..     LD     A, ($0003)
1832  E6 0C              ..      AND    $0C
1834  06 82              ..      LD     B, $82
1836  28 CA              (.      JR     Z, $1802
1838  FE 04              ..      CP     $04
183A  06 90              ..      LD     B, $90
183C  28 C4              (.      JR     Z, $1802
183E  FE 08              ..      CP     $08
1840  06 83              ..      LD     B, $83
1842  28 BE              (.      JR     Z, $1802
1844  06 84              ..      LD     B, $84
1846  C3 DE F1           ...     JP     $F1DE
1849  3A 03 00           :..     LD     A, ($0003)
184C  E6 C0              ..      AND    $C0
184E  06 8A              ..      LD     B, $8A
1850  CA 01 F2           ...     JP     Z $F201
1853  FE 40              .@      CP     $40
1855  06 8D              ..      LD     B, $8D
1857  CA 01 F2           ...     JP     Z $F201
185A  FE 80              ..      CP     $80
185C  06 8E              ..      LD     B, $8E
185E  CA 01 F2           ...     JP     Z $F201
1861  06 8F              ..      LD     B, $8F
1863  C3 01 F2           ...     JP     $F201
1866  3A 03 00           :..     LD     A, ($0003)
1869  E6 30              .0      AND    $30
186B  06 8A              ..      LD     B, $8A
186D  CA 01 F2           ...     JP     Z $F201
1870  FE 10              ..      CP     $10
1872  06 91              ..      LD     B, $91
1874  CA 01 F2           ...     JP     Z $F201
1877  FE 20              .       CP     $20
1879  06 8B              ..      LD     B, $8B
187B  CA 01 F2           ...     JP     Z $F201
187E  06 8C              ..      LD     B, $8C
1880  C3 01 F2           ...     JP     $F201
1883  60                 `       LD     H, B
1884  69                 i       LD     L, C
1885  22 91 F7           "..     LD     ($F791), HL
1888  06 B3              ..      LD     B, $B3
188A  C3 01 F2           ...     JP     $F201
188D  60                 `       LD     H, B
188E  69                 i       LD     L, C
188F  22 93 F7           "..     LD     ($F793), HL
1892  06 B5              ..      LD     B, $B5
1894  C3 01 F2           ...     JP     $F201
1897  69                 i       LD     L, C
1898  60                 `       LD     H, B
1899  22 95 F7           "..     LD     ($F795), HL
189C  C9                 .       RET
189D  21 00 00           !..     LD     HL, $0000
18A0  79                 y       LD     A, C
18A1  32 97 F7           2..     LD     ($F797), A
18A4  FE 04              ..      CP     $04
18A6  D0                 .       RET    NC
18A7  CD A1 F0           ...     CALL   $F0A1
18AA  79                 y       LD     A, C
18AB  D3 01              ..      OUT    ($01), A
18AD  3E B6              >.      LD     A, $B6
18AF  CD 8E F0           ...     CALL   $F08E
18B2  69                 i       LD     L, C
18B3  26 00              &.      LD     H, $00
18B5  29                 )       ADD    HL, HL
18B6  29                 )       ADD    HL, HL
18B7  29                 )       ADD    HL, HL
18B8  29                 )       ADD    HL, HL
18B9  11 3C F0           .<.     LD     DE, $F03C
18BC  19                 .       ADD    HL, DE
18BD  C9                 .       RET
18BE  01 00 00           ...     LD     BC, $0000
18C1  C3 5F F2           ._.     JP     $F25F
18C4  60                 `       LD     H, B
18C5  69                 i       LD     L, C
18C6  C9                 .       RET
18C7  06 88              ..      LD     B, $88
18C9  C3 B7 F1           ...     JP     $F1B7
18CC  AF                 .       XOR    A
18CD  32 6C F7           2l.     LD     ($F76C), A
18D0  CD A1 F0           ...     CALL   $F0A1
18D3  06 80              ..      LD     B, $80
18D5  2A 95 F7           *..     LD     HL, ($F795)
.
18D8  3E B9              >.      LD     A, $B9
18DA  CD 8E F0           ...     CALL   $F08E
18DD  CD A1 F0           ...     CALL   $F0A1
18E0  DB 01              ..      IN     A, ($01)
18E2  77                 w       LD     (HL), A
18E3  23                 #       INC    HL
18E4  10 F2              ..      DJNZ   $18D8
18E6  3A 6C F7           :l.     LD     A, ($F76C)
18E9  C9                 .       RET
18EA  AF                 .       XOR    A
18EB  32 6C F7           2l.     LD     ($F76C), A
18EE  2A 95 F7           *..     LD     HL, ($F795)
18F1  06 80              ..      LD     B, $80
.
18F3  CD A1 F0           ...     CALL   $F0A1
18F6  7E                 ~       LD     A, (HL)
18F7  D3 01              ..      OUT    ($01), A
18F9  3E B7              >.      LD     A, $B7
18FB  CD 8E F0           ...     CALL   $F08E
18FE  23                 #       INC    HL
18FF  10 F2              ..      DJNZ   $18F3
1901  3A 6C F7           :l.     LD     A, ($F76C)
1904  C9                 .       RET
1905  E5                 .       PUSH   HL
1906  D5                 .       PUSH   DE
1907  C5                 .       PUSH   BC
1908  F5                 .       PUSH   AF
1909  CD 38 F3           .8.     CALL   $F338
190C  CD B4 F3           ...     CALL   $F3B4
190F  F1                 .       POP    AF
1910  F5                 .       PUSH   AF
1911  CB 4F              .O      BIT    1, A
1913  28 27              ('      JR     Z, $193C
1915  3E 01              >.      LD     A, $01
1917  32 6C F7           2l.     LD     ($F76C), A
191A  21 1D F3           !..     LD     HL, $F31D
.
191D  7E                 ~       LD     A, (HL)
191E  FE 24              .$      CP     $24
1920  28 06              (.      JR     Z, $1928
1922  CD C1 F3           ...     CALL   $F3C1
1925  23                 #       INC    HL
1926  18 F5              ..      JR     $191D
.
1928  3E 0F              >.      LD     A, $0F
192A  21 00 00           !..     LD     HL, $0000
192D  CD DA F4           ...     CALL   $F4DA
1930  CD 87 F3           ...     CALL   $F387
1933  FE 69              .i      CP     $69
1935  28 05              (.      JR     Z, $193C
1937  FE 49              .I      CP     $49
1939  C2 00 00           ...     JP     NZ $0000
.
193C  F1                 .       POP    AF
193D  C1                 .       POP    BC
193E  D1                 .       POP    DE
193F  E1                 .       POP    HL
1940  C9                 .       RET
1941  0D                 .       DEC    C
1942  0A                 .       LD     A, (BC)
1943  20 28               (      JR     NZ $196D
1945  52                 R       LD     D, D
1946  29                 )       ADD    HL, HL
1947  65                 e       LD     H, L
1948  62                 b       LD     H, D
1949  6F                 o       LD     L, A
194A  6F                 o       LD     L, A
194B  74                 t       LD     (HL), H
194C  20 6F               o      JR     NZ $19BD
194E  72                 r       LD     (HL), D
194F  20 28               (      JR     NZ $1979
1951  49                 I       LD     C, C
1952  29                 )       ADD    HL, HL
1953  67                 g       LD     H, A
1954  6E                 n       LD     L, (HL)
1955  6F                 o       LD     L, A
1956  72                 r       LD     (HL), D
1957  65                 e       LD     H, L
1958  3F                 ?       CCF
1959  0D                 .       DEC    C
195A  0A                 .       LD     A, (BC)
195B  24                 $       INC    H
195C  CD B4 F3           ...     CALL   $F3B4
195F  21 FD 00           !..     LD     HL, $00FD
1962  CD 49 F4           .I.     CALL   $F449
1965  CD A1 F0           ...     CALL   $F0A1
1968  3E C9              >.      LD     A, $C9
196A  CD 77 F3           .w.     CALL   $F377
.
196D  CD A1 F0           ...     CALL   $F0A1
1970  DB 01              ..      IN     A, ($01)
1972  6F                 o       LD     L, A
1973  3E C9              >.      LD     A, $C9
1975  CD 77 F3           .w.     CALL   $F377
1978  CD A1 F0           ...     CALL   $F0A1
197B  DB 01              ..      IN     A, ($01)
197D  67                 g       LD     H, A
197E  CD 49 F4           .I.     CALL   $F449
1981  CD 08 F5           ...     CALL   $F508
1984  32 81 FF           2..     LD     ($FF81), A
.
1987  CD A1 F0           ...     CALL   $F0A1
198A  3E C9              >.      LD     A, $C9
198C  CD 77 F3           .w.     CALL   $F377
198F  CD A1 F0           ...     CALL   $F0A1
1992  DB 01              ..      IN     A, ($01)
1994  B7                 .       OR     A
1995  C8                 .       RET    Z
1996  CD C1 F3           ...     CALL   $F3C1
1999  18 EC              ..      JR     $1987
199B  5F                 _       LD     E, A
199C  DB 00              ..      IN     A, ($00)
199E  E6 04              ..      AND    $04
19A0  28 05              (.      JR     Z, $19A7
19A2  3E 80              >.      LD     A, $80
19A4  32 80 FF           2..     LD     ($FF80), A
.
19A7  7B                 {       LD     A, E
19A8  C3 8E F0           ...     JP     $F08E
19AB  D5                 .       PUSH   DE
19AC  CD A1 F0           ...     CALL   $F0A1
19AF  3E A6              >.      LD     A, $A6
.
19B1  CD 77 F3           .w.     CALL   $F377
19B4  CD 82 F4           ...     CALL   $F482
19B7  57                 W       LD     D, A
19B8  CD 37 F4           .7.     CALL   $F437
19BB  7A                 z       LD     A, D
19BC  D1                 .       POP    DE
.
19BD  C9                 .       RET
19BE  D5                 .       PUSH   DE
19BF  CD A1 F0           ...     CALL   $F0A1
19C2  3E AE              >.      LD     A, $AE
19C4  18 EB              ..      JR     $19B1
19C6  D5                 .       PUSH   DE
19C7  16 A7              ..      LD     D, $A7
.
19C9  F5                 .       PUSH   AF
19CA  CD A1 F0           ...     CALL   $F0A1
19CD  F1                 .       POP    AF
19CE  F5                 .       PUSH   AF
19CF  D3 01              ..      OUT    ($01), A
19D1  7A                 z       LD     A, D
19D2  CD 77 F3           .w.     CALL   $F377
19D5  F1                 .       POP    AF
19D6  D1                 .       POP    DE
19D7  C9                 .       RET
19D8  D5                 .       PUSH   DE
19D9  CD A1 F0           ...     CALL   $F0A1
19DC  3E A8              >.      LD     A, $A8
19DE  CD 77 F3           .w.     CALL   $F377
19E1  3E 0D              >.      LD     A, $0D
19E3  D1                 .       POP    DE
19E4  C9                 .       RET
19E5  D5                 .       PUSH   DE
19E6  16 A9              ..      LD     D, $A9
19E8  18 DF              ..      JR     $19C9
19EA  D5                 .       PUSH   DE
19EB  16 AF              ..      LD     D, $AF
19ED  18 DA              ..      JR     $19C9
19EF  D5                 .       PUSH   DE
19F0  F5                 .       PUSH   AF
19F1  CD 90 F4           ...     CALL   $F490
19F4  E5                 .       PUSH   HL
19F5  CD 46 F4           .F.     CALL   $F446
19F8  E1                 .       POP    HL
19F9  F1                 .       POP    AF
19FA  B7                 .       OR     A
19FB  CA 9C F4           ...     JP     Z $F49C
19FE  FE 0E              ..      CP     $0E
1A00  D2 D8 F5           ...     JP     NC $F5D8
1A03  E5                 .       PUSH   HL
1A04  3E 10              >.      LD     A, $10
1A06  CD 5F F4           ._.     CALL   $F45F
1A09  CD C9 F4           ...     CALL   $F4C9
1A0C  CD 46 F4           .F.     CALL   $F446
1A0F  E1                 .       POP    HL
1A10  E5                 .       PUSH   HL
1A11  3E 10              >.      LD     A, $10
1A13  CD 6F F4           .o.     CALL   $F46F
1A16  CD F8 F3           ...     CALL   $F3F8
1A19  E1                 .       POP    HL
1A1A  D1                 .       POP    DE
1A1B  C9                 .       RET
1A1C  CD 1A F4           ...     CALL   $F41A
1A1F  CD 82 F4           ...     CALL   $F482
1A22  57                 W       LD     D, A
1A23  CD 37 F4           .7.     CALL   $F437
1A26  7A                 z       LD     A, D
1A27  C9                 .       RET
1A28  CD A1 F0           ...     CALL   $F0A1
1A2B  7D                 }       LD     A, L
1A2C  D3 01              ..      OUT    ($01), A
1A2E  3E C0              >.      LD     A, $C0
1A30  CD 77 F3           .w.     CALL   $F377
1A33  CD A1 F0           ...     CALL   $F0A1
1A36  7C                 |       LD     A, H
1A37  D3 01              ..      OUT    ($01), A
1A39  3E C1              >.      LD     A, $C1
1A3B  C3 77 F3           .w.     JP     $F377
1A3E  CD A1 F0           ...     CALL   $F0A1
1A41  3E C3              >.      LD     A, $C3
1A43  CD 77 F3           .w.     CALL   $F377
1A46  CD A1 F0           ...     CALL   $F0A1
1A49  DB 01              ..      IN     A, ($01)
1A4B  6F                 o       LD     L, A
1A4C  CD A1 F0           ...     CALL   $F0A1
1A4F  3E C4              >.      LD     A, $C4
1A51  CD 77 F3           .w.     CALL   $F377
1A54  CD A1 F0           ...     CALL   $F0A1
1A57  DB 01              ..      IN     A, ($01)
1A59  67                 g       LD     H, A
1A5A  C9                 .       RET
1A5B  CD A1 F0           ...     CALL   $F0A1
1A5E  3E CA              >.      LD     A, $CA
1A60  CD 77 F3           .w.     CALL   $F377
1A63  CD A1 F0           ...     CALL   $F0A1
1A66  DB 01              ..      IN     A, ($01)
1A68  1F                 .       RRA
1A69  C9                 .       RET
1A6A  21 00 06           !..     LD     HL, $0600
1A6D  CD A1 F0           ...     CALL   $F0A1
1A70  7C                 |       LD     A, H
1A71  D3 01              ..      OUT    ($01), A
1A73  3E C8              >.      LD     A, $C8
1A75  CD 77 F3           .w.     CALL   $F377
1A78  CD A1 F0           ...     CALL   $F0A1
1A7B  7D                 }       LD     A, L
1A7C  D3 01              ..      OUT    ($01), A
1A7E  3E C7              >.      LD     A, $C7
1A80  C3 77 F3           .w.     JP     $F377
1A83  47                 G       LD     B, A
.
1A84  CD A1 F0           ...     CALL   $F0A1
1A87  7E                 ~       LD     A, (HL)
1A88  D3 01              ..      OUT    ($01), A
1A8A  3E CB              >.      LD     A, $CB
1A8C  CD 77 F3           .w.     CALL   $F377
1A8F  23                 #       INC    HL
1A90  10 F2              ..      DJNZ   $1A84
1A92  C9                 .       RET
1A93  47                 G       LD     B, A
1A94  CD A1 F0           ...     CALL   $F0A1
.
1A97  3E C9              >.      LD     A, $C9
1A99  CD 77 F3           .w.     CALL   $F377
1A9C  CD A1 F0           ...     CALL   $F0A1
1A9F  DB 01              ..      IN     A, ($01)
1AA1  77                 w       LD     (HL), A
1AA2  23                 #       INC    HL
1AA3  10 F2              ..      DJNZ   $1A97
1AA5  C9                 .       RET
1AA6  CD A1 F0           ...     CALL   $F0A1
1AA9  3E C5              >.      LD     A, $C5
1AAB  CD 77 F3           .w.     CALL   $F377
1AAE  CD A1 F0           ...     CALL   $F0A1
1AB1  DB 01              ..      IN     A, ($01)
1AB3  C9                 .       RET
1AB4  F5                 .       PUSH   AF
1AB5  CD A1 F0           ...     CALL   $F0A1
1AB8  F1                 .       POP    AF
1AB9  D3 01              ..      OUT    ($01), A
1ABB  3E C2              >.      LD     A, $C2
1ABD  C3 77 F3           .w.     JP     $F377
1AC0  5E                 ^       LD     E, (HL)
1AC1  36 00              6.      LD     (HL), $00
1AC3  23                 #       INC    HL
1AC4  56                 V       LD     D, (HL)
1AC5  36 07              6.      LD     (HL), $07
1AC7  2B                 +       DEC    HL
1AC8  3E 05              >.      LD     A, $05
1ACA  D5                 .       PUSH   DE
1ACB  E5                 .       PUSH   HL
1ACC  CD 5F F4           ._.     CALL   $F45F
1ACF  CD C9 F4           ...     CALL   $F4C9
1AD2  E1                 .       POP    HL
1AD3  D1                 .       POP    DE
1AD4  E5                 .       PUSH   HL
1AD5  D5                 .       PUSH   DE
1AD6  73                 s       LD     (HL), E
1AD7  23                 #       INC    HL
1AD8  72                 r       LD     (HL), D
1AD9  21 00 07           !..     LD     HL, $0700
1ADC  CD 49 F4           .I.     CALL   $F449
1ADF  CD 28 F4           .(.     CALL   $F428
1AE2  3C                 <       INC    A
1AE3  E1                 .       POP    HL
1AE4  CD 6F F4           .o.     CALL   $F46F
1AE7  CD F8 F3           ...     CALL   $F3F8
1AEA  E1                 .       POP    HL
1AEB  D1                 .       POP    DE
1AEC  C9                 .       RET
1AED  E5                 .       PUSH   HL
1AEE  21 00 06           !..     LD     HL, $0600
1AF1  CD 04 F4           ...     CALL   $F404
1AF4  CD A1 F0           ...     CALL   $F0A1
1AF7  3E AA              >.      LD     A, $AA
1AF9  CD 77 F3           .w.     CALL   $F377
1AFC  E1                 .       POP    HL
1AFD  C9                 .       RET
1AFE  D5                 .       PUSH   DE
1AFF  FE 7E              .~      CP     $7E
1B01  C2 E6 F4           ...     JP     NZ $F4E6
1B04  AF                 .       XOR    A
1B05  32 80 FF           2..     LD     ($FF80), A
1B08  3E 7E              >~      LD     A, $7E
1B0A  CD F6 F4           ...     CALL   $F4F6
1B0D  CD A1 F0           ...     CALL   $F0A1
1B10  3E AB              >.      LD     A, $AB
1B12  CD 77 F3           .w.     CALL   $F377
1B15  CD F8 F3           ...     CALL   $F3F8
1B18  D1                 .       POP    DE
1B19  C9                 .       RET
1B1A  CD 90 F4           ...     CALL   $F490
1B1D  C3 04 F4           ...     JP     $F404
1B20  F5                 .       PUSH   AF
1B21  CD A1 F0           ...     CALL   $F0A1
1B24  F1                 .       POP    AF
1B25  D3 01              ..      OUT    ($01), A
1B27  3E CB              >.      LD     A, $CB
1B29  C3 77 F3           .w.     JP     $F377
1B2C  CD A1 F0           ...     CALL   $F0A1
1B2F  3E C9              >.      LD     A, $C9
1B31  CD 77 F3           .w.     CALL   $F377
1B34  CD A1 F0           ...     CALL   $F0A1
1B37  DB 01              ..      IN     A, ($01)
1B39  C9                 .       RET
1B3A  D5                 .       PUSH   DE
1B3B  CD 24 F5           .$.     CALL   $F524
1B3E  3E AC              >.      LD     A, $AC
1B40  CD 77 F3           .w.     CALL   $F377
1B43  CD A1 F0           ...     CALL   $F0A1
1B46  D1                 .       POP    DE
1B47  C9                 .       RET
1B48  E5                 .       PUSH   HL
1B49  CD 46 F4           .F.     CALL   $F446
1B4C  E1                 .       POP    HL
.
1B4D  CD A1 F0           ...     CALL   $F0A1
1B50  7E                 ~       LD     A, (HL)
1B51  57                 W       LD     D, A
1B52  D3 01              ..      OUT    ($01), A
1B54  3E CB              >.      LD     A, $CB
1B56  CD 77 F3           .w.     CALL   $F377
1B59  23                 #       INC    HL
1B5A  3E 0D              >.      LD     A, $0D
1B5C  BA                 .       CP     D
1B5D  20 EE               .      JR     NZ $1B4D
1B5F  21 00 06           !..     LD     HL, $0600
1B62  CD 04 F4           ...     CALL   $F404
1B65  CD A1 F0           ...     CALL   $F0A1
1B68  C9                 .       RET
1B69  D5                 .       PUSH   DE
1B6A  E5                 .       PUSH   HL
1B6B  F5                 .       PUSH   AF
1B6C  CD F6 F4           ...     CALL   $F4F6
1B6F  CD A1 F0           ...     CALL   $F0A1
1B72  3E A2              >.      LD     A, $A2
1B74  CD 77 F3           .w.     CALL   $F377
1B77  F1                 .       POP    AF
.
1B78  57                 W       LD     D, A
1B79  CD 37 F4           .7.     CALL   $F437
1B7C  7A                 z       LD     A, D
1B7D  E1                 .       POP    HL
1B7E  D1                 .       POP    DE
1B7F  C9                 .       RET
1B80  D5                 .       PUSH   DE
1B81  E5                 .       PUSH   HL
1B82  CD 0F F4           ...     CALL   $F40F
1B85  CD A1 F0           ...     CALL   $F0A1
1B88  3E A3              >.      LD     A, $A3
1B8A  CD 77 F3           .w.     CALL   $F377
1B8D  CD 82 F4           ...     CALL   $F482
1B90  18 E6              ..      JR     $1B78
1B92  E5                 .       PUSH   HL
1B93  D5                 .       PUSH   DE
1B94  F5                 .       PUSH   AF
1B95  B7                 .       OR     A
1B96  28 15              (.      JR     Z, $1BAD
1B98  CD 24 F5           .$.     CALL   $F524
.
1B9B  F1                 .       POP    AF
1B9C  CD 90 F4           ...     CALL   $F490
1B9F  CD A1 F0           ...     CALL   $F0A1
1BA2  3E A0              >.      LD     A, $A0
1BA4  CD 77 F3           .w.     CALL   $F377
1BA7  CD 82 F4           ...     CALL   $F482
1BAA  D1                 .       POP    DE
1BAB  E1                 .       POP    HL
1BAC  C9                 .       RET
.
1BAD  CD 04 F4           ...     CALL   $F404
1BB0  18 E9              ..      JR     $1B9B
1BB2  C5                 .       PUSH   BC
1BB3  D5                 .       PUSH   DE
1BB4  F5                 .       PUSH   AF
1BB5  E5                 .       PUSH   HL
1BB6  21 8C 00           !..     LD     HL, $008C
1BB9  CD 49 F4           .I.     CALL   $F449
1BBC  E1                 .       POP    HL
1BBD  E5                 .       PUSH   HL
1BBE  26 00              &.      LD     H, $00
1BC0  3E 04              >.      LD     A, $04
1BC2  CD 5F F4           ._.     CALL   $F45F
1BC5  E1                 .       POP    HL
1BC6  F1                 .       POP    AF
1BC7  F5                 .       PUSH   AF
1BC8  E5                 .       PUSH   HL
1BC9  2E 8C              ..      LD     L, $8C
1BCB  CD F6 F4           ...     CALL   $F4F6
1BCE  CD A1 F0           ...     CALL   $F0A1
1BD1  3E A4              >.      LD     A, $A4
1BD3  CD 77 F3           .w.     CALL   $F377
1BD6  E1                 .       POP    HL
1BD7  E5                 .       PUSH   HL
1BD8  21 8C 00           !..     LD     HL, $008C
1BDB  CD 49 F4           .I.     CALL   $F449
1BDE  E1                 .       POP    HL
1BDF  E5                 .       PUSH   HL
1BE0  26 00              &.      LD     H, $00
1BE2  3E 04              >.      LD     A, $04
1BE4  CD 6F F4           .o.     CALL   $F46F
1BE7  E1                 .       POP    HL
1BE8  F1                 .       POP    AF
1BE9  FE 01              ..      CP     $01
1BEB  20 09               .      JR     NZ $1BF6
1BED  AF                 .       XOR    A
1BEE  BC                 .       CP     H
1BEF  20 05               .      JR     NZ $1BF6
1BF1  54                 T       LD     D, H
1BF2  CD 1A F4           ...     CALL   $F41A
1BF5  62                 b       LD     H, D
.
1BF6  CD 82 F4           ...     CALL   $F482
1BF9  D1                 .       POP    DE
1BFA  C1                 .       POP    BC
1BFB  C9                 .       RET
1BFC  FE 7E              .~      CP     $7E
1BFE  20 0F               .      JR     NZ $1C0F
1C00  E5                 .       PUSH   HL
1C01  CD C9 F4           ...     CALL   $F4C9
1C04  CD 46 F4           .F.     CALL   $F446
1C07  3E 04              >.      LD     A, $04
1C09  E1                 .       POP    HL
1C0A  CD 6F F4           .o.     CALL   $F46F
1C0D  D1                 .       POP    DE
1C0E  C9                 .       RET
.
1C0F  FE 7F              .      CP     $7F
1C11  D1                 .       POP    DE
1C12  C0                 .       RET    NZ
1C13  D5                 .       PUSH   DE
1C14  C5                 .       PUSH   BC
1C15  22 61 F7           "a.     LD     ($F761), HL
1C18  21 00 06           !..     LD     HL, $0600
1C1B  CD 49 F4           .I.     CALL   $F449
1C1E  2A 61 F7           *a.     LD     HL, ($F761)
1C21  7E                 ~       LD     A, (HL)
1C22  CD FC F4           ...     CALL   $F4FC
1C25  3E 83              >.      LD     A, $83
1C27  CD DA F4           ...     CALL   $F4DA
1C2A  22 63 F7           "c.     LD     ($F763), HL
1C2D  7D                 }       LD     A, L
1C2E  CD FC F4           ...     CALL   $F4FC
1C31  7C                 |       LD     A, H
1C32  CD FC F4           ...     CALL   $F4FC
1C35  AF                 .       XOR    A
1C36  CD FC F4           ...     CALL   $F4FC
1C39  CD FC F4           ...     CALL   $F4FC
1C3C  2A 61 F7           *a.     LD     HL, ($F761)
1C3F  23                 #       INC    HL
1C40  7E                 ~       LD     A, (HL)
1C41  32 65 F7           2e.     LD     ($F765), A
1C44  23                 #       INC    HL
1C45  7E                 ~       LD     A, (HL)
1C46  32 66 F7           2f.     LD     ($F766), A
1C49  23                 #       INC    HL
1C4A  23                 #       INC    HL
1C4B  23                 #       INC    HL
1C4C  7E                 ~       LD     A, (HL)
1C4D  32 67 F7           2g.     LD     ($F767), A
1C50  CD FC F4           ...     CALL   $F4FC
1C53  23                 #       INC    HL
1C54  7E                 ~       LD     A, (HL)
1C55  32 68 F7           2h.     LD     ($F768), A
1C58  CD FC F4           ...     CALL   $F4FC
1C5B  23                 #       INC    HL
1C5C  06 00              ..      LD     B, $00
.
1C5E  7E                 ~       LD     A, (HL)
1C5F  4F                 O       LD     C, A
1C60  CD FC F4           ...     CALL   $F4FC
1C63  23                 #       INC    HL
1C64  3E 02              >.      LD     A, $02
1C66  B8                 .       CP     B
1C67  20 04               .      JR     NZ $1C6D
1C69  79                 y       LD     A, C
1C6A  32 6B F7           2k.     LD     ($F76B), A
.
1C6D  3A 67 F7           :g.     LD     A, ($F767)
1C70  04                 .       INC    B
1C71  B8                 .       CP     B
1C72  20 EA               .      JR     NZ $1C5E
1C74  22 61 F7           "a.     LD     ($F761), HL
1C77  3A 68 F7           :h.     LD     A, ($F768)
1C7A  FE 63              .c      CP     $63
1C7C  28 04              (.      JR     Z, $1C82
1C7E  FE 5B              .[      CP     $5B
1C80  20 0E               .      JR     NZ $1C90
.
1C82  3A 6B F7           :k.     LD     A, ($F76B)
1C85  E6 1F              ..      AND    $1F
1C87  CB 27              .'      SLA    A
1C89  CB 27              .'      SLA    A
1C8B  6F                 o       LD     L, A
1C8C  26 00              &.      LD     H, $00
1C8E  18 40              .@      JR     $1CD0
.
1C90  FE 5F              ._      CP     $5F
1C92  28 04              (.      JR     Z, $1C98
1C94  FE 69              .i      CP     $69
1C96  20 05               .      JR     NZ $1C9D
.
1C98  21 00 00           !..     LD     HL, $0000
1C9B  18 33              .3      JR     $1CD0
.
1C9D  FE 53              .S      CP     $53
1C9F  28 0D              (.      JR     Z, $1CAE
1CA1  FE 57              .W      CP     $57
1CA3  28 09              (.      JR     Z, $1CAE
1CA5  FE 4F              .O      CP     $4F
1CA7  28 05              (.      JR     Z, $1CAE
1CA9  FE 4B              .K      CP     $4B
1CAB  C2 FB F6           ...     JP     NZ $F6FB
.
1CAE  3A 6B F7           :k.     LD     A, ($F76B)
1CB1  4F                 O       LD     C, A
1CB2  E6 1F              ..      AND    $1F
1CB4  5F                 _       LD     E, A
1CB5  79                 y       LD     A, C
1CB6  E6 E0              ..      AND    $E0
1CB8  07                 .       RCLA
1CB9  07                 .       RCLA
1CBA  07                 .       RCLA
1CBB  07                 .       RCLA
1CBC  4F                 O       LD     C, A
1CBD  06 00              ..      LD     B, $00
1CBF  21 28 F7           !(.     LD     HL, $F728
1CC2  09                 .       ADD    HL, BC
1CC3  4E                 N       LD     C, (HL)
1CC4  23                 #       INC    HL
1CC5  46                 F       LD     B, (HL)
1CC6  AF                 .       XOR    A
1CC7  67                 g       LD     H, A
1CC8  6F                 o       LD     L, A
1CC9  BB                 .       CP     E
1CCA  28 04              (.      JR     Z, $1CD0
.
1CCC  09                 .       ADD    HL, BC
1CCD  1D                 .       DEC    E
1CCE  20 FC               .      JR     NZ $1CCC
.
1CD0  22 69 F7           "i.     LD     ($F769), HL
1CD3  3A 68 F7           :h.     LD     A, ($F768)
1CD6  FE 4F              .O      CP     $4F
1CD8  28 08              (.      JR     Z, $1CE2
1CDA  FE 4B              .K      CP     $4B
1CDC  28 04              (.      JR     Z, $1CE2
1CDE  FE 63              .c      CP     $63
1CE0  20 1C               .      JR     NZ $1CFE
.
1CE2  2A 63 F7           *c.     LD     HL, ($F763)
1CE5  CD 49 F4           .I.     CALL   $F449
1CE8  ED 4B 69 F7        .Ki.    LD     BC, ($F769)
1CEC  2A 65 F7           *e.     LD     HL, ($F765)
.
1CEF  7E                 ~       LD     A, (HL)
1CF0  CD FC F4           ...     CALL   $F4FC
1CF3  23                 #       INC    HL
1CF4  0B                 .       DEC    BC
1CF5  78                 x       LD     A, B
1CF6  B1                 .       OR     C
1CF7  20 F6               .      JR     NZ $1CEF
1CF9  CD 03 F7           ...     CALL   $F703
1CFC  18 24              .$      JR     $1D22
.
1CFE  CD 03 F7           ...     CALL   $F703
1D01  2A 63 F7           *c.     LD     HL, ($F763)
1D04  CD 49 F4           .I.     CALL   $F449
1D07  ED 4B 69 F7        .Ki.    LD     BC, ($F769)
1D0B  AF                 .       XOR    A
1D0C  B8                 .       CP     B
1D0D  20 03               .      JR     NZ $1D12
1D0F  B9                 .       CP     C
1D10  28 0D              (.      JR     Z, $1D1F
.
1D12  2A 65 F7           *e.     LD     HL, ($F765)
.
1D15  CD 08 F5           ...     CALL   $F508
1D18  77                 w       LD     (HL), A
1D19  23                 #       INC    HL
1D1A  0B                 .       DEC    BC
1D1B  78                 x       LD     A, B
1D1C  B1                 .       OR     C
1D1D  20 F6               .      JR     NZ $1D15
.
1D1F  2A 61 F7           *a.     LD     HL, ($F761)
.
1D22  3E 7F              >      LD     A, $7F
1D24  C1                 .       POP    BC
1D25  D1                 .       POP    DE
1D26  C9                 .       RET
1D27  3E 7F              >      LD     A, $7F
1D29  21 00 06           !..     LD     HL, $0600
1D2C  CD F6 F4           ...     CALL   $F4F6
1D2F  CD A1 F0           ...     CALL   $F0A1
1D32  3E AA              >.      LD     A, $AA
1D34  CD 8E F0           ...     CALL   $F08E
1D37  21 07 06           !..     LD     HL, $0607
1D3A  06 00              ..      LD     B, $00
1D3C  3A 67 F7           :g.     LD     A, ($F767)
1D3F  4F                 O       LD     C, A
1D40  09                 .       ADD    HL, BC
1D41  CD 49 F4           .I.     CALL   $F449
1D44  CD 08 F5           ...     CALL   $F508
1D47  2A 61 F7           *a.     LD     HL, ($F761)
1D4A  77                 w       LD     (HL), A
1D4B  C9                 .       RET
1D4C  80                 .       ADD    A, B
1D4D  00                 .       NOP
1D4E  00                 .       NOP
1D4F  01 00 02           ...     LD     BC, $0200
1D52  00                 .       NOP
1D53  04                 .       INC    B
1D54  C3 BE F0           ...     JP     $F0BE
1D57  C3 BE F0           ...     JP     $F0BE
1D5A  C3 BE F0           ...     JP     $F0BE
1D5D  C3 BE F0           ...     JP     $F0BE
1D60  42                 B       LD     B, D
1D61  69                 i       LD     L, C
1D62  6F                 o       LD     L, A
1D63  73                 s       LD     (HL), E
1D64  20 32               2      JR     NZ $1D98
1D66  2E 30              .0      LD     L, $30
1D68  28 63              (c      JR     Z, $1DCD
1D6A  29                 )       ADD    HL, HL
1D6B  52                 R       LD     D, D
1D6C  2E 48              .H      LD     L, $48
1D6E  6F                 o       LD     L, A
1D6F  64                 d       LD     H, H
1D70  67                 g       LD     H, A
1D71  73                 s       LD     (HL), E
1D72  6F                 o       LD     L, A
1D73  6E                 n       LD     L, (HL)
1D74  20 31               1      JR     NZ $1DA7
1D76  39                 9       ADD    HL, SP
1D77  2F                 /       CPL
1D78  31 30 2F           10/     LD     SP, $2F30
1D7B  38 35              85      JR     C, $1DB2
1D7D  20 66               f      JR     NZ $1DE5
1D7F  6F                 o       LD     L, A
1D80  72                 r       LD     (HL), D
1D81  20 4F               O      JR     NZ $1DD2
1D83  53                 S       LD     D, E
1D84  4D                 M       LD     C, L
1D85  FF                 .       RST    38H
1D86  FF                 .       RST    38H
1D87  FF                 .       RST    38H
1D88  FF                 .       RST    38H
1D89  FF                 .       RST    38H
1D8A  FF                 .       RST    38H
1D8B  FF                 .       RST    38H
1D8C  FF                 .       RST    38H
1D8D  FF                 .       RST    38H
1D8E  FF                 .       RST    38H
1D8F  FF                 .       RST    38H
1D90  FF                 .       RST    38H
1D91  FF                 .       RST    38H
1D92  FF                 .       RST    38H
1D93  FF                 .       RST    38H
1D94  FF                 .       RST    38H
1D95  FF                 .       RST    38H
1D96  FF                 .       RST    38H
1D97  FF                 .       RST    38H
.
1D98  FF                 .       RST    38H
1D99  FF                 .       RST    38H
1D9A  FF                 .       RST    38H
1D9B  FF                 .       RST    38H
1D9C  FF                 .       RST    38H
1D9D  FF                 .       RST    38H
1D9E  FF                 .       RST    38H
1D9F  FF                 .       RST    38H
1DA0  FF                 .       RST    38H
1DA1  FF                 .       RST    38H
1DA2  FF                 .       RST    38H
1DA3  FF                 .       RST    38H
1DA4  FF                 .       RST    38H
1DA5  FF                 .       RST    38H
1DA6  FF                 .       RST    38H
.
1DA7  FF                 .       RST    38H
1DA8  FF                 .       RST    38H
1DA9  FF                 .       RST    38H
1DAA  FF                 .       RST    38H
1DAB  FF                 .       RST    38H
1DAC  FF                 .       RST    38H
1DAD  FF                 .       RST    38H
1DAE  FF                 .       RST    38H
1DAF  FF                 .       RST    38H
1DB0  FF                 .       RST    38H
1DB1  FF                 .       RST    38H
.
1DB2  FF                 .       RST    38H
1DB3  FF                 .       RST    38H
1DB4  FF                 .       RST    38H
1DB5  FF                 .       RST    38H
1DB6  FF                 .       RST    38H
1DB7  FF                 .       RST    38H
1DB8  FF                 .       RST    38H
1DB9  FF                 .       RST    38H
1DBA  FF                 .       RST    38H
1DBB  FF                 .       RST    38H
1DBC  FF                 .       RST    38H
1DBD  FF                 .       RST    38H
1DBE  FF                 .       RST    38H
1DBF  FF                 .       RST    38H
1DC0  FF                 .       RST    38H
1DC1  FF                 .       RST    38H
1DC2  FF                 .       RST    38H
1DC3  FF                 .       RST    38H
1DC4  FF                 .       RST    38H
1DC5  FF                 .       RST    38H
1DC6  FF                 .       RST    38H
1DC7  FF                 .       RST    38H
1DC8  FF                 .       RST    38H
1DC9  FF                 .       RST    38H
1DCA  FF                 .       RST    38H
1DCB  FF                 .       RST    38H
1DCC  FF                 .       RST    38H
.
1DCD  FF                 .       RST    38H
1DCE  FF                 .       RST    38H
1DCF  FF                 .       RST    38H
1DD0  FF                 .       RST    38H
1DD1  FF                 .       RST    38H
.
1DD2  FF                 .       RST    38H
1DD3  FF                 .       RST    38H
1DD4  FF                 .       RST    38H
1DD5  FF                 .       RST    38H
1DD6  FF                 .       RST    38H
1DD7  FF                 .       RST    38H
1DD8  FF                 .       RST    38H
1DD9  FF                 .       RST    38H
1DDA  FF                 .       RST    38H
1DDB  FF                 .       RST    38H
1DDC  FF                 .       RST    38H
1DDD  FF                 .       RST    38H
1DDE  FF                 .       RST    38H
1DDF  FF                 .       RST    38H
1DE0  FF                 .       RST    38H
1DE1  FF                 .       RST    38H
1DE2  FF                 .       RST    38H
1DE3  FF                 .       RST    38H
1DE4  FF                 .       RST    38H
.
1DE5  FF                 .       RST    38H
1DE6  FF                 .       RST    38H
1DE7  FF                 .       RST    38H
1DE8  FF                 .       RST    38H
1DE9  FF                 .       RST    38H
1DEA  FF                 .       RST    38H
1DEB  FF                 .       RST    38H
1DEC  FF                 .       RST    38H
1DED  FF                 .       RST    38H
1DEE  FF                 .       RST    38H
1DEF  FF                 .       RST    38H
1DF0  FF                 .       RST    38H
1DF1  FF                 .       RST    38H
1DF2  FF                 .       RST    38H
1DF3  FF                 .       RST    38H
1DF4  FF                 .       RST    38H
1DF5  FF                 .       RST    38H
1DF6  FF                 .       RST    38H
1DF7  FF                 .       RST    38H
1DF8  FF                 .       RST    38H
1DF9  FF                 .       RST    38H
1DFA  FF                 .       RST    38H
1DFB  FF                 .       RST    38H
1DFC  FF                 .       RST    38H
1DFD  FF                 .       RST    38H
1DFE  FF                 .       RST    38H
1DFF  FF                 .       RST    38H
1E00  FF                 .       RST    38H
1E01  FF                 .       RST    38H
1E02  FF                 .       RST    38H
1E03  FF                 .       RST    38H
1E04  FF                 .       RST    38H
1E05  FF                 .       RST    38H
1E06  FF                 .       RST    38H
1E07  FF                 .       RST    38H
1E08  FF                 .       RST    38H
1E09  FF                 .       RST    38H
1E0A  FF                 .       RST    38H
1E0B  FF                 .       RST    38H
1E0C  FF                 .       RST    38H
1E0D  FF                 .       RST    38H
1E0E  FF                 .       RST    38H
1E0F  FF                 .       RST    38H
1E10  FF                 .       RST    38H
1E11  FF                 .       RST    38H
1E12  FF                 .       RST    38H
1E13  FF                 .       RST    38H
1E14  FF                 .       RST    38H
1E15  FF                 .       RST    38H
1E16  FF                 .       RST    38H
1E17  FF                 .       RST    38H
1E18  FF                 .       RST    38H
1E19  FF                 .       RST    38H
1E1A  FF                 .       RST    38H
1E1B  FF                 .       RST    38H
1E1C  FF                 .       RST    38H
1E1D  FF                 .       RST    38H
1E1E  FF                 .       RST    38H
1E1F  FF                 .       RST    38H
1E20  FF                 .       RST    38H
1E21  FF                 .       RST    38H
1E22  FF                 .       RST    38H
1E23  FF                 .       RST    38H
1E24  FF                 .       RST    38H
1E25  FF                 .       RST    38H
1E26  FF                 .       RST    38H
1E27  FF                 .       RST    38H
1E28  FF                 .       RST    38H
1E29  FF                 .       RST    38H
1E2A  FF                 .       RST    38H
1E2B  FF                 .       RST    38H
1E2C  FF                 .       RST    38H
1E2D  FF                 .       RST    38H
1E2E  FF                 .       RST    38H
1E2F  FF                 .       RST    38H
1E30  FF                 .       RST    38H
1E31  FF                 .       RST    38H
1E32  FF                 .       RST    38H
1E33  FF                 .       RST    38H
1E34  FF                 .       RST    38H
1E35  FF                 .       RST    38H
1E36  FF                 .       RST    38H
1E37  FF                 .       RST    38H
1E38  FF                 .       RST    38H
1E39  FF                 .       RST    38H
1E3A  FF                 .       RST    38H
1E3B  FF                 .       RST    38H
1E3C  FF                 .       RST    38H
1E3D  FF                 .       RST    38H
1E3E  FF                 .       RST    38H
1E3F  FF                 .       RST    38H
1E40  FF                 .       RST    38H
1E41  FF                 .       RST    38H
1E42  FF                 .       RST    38H
1E43  FF                 .       RST    38H
1E44  FF                 .       RST    38H
1E45  FF                 .       RST    38H
1E46  FF                 .       RST    38H
1E47  FF                 .       RST    38H
1E48  FF                 .       RST    38H
1E49  FF                 .       RST    38H
1E4A  FF                 .       RST    38H
1E4B  FF                 .       RST    38H
1E4C  FF                 .       RST    38H
1E4D  FF                 .       RST    38H
1E4E  FF                 .       RST    38H
1E4F  FF                 .       RST    38H
1E50  FF                 .       RST    38H
1E51  FF                 .       RST    38H
1E52  FF                 .       RST    38H
1E53  FF                 .       RST    38H
1E54  FF                 .       RST    38H
1E55  FF                 .       RST    38H
1E56  FF                 .       RST    38H
1E57  FF                 .       RST    38H
1E58  FF                 .       RST    38H
1E59  FF                 .       RST    38H
1E5A  FF                 .       RST    38H
1E5B  FF                 .       RST    38H
1E5C  FF                 .       RST    38H
1E5D  FF                 .       RST    38H
1E5E  FF                 .       RST    38H
1E5F  FF                 .       RST    38H
1E60  FF                 .       RST    38H
1E61  FF                 .       RST    38H
1E62  FF                 .       RST    38H
1E63  FF                 .       RST    38H
1E64  FF                 .       RST    38H
1E65  FF                 .       RST    38H
1E66  FF                 .       RST    38H
1E67  FF                 .       RST    38H
1E68  FF                 .       RST    38H
1E69  FF                 .       RST    38H
1E6A  FF                 .       RST    38H
1E6B  FF                 .       RST    38H
1E6C  FF                 .       RST    38H
1E6D  FF                 .       RST    38H
1E6E  FF                 .       RST    38H
1E6F  FF                 .       RST    38H
1E70  FF                 .       RST    38H
1E71  FF                 .       RST    38H
1E72  FF                 .       RST    38H
1E73  FF                 .       RST    38H
1E74  FF                 .       RST    38H
1E75  FF                 .       RST    38H
1E76  FF                 .       RST    38H
1E77  FF                 .       RST    38H
1E78  FF                 .       RST    38H
1E79  FF                 .       RST    38H
1E7A  FF                 .       RST    38H
1E7B  FF                 .       RST    38H
1E7C  FF                 .       RST    38H
1E7D  FF                 .       RST    38H
1E7E  FF                 .       RST    38H
1E7F  FF                 .       RST    38H
1E80  FF                 .       RST    38H
1E81  FF                 .       RST    38H
1E82  FF                 .       RST    38H
1E83  FF                 .       RST    38H
1E84  FF                 .       RST    38H
1E85  FF                 .       RST    38H
1E86  FF                 .       RST    38H
1E87  FF                 .       RST    38H
1E88  FF                 .       RST    38H
1E89  FF                 .       RST    38H
1E8A  FF                 .       RST    38H
1E8B  FF                 .       RST    38H
1E8C  FF                 .       RST    38H
1E8D  FF                 .       RST    38H
1E8E  FF                 .       RST    38H
1E8F  FF                 .       RST    38H
1E90  FF                 .       RST    38H
1E91  FF                 .       RST    38H
1E92  FF                 .       RST    38H
1E93  FF                 .       RST    38H
1E94  FF                 .       RST    38H
1E95  FF                 .       RST    38H
1E96  FF                 .       RST    38H
1E97  FF                 .       RST    38H
1E98  FF                 .       RST    38H
1E99  FF                 .       RST    38H
1E9A  FF                 .       RST    38H
1E9B  FF                 .       RST    38H
1E9C  FF                 .       RST    38H
1E9D  FF                 .       RST    38H
1E9E  FF                 .       RST    38H
1E9F  FF                 .       RST    38H
1EA0  FF                 .       RST    38H
1EA1  FF                 .       RST    38H
1EA2  FF                 .       RST    38H
1EA3  FF                 .       RST    38H
1EA4  FF                 .       RST    38H
1EA5  FF                 .       RST    38H
1EA6  FF                 .       RST    38H
1EA7  FF                 .       RST    38H
1EA8  FF                 .       RST    38H
1EA9  FF                 .       RST    38H
1EAA  FF                 .       RST    38H
1EAB  FF                 .       RST    38H
1EAC  FF                 .       RST    38H
1EAD  FF                 .       RST    38H
1EAE  FF                 .       RST    38H
1EAF  FF                 .       RST    38H
1EB0  FF                 .       RST    38H
1EB1  FF                 .       RST    38H
1EB2  FF                 .       RST    38H
1EB3  FF                 .       RST    38H
1EB4  FF                 .       RST    38H
1EB5  FF                 .       RST    38H
1EB6  FF                 .       RST    38H
1EB7  FF                 .       RST    38H
1EB8  FF                 .       RST    38H
1EB9  FF                 .       RST    38H
1EBA  FF                 .       RST    38H
1EBB  FF                 .       RST    38H
1EBC  FF                 .       RST    38H
1EBD  FF                 .       RST    38H
1EBE  FF                 .       RST    38H
1EBF  FF                 .       RST    38H
1EC0  FF                 .       RST    38H
1EC1  FF                 .       RST    38H
1EC2  FF                 .       RST    38H
1EC3  FF                 .       RST    38H
1EC4  FF                 .       RST    38H
1EC5  FF                 .       RST    38H
1EC6  FF                 .       RST    38H
1EC7  FF                 .       RST    38H
1EC8  FF                 .       RST    38H
1EC9  FF                 .       RST    38H
1ECA  FF                 .       RST    38H
1ECB  FF                 .       RST    38H
1ECC  FF                 .       RST    38H
1ECD  FF                 .       RST    38H
1ECE  FF                 .       RST    38H
1ECF  FF                 .       RST    38H
1ED0  FF                 .       RST    38H
1ED1  FF                 .       RST    38H
1ED2  FF                 .       RST    38H
1ED3  FF                 .       RST    38H
1ED4  FF                 .       RST    38H
1ED5  FF                 .       RST    38H
1ED6  FF                 .       RST    38H
1ED7  FF                 .       RST    38H
1ED8  FF                 .       RST    38H
1ED9  FF                 .       RST    38H
1EDA  FF                 .       RST    38H
1EDB  FF                 .       RST    38H
1EDC  FF                 .       RST    38H
1EDD  FF                 .       RST    38H
1EDE  FF                 .       RST    38H
1EDF  FF                 .       RST    38H
1EE0  FF                 .       RST    38H
1EE1  FF                 .       RST    38H
1EE2  FF                 .       RST    38H
1EE3  FF                 .       RST    38H
1EE4  FF                 .       RST    38H
1EE5  FF                 .       RST    38H
1EE6  FF                 .       RST    38H
1EE7  FF                 .       RST    38H
1EE8  FF                 .       RST    38H
1EE9  FF                 .       RST    38H
1EEA  FF                 .       RST    38H
1EEB  FF                 .       RST    38H
1EEC  FF                 .       RST    38H
1EED  FF                 .       RST    38H
1EEE  FF                 .       RST    38H
1EEF  FF                 .       RST    38H
1EF0  FF                 .       RST    38H
1EF1  FF                 .       RST    38H
1EF2  FF                 .       RST    38H
1EF3  FF                 .       RST    38H
1EF4  FF                 .       RST    38H
1EF5  FF                 .       RST    38H
1EF6  FF                 .       RST    38H
1EF7  FF                 .       RST    38H
1EF8  FF                 .       RST    38H
1EF9  FF                 .       RST    38H
1EFA  FF                 .       RST    38H
1EFB  FF                 .       RST    38H
1EFC  FF                 .       RST    38H
1EFD  FF                 .       RST    38H
1EFE  FF                 .       RST    38H
1EFF  FF                 .       RST    38H
1F00  FF                 .       RST    38H
1F01  FF                 .       RST    38H
1F02  FF                 .       RST    38H
1F03  FF                 .       RST    38H
1F04  FF                 .       RST    38H
1F05  FF                 .       RST    38H
1F06  FF                 .       RST    38H
1F07  FF                 .       RST    38H
1F08  FF                 .       RST    38H
1F09  FF                 .       RST    38H
1F0A  FF                 .       RST    38H
1F0B  FF                 .       RST    38H
1F0C  FF                 .       RST    38H
1F0D  FF                 .       RST    38H
1F0E  FF                 .       RST    38H
1F0F  FF                 .       RST    38H
1F10  FF                 .       RST    38H
1F11  FF                 .       RST    38H
1F12  FF                 .       RST    38H
1F13  FF                 .       RST    38H
1F14  FF                 .       RST    38H
1F15  FF                 .       RST    38H
1F16  FF                 .       RST    38H
1F17  FF                 .       RST    38H
1F18  FF                 .       RST    38H
1F19  FF                 .       RST    38H
1F1A  FF                 .       RST    38H
1F1B  FF                 .       RST    38H
1F1C  FF                 .       RST    38H
1F1D  FF                 .       RST    38H
1F1E  FF                 .       RST    38H
1F1F  FF                 .       RST    38H
1F20  FF                 .       RST    38H
1F21  FF                 .       RST    38H
1F22  FF                 .       RST    38H
1F23  FF                 .       RST    38H
1F24  FF                 .       RST    38H
1F25  FF                 .       RST    38H
1F26  FF                 .       RST    38H
1F27  FF                 .       RST    38H
1F28  FF                 .       RST    38H
1F29  FF                 .       RST    38H
1F2A  FF                 .       RST    38H
1F2B  FF                 .       RST    38H
1F2C  FF                 .       RST    38H
1F2D  FF                 .       RST    38H
1F2E  FF                 .       RST    38H
1F2F  FF                 .       RST    38H
1F30  FF                 .       RST    38H
1F31  FF                 .       RST    38H
1F32  FF                 .       RST    38H
1F33  FF                 .       RST    38H
1F34  FF                 .       RST    38H
1F35  FF                 .       RST    38H
1F36  FF                 .       RST    38H
1F37  FF                 .       RST    38H
1F38  FF                 .       RST    38H
1F39  FF                 .       RST    38H
1F3A  FF                 .       RST    38H
1F3B  FF                 .       RST    38H
1F3C  FF                 .       RST    38H
1F3D  FF                 .       RST    38H
1F3E  FF                 .       RST    38H
1F3F  FF                 .       RST    38H
1F40  FF                 .       RST    38H
1F41  FF                 .       RST    38H
1F42  FF                 .       RST    38H
1F43  FF                 .       RST    38H
1F44  FF                 .       RST    38H
1F45  FF                 .       RST    38H
1F46  FF                 .       RST    38H
1F47  FF                 .       RST    38H
1F48  FF                 .       RST    38H
1F49  FF                 .       RST    38H
1F4A  FF                 .       RST    38H
1F4B  FF                 .       RST    38H
1F4C  FF                 .       RST    38H
1F4D  FF                 .       RST    38H
1F4E  FF                 .       RST    38H
1F4F  FF                 .       RST    38H
1F50  FF                 .       RST    38H
1F51  FF                 .       RST    38H
1F52  FF                 .       RST    38H
1F53  FF                 .       RST    38H
1F54  FF                 .       RST    38H
1F55  FF                 .       RST    38H
1F56  FF                 .       RST    38H
1F57  FF                 .       RST    38H
1F58  FF                 .       RST    38H
1F59  FF                 .       RST    38H
1F5A  FF                 .       RST    38H
1F5B  FF                 .       RST    38H
1F5C  FF                 .       RST    38H
1F5D  FF                 .       RST    38H
1F5E  FF                 .       RST    38H
1F5F  FF                 .       RST    38H
1F60  FF                 .       RST    38H
1F61  FF                 .       RST    38H
1F62  FF                 .       RST    38H
1F63  FF                 .       RST    38H
1F64  FF                 .       RST    38H
1F65  FF                 .       RST    38H
1F66  FF                 .       RST    38H
1F67  FF                 .       RST    38H
1F68  FF                 .       RST    38H
1F69  FF                 .       RST    38H
1F6A  FF                 .       RST    38H
1F6B  FF                 .       RST    38H
1F6C  FF                 .       RST    38H
1F6D  FF                 .       RST    38H
1F6E  FF                 .       RST    38H
1F6F  FF                 .       RST    38H
1F70  FF                 .       RST    38H
1F71  FF                 .       RST    38H
1F72  FF                 .       RST    38H
1F73  FF                 .       RST    38H
1F74  FF                 .       RST    38H
1F75  FF                 .       RST    38H
1F76  FF                 .       RST    38H
1F77  FF                 .       RST    38H
1F78  FF                 .       RST    38H
1F79  FF                 .       RST    38H
1F7A  FF                 .       RST    38H
1F7B  FF                 .       RST    38H
1F7C  FF                 .       RST    38H
1F7D  FF                 .       RST    38H
1F7E  FF                 .       RST    38H
1F7F  FF                 .       RST    38H
1F80  FF                 .       RST    38H
1F81  FF                 .       RST    38H
1F82  FF                 .       RST    38H
1F83  FF                 .       RST    38H
1F84  FF                 .       RST    38H
1F85  FF                 .       RST    38H
1F86  FF                 .       RST    38H
1F87  FF                 .       RST    38H
1F88  FF                 .       RST    38H
1F89  FF                 .       RST    38H
1F8A  FF                 .       RST    38H
1F8B  FF                 .       RST    38H
1F8C  FF                 .       RST    38H
1F8D  FF                 .       RST    38H
1F8E  FF                 .       RST    38H
1F8F  FF                 .       RST    38H
1F90  FF                 .       RST    38H
1F91  FF                 .       RST    38H
1F92  FF                 .       RST    38H
1F93  FF                 .       RST    38H
1F94  FF                 .       RST    38H
1F95  FF                 .       RST    38H
1F96  FF                 .       RST    38H
1F97  FF                 .       RST    38H
1F98  FF                 .       RST    38H
1F99  FF                 .       RST    38H
1F9A  FF                 .       RST    38H
1F9B  FF                 .       RST    38H
1F9C  FF                 .       RST    38H
1F9D  FF                 .       RST    38H
1F9E  FF                 .       RST    38H
1F9F  FF                 .       RST    38H
1FA0  FF                 .       RST    38H
1FA1  FF                 .       RST    38H
1FA2  FF                 .       RST    38H
1FA3  FF                 .       RST    38H
1FA4  FF                 .       RST    38H
1FA5  FF                 .       RST    38H
1FA6  FF                 .       RST    38H
1FA7  FF                 .       RST    38H
1FA8  FF                 .       RST    38H
1FA9  FF                 .       RST    38H
1FAA  FF                 .       RST    38H
1FAB  FF                 .       RST    38H
1FAC  FF                 .       RST    38H
1FAD  FF                 .       RST    38H
1FAE  FF                 .       RST    38H
1FAF  FF                 .       RST    38H
1FB0  FF                 .       RST    38H
1FB1  FF                 .       RST    38H
1FB2  FF                 .       RST    38H
1FB3  FF                 .       RST    38H
1FB4  FF                 .       RST    38H
1FB5  FF                 .       RST    38H
1FB6  FF                 .       RST    38H
1FB7  FF                 .       RST    38H
1FB8  FF                 .       RST    38H
1FB9  FF                 .       RST    38H
1FBA  FF                 .       RST    38H
1FBB  FF                 .       RST    38H
1FBC  FF                 .       RST    38H
1FBD  FF                 .       RST    38H
1FBE  FF                 .       RST    38H
1FBF  FF                 .       RST    38H
1FC0  FF                 .       RST    38H
1FC1  FF                 .       RST    38H
1FC2  FF                 .       RST    38H
1FC3  FF                 .       RST    38H
1FC4  FF                 .       RST    38H
1FC5  FF                 .       RST    38H
1FC6  FF                 .       RST    38H
1FC7  FF                 .       RST    38H
1FC8  FF                 .       RST    38H
1FC9  FF                 .       RST    38H
1FCA  FF                 .       RST    38H
1FCB  FF                 .       RST    38H
1FCC  FF                 .       RST    38H
1FCD  FF                 .       RST    38H
1FCE  FF                 .       RST    38H
1FCF  FF                 .       RST    38H
1FD0  FF                 .       RST    38H
1FD1  FF                 .       RST    38H
1FD2  FF                 .       RST    38H
1FD3  FF                 .       RST    38H
1FD4  FF                 .       RST    38H
1FD5  FF                 .       RST    38H
1FD6  FF                 .       RST    38H
1FD7  FF                 .       RST    38H
1FD8  FF                 .       RST    38H
1FD9  FF                 .       RST    38H
1FDA  FF                 .       RST    38H
1FDB  FF                 .       RST    38H
1FDC  FF                 .       RST    38H
1FDD  FF                 .       RST    38H
1FDE  FF                 .       RST    38H
1FDF  FF                 .       RST    38H
1FE0  FF                 .       RST    38H
1FE1  FF                 .       RST    38H
1FE2  FF                 .       RST    38H
1FE3  FF                 .       RST    38H
1FE4  FF                 .       RST    38H
1FE5  FF                 .       RST    38H
1FE6  FF                 .       RST    38H
1FE7  FF                 .       RST    38H
1FE8  FF                 .       RST    38H
1FE9  FF                 .       RST    38H
1FEA  FF                 .       RST    38H
1FEB  FF                 .       RST    38H
1FEC  FF                 .       RST    38H
1FED  FF                 .       RST    38H
1FEE  FF                 .       RST    38H
1FEF  FF                 .       RST    38H
1FF0  FF                 .       RST    38H
1FF1  FF                 .       RST    38H
1FF2  FF                 .       RST    38H
1FF3  FF                 .       RST    38H
1FF4  FF                 .       RST    38H
1FF5  FF                 .       RST    38H
1FF6  FF                 .       RST    38H
1FF7  FF                 .       RST    38H
1FF8  FF                 .       RST    38H
1FF9  FF                 .       RST    38H
1FFA  FF                 .       RST    38H
1FFB  FF                 .       RST    38H
1FFC  FF                 .       RST    38H
1FFD  FF                 .       RST    38H
1FFE  FF                 .       RST    38H
1FFF  FF                 .       RST    38H
